 ConEmuLn

 Timestamp is 5b32b102 (Wed Jun 27 00:32:50 2018)

 Preferred load address is 10000000

 Start         Length     Name                   Class
 0001:00000000 0001293bH .text$mn                CODE
 0001:0001293b 00000000H .text$x                 CODE
 0002:00000000 00000184H .idata$5                DATA
 0002:00000184 00000004H .00cfg                  DATA
 0002:00000188 00000004H .CRT$XCA                DATA
 0002:0000018c 00000004H .CRT$XCZ                DATA
 0002:00000190 00000004H .CRT$XIA                DATA
 0002:00000194 0000000cH .CRT$XIC                DATA
 0002:000001a0 00000004H .CRT$XIZ                DATA
 0002:000001a4 00000004H .CRT$XPA                DATA
 0002:000001a8 00000008H .CRT$XPX                DATA
 0002:000001b0 00000004H .CRT$XPXA               DATA
 0002:000001b4 00000004H .CRT$XPZ                DATA
 0002:000001b8 00000004H .CRT$XTA                DATA
 0002:000001bc 00000004H .CRT$XTZ                DATA
 0002:000001c0 00000000H .gfids$x                DATA
 0002:000001c0 00000000H .gfids$y                DATA
 0002:000001c0 00005bb0H .rdata                  DATA
 0002:00005d68 00000000H .rdata$r                DATA
 0002:00005d70 0000000cH .rdata$sxdata           DATA
 0002:00005d7c 000002d8H .rdata$zzzdbg           DATA
 0002:00006054 00000004H .rtc$IAA                DATA
 0002:00006058 00000004H .rtc$IZZ                DATA
 0002:0000605c 00000004H .rtc$TAA                DATA
 0002:00006060 00000008H .rtc$TZZ                DATA
 0002:00006068 00000398H .xdata$x                DATA
 0002:00006400 0000018cH .edata                  DATA
 0002:0000658c 00000064H .idata$2                DATA
 0002:000065f0 00000014H .idata$3                DATA
 0002:00006604 00000184H .idata$4                DATA
 0002:00006788 0000068aH .idata$6                DATA
 0003:00000000 000008a0H .data                   DATA
 0003:000008a0 00000000H .data$r                 DATA
 0003:000008a0 00001188H .bss                    DATA
 0004:00000000 000000a0H .rsrc$01                DATA
 0004:000000a0 00000498H .rsrc$02                DATA

  Address         Publics by Value              Rva+Base       Lib:Object

 0000:00000000       ___guard_fids_count        00000000     <absolute>
 0000:00000000       ___enclave_config          00000000     <absolute>
 0000:00000000       ___guard_longjmp_count     00000000     <absolute>
 0000:00000000       __except_list              00000000     <absolute>
 0000:00000000       ___guard_longjmp_table     00000000     <absolute>
 0000:00000000       ___guard_iat_table         00000000     <absolute>
 0000:00000000       ___guard_iat_count         00000000     <absolute>
 0000:00000000       ___hybrid_auxiliary_iat    00000000     <absolute>
 0000:00000000       ___hybrid_code_map         00000000     <absolute>
 0000:00000000       ___guard_fids_table        00000000     <absolute>
 0000:00000000       ___hybrid_code_map_count   00000000     <absolute>
 0000:00000000       ___dynamic_value_reloc_table 00000000     <absolute>
 0000:00000003       ___safe_se_handler_count   00000003     <absolute>
 0000:00000100       ___guard_flags             00000100     <absolute>
 0000:00000000       ___ImageBase               10000000     <linker-defined>
 0001:00000000       _ConfigureW@4              10001000 f   ConEmuLn.obj
 0001:00000046       _ExitFARW@0                10001046 f   ConEmuLn.obj
 0001:0000006b       ?ExitFARW3@@YGXPAX@Z       1000106b f   ConEmuLn.obj
 0001:00000099       ?ConfigureW3@@YGHPAX@Z     10001099 f   ConEmuLn.obj
 0001:0000020c       ?ExitPlugin@@YAXXZ         1000120c f   ConEmuLn.obj
 0001:0000024d       ?GetMsgW@@YAPB_WH@Z        1000124d f   ConEmuLn.obj
 0001:0000028d       ?GetPluginInfoWcmn@@YGXPAX@Z 1000128d f   ConEmuLn.obj
 0001:000002be       ?LoadFarVersion@@YAHXZ     100012be f   ConEmuLn.obj
 0001:000005f8       ?OnConEmuLoaded@@YGXPAUConEmuLoadedArg@@@Z 100015f8 f   ConEmuLn.obj
 0001:00000628       ?OpenPluginWcmn@@YAPAXHH@Z 10001628 f   ConEmuLn.obj
 0001:00000655       ?OpenW@@YGPAXPBX@Z         10001655 f   ConEmuLn.obj
 0001:00000680       ?PaintBack@@YAXPAUHDC__@@KUtagRECT@@@Z 10001680 f   ConEmuLn.obj
 0001:000006ce       ?PaintConEmuBackground@@YGHPAUPaintBackgroundArg@@@Z 100016ce f   ConEmuLn.obj
 0001:0000093c       ?PaintLines@@YAXPAUHDC__@@KHHHHH@Z 1000193c f   ConEmuLn.obj
 0001:00000a27       ?SettingsLoad@@YAXXZ       10001a27 f   ConEmuLn.obj
 0001:00000a66       ?SettingsLoadReg@@YAXPB_W@Z 10001a66 f   ConEmuLn.obj
 0001:00000b2b       ?SettingsSave@@YAXXZ       10001b2b f   ConEmuLn.obj
 0001:00000b60       ?SettingsSaveReg@@YAXPB_W@Z 10001b60 f   ConEmuLn.obj
 0001:00000bdf       ?StartPlugin@@YAXH@Z       10001bdf f   ConEmuLn.obj
 0001:00000d2e       ?StringCchCatW@@YGJPA_WIPB_W@Z 10001d2e f i ConEmuLn.obj
 0001:00000d6c       ?StringCchCopyW@@YGJPA_WIPB_W@Z 10001d6c f i ConEmuLn.obj
 0001:00000e82       _DllMain@12                10001e82 f   ConEmuLn.obj
 0001:00000ed9       _GetMinFarVersionW@0       10001ed9 f   ConEmuLn.obj
 0001:00000edf       _SetStartupInfoW@4         10001edf f   ConEmuLn.obj
 0001:00001756       ?ConfigureW1900@@YAHH@Z    10002756 f   ConEmuLn1900.obj
 0001:0000176c       ?ExitFARW1900@@YAXXZ       1000276c f   ConEmuLn1900.obj
 0001:0000179b       ?GetMsgW1900@@YAPB_WH@Z    1000279b f   ConEmuLn1900.obj
 0001:000017c1       ?GetPluginInfoW1900@@YAXPAX@Z 100027c1 f   ConEmuLn1900.obj
 0001:00001825       ?OpenW2800@@YGPAXPBX@Z     10002825 f   ConEmuLn2800.obj
 0001:00001825       ?OpenW1900@@YGPAXPBX@Z     10002825 f   ConEmuLn1900.obj
 0001:00001849       ?SetStartupInfoW1900@@YAXPAX@Z 10002849 f   ConEmuLn1900.obj
 0001:0000193e       ?SettingsLoadW1900@@YAXXZ  1000293e f   ConEmuLn1900.obj
 0001:00001a3a       ?SettingsSaveW1900@@YAXXZ  10002a3a f   ConEmuLn1900.obj
 0001:0000234d       ?ConfigureW2800@@YAHH@Z    1000334d f   ConEmuLn2800.obj
 0001:00002363       ?ExitFARW2800@@YAXXZ       10003363 f   ConEmuLn2800.obj
 0001:00002392       ?GetMsgW2800@@YAPB_WH@Z    10003392 f   ConEmuLn2800.obj
 0001:000023b8       ?GetPluginInfoW2800@@YAXPAX@Z 100033b8 f   ConEmuLn2800.obj
 0001:0000241c       ?SetStartupInfoW2800@@YAXPAX@Z 1000341c f   ConEmuLn2800.obj
 0001:00002511       ?SettingsLoadW2800@@YAXXZ  10003511 f   ConEmuLn2800.obj
 0001:00002603       ?SettingsSaveW2800@@YAXXZ  10003603 f   ConEmuLn2800.obj
 0001:000026d4       _GetGlobalInfoW@4          100036d4 f   ConEmuLn2800.obj
 0001:00002f45       ?ConfigureW995@@YAHH@Z     10003f45 f   ConEmuLn995.obj
 0001:00002f5b       ?ExitFARW995@@YAXXZ        10003f5b f   ConEmuLn995.obj
 0001:00002fa1       ?GetMsgW995@@YAPB_WH@Z     10003fa1 f   ConEmuLn995.obj
 0001:00002fc5       ?GetPluginInfoW995@@YAXPAX@Z 10003fc5 f   ConEmuLn995.obj
 0001:0000301c       ?SetStartupInfoW995@@YAXPAX@Z 1000401c f   ConEmuLn995.obj
 0001:00003159       ?SettingsLoadW995@@YAXXZ   10004159 f   ConEmuLn995.obj
 0001:00003166       ?SettingsSaveW995@@YAXXZ   10004166 f   ConEmuLn995.obj
 0001:00003173       _OpenPluginW@8             10004173 f   ConEmuLn995.obj
 0001:00003a3d       ?SettingsLoadA@@YAXXZ      10004a3d f   ConEmuLnA.obj
 0001:00003a4a       ?SettingsSaveA@@YAXXZ      10004a4a f   ConEmuLnA.obj
 0001:00003a57       _Configure@4               10004a57 f   ConEmuLnA.obj
 0001:00003a74       _ExitFAR@0                 10004a74 f   ConEmuLnA.obj
 0001:00003abf       _GetMinFarVersion@0        10004abf f   ConEmuLnA.obj
 0001:00003ae4       _GetPluginInfo@4           10004ae4 f   ConEmuLnA.obj
 0001:00003b50       _OpenPlugin@8              10004b50 f   ConEmuLnA.obj
 0001:00003b67       _SetStartupInfo@4          10004b67 f   ConEmuLnA.obj
 0001:00003cd1       _GetFileVersionInfoSizeW@8 10004cd1 f   version:VERSION.dll
 0001:00003cd7       _GetFileVersionInfoW@16    10004cd7 f   version:VERSION.dll
 0001:00003cdd       _VerQueryValueW@16         10004cdd f   version:VERSION.dll
 0001:00003ce3       ?StringCchVPrintfW@@YGJPA_WIPB_WPAD@Z 10004ce3 f i common-kernel32:MStrSafe.obj
 0001:00003d3a       ?swprintf_c@@YAHPA_WHPB_WZZ 10004d3a f   common-kernel32:MStrSafe.obj
 0001:00003d5d       ___local_stdio_printf_options 10004d5d f i common-kernel32:MStrSafe.obj
 0001:00003d63       __vsnwprintf_l             10004d63 f i common-kernel32:MStrSafe.obj
 0001:00003d95       ?HeapDeinitialize@@YAXXZ   10004d95 f   common-kernel32:Memory.obj
 0001:00003dad       ?HeapInitialize@@YA_NXZ    10004dad f   common-kernel32:Memory.obj
 0001:00003dcf       ?xf_calloc@@YAPAXII@Z      10004dcf f   common-kernel32:Memory.obj
 0001:00003dea       ?xf_free@@YAXPAX@Z         10004dea f   common-kernel32:Memory.obj
 0001:00003e0a       @__security_check_cookie@4 10004e0a f   LIBCMT:_secchk_.obj
 0001:00003e20       __alloca_probe             10004e20 f   LIBCMT:chkstk.obj
 0001:00003e20       __chkstk                   10004e20 f   LIBCMT:chkstk.obj
 0001:00004159       __DllMainCRTStartup@12     10005159 f   LIBCMT:dll_dllmain.obj
 0001:0000417c       ___raise_securityfailure   1000517c f   LIBCMT:gs_report.obj
 0001:000041a4       ___report_gsfailure        100051a4 f   LIBCMT:gs_report.obj
 0001:000042ee       ___security_init_cookie    100052ee f   LIBCMT:gs_support.obj
 0001:00004339       ?__scrt_initialize_type_info@@YAXXZ 10005339 f   LIBCMT:tncleanup.obj
 0001:00004345       ?__scrt_uninitialize_type_info@@YAXXZ 10005345 f   LIBCMT:tncleanup.obj
 0001:00004351       ___local_stdio_scanf_options 10005351 f i LIBCMT:default_local_stdio_options.obj
 0001:00004357       ___scrt_initialize_default_local_stdio_options 10005357 f   LIBCMT:default_local_stdio_options.obj
 0001:000043b8       ___scrt_acquire_startup_lock 100053b8 f   LIBCMT:utility.obj
 0001:000043ea       ___scrt_dllmain_after_initialize_c 100053ea f   LIBCMT:utility.obj
 0001:00004415       ___scrt_dllmain_before_initialize_c 10005415 f   LIBCMT:utility.obj
 0001:00004423       ___scrt_dllmain_crt_thread_attach 10005423 f   LIBCMT:utility.obj
 0001:00004442       ___scrt_dllmain_crt_thread_detach 10005442 f   LIBCMT:utility.obj
 0001:0000444f       ___scrt_dllmain_exception_filter 1000544f f   LIBCMT:utility.obj
 0001:00004483       ___scrt_dllmain_uninitialize_c 10005483 f   LIBCMT:utility.obj
 0001:000044a6       ___scrt_dllmain_uninitialize_critical 100054a6 f   LIBCMT:utility.obj
 0001:000044b3       ___scrt_initialize_crt     100054b3 f   LIBCMT:utility.obj
 0001:000044ec       ___scrt_initialize_onexit_tables 100054ec f   LIBCMT:utility.obj
 0001:00004596       ___scrt_is_nonwritable_in_current_image 10005596 f   LIBCMT:utility.obj
 0001:00004620       ___scrt_release_startup_lock 10005620 f   LIBCMT:utility.obj
 0001:0000463d       ___scrt_uninitialize_crt   1000563d f   LIBCMT:utility.obj
 0001:00004665       ___scrt_get_dyn_tls_init_callback 10005665 f   LIBCMT:dyn_tls_init.obj
 0001:0000466b       ___scrt_fastfail           1000566b f   LIBCMT:utility_desktop.obj
 0001:00004787       __crt_debugger_hook        10005787 f   LIBCMT:utility_desktop.obj
 0001:0000478f       __RTC_Initialize           1000578f f   LIBCMT:_initsect_.obj
 0001:000047bb       __RTC_Terminate            100057bb f   LIBCMT:_initsect_.obj
 0001:000047f0       __SEH_prolog4              100057f0 f   LIBCMT:_sehprolg4_.obj
 0001:00004836       __SEH_epilog4              10005836 f   LIBCMT:_sehprolg4_.obj
 0001:0000484b       @_guard_check_icall_nop@4  1000584b f i LIBCMT:guard_support.obj
 0001:0000484c       ___isa_available_init      1000584c f   LIBCMT:_cpu_disp_.obj
 0001:000049e5       __get_startup_argv_mode    100059e5 f   LIBCMT:argv_mode.obj
 0001:000049e9       ___scrt_is_ucrt_dll_in_use 100059e9 f   LIBCMT:ucrt_detection.obj
 0001:00004a00       _memmove                   10005a00 f   libvcruntime:memmove.obj
 0001:00004f80       _memset                    10005f80 f   libvcruntime:memset.obj
 0001:00005120       __except_handler4          10006120 f   libvcruntime:_chandler4_.obj
 0001:00005277       ___std_type_info_destroy_list 10006277 f   libvcruntime:std_type_info.obj
 0001:0000529a       ___vcrt_initialize         1000629a f   libvcruntime:initialization.obj
 0001:000052c3       ___vcrt_thread_attach      100062c3 f   libvcruntime:initialization.obj
 0001:000052ce       ___vcrt_thread_detach      100062ce f   libvcruntime:initialization.obj
 0001:000052d9       ___vcrt_uninitialize       100062d9 f   libvcruntime:initialization.obj
 0001:000052f8       ___vcrt_uninitialize_critical 100062f8 f   libvcruntime:initialization.obj
 0001:00005300       __local_unwind4            10006300 f   libvcruntime:_exsup4_.obj
 0001:000053d8       __seh_longjmp_unwind4@4    100063d8 f   libvcruntime:_exsup4_.obj
 0001:00005400       @_EH4_CallFilterFunc@8     10006400 f   libvcruntime:_exsup4_.obj
 0001:00005418       @_EH4_TransferToHandler@8  10006418 f   libvcruntime:_exsup4_.obj
 0001:00005434       @_EH4_GlobalUnwind2@8      10006434 f   libvcruntime:_exsup4_.obj
 0001:00005450       @_EH4_LocalUnwind@16       10006450 f   libvcruntime:_exsup4_.obj
 0001:00005467       ___except_validate_context_record 10006467 f   libvcruntime:jbcxrval.obj
 0001:00005497       ___except_validate_jump_buffer 10006497 f   libvcruntime:jbcxrval.obj
 0001:000054c4       ___vcrt_freefls@4          100064c4 f   libvcruntime:per_thread_data.obj
 0001:000054e0       ___vcrt_freeptd            100064e0 f   libvcruntime:per_thread_data.obj
 0001:00005523       ___vcrt_getptd_noexit      10006523 f   libvcruntime:per_thread_data.obj
 0001:000055b5       ___vcrt_initialize_ptd     100065b5 f   libvcruntime:per_thread_data.obj
 0001:000055f9       ___vcrt_uninitialize_ptd   100065f9 f   libvcruntime:per_thread_data.obj
 0001:00005614       ___vcrt_initialize_locks   10006614 f   libvcruntime:locks.obj
 0001:00005650       ___vcrt_uninitialize_locks 10006650 f   libvcruntime:locks.obj
 0001:0000567f       ??$__crt_fast_encode_pointer@PAX@@YAPAXQAX@Z 1000667f f i libvcruntime:winapi_downlevel.obj
 0001:000057d1       ___vcrt_FlsAlloc           100067d1 f   libvcruntime:winapi_downlevel.obj
 0001:0000580c       ___vcrt_FlsFree            1000680c f   libvcruntime:winapi_downlevel.obj
 0001:00005847       ___vcrt_FlsGetValue        10006847 f   libvcruntime:winapi_downlevel.obj
 0001:00005882       ___vcrt_FlsSetValue        10006882 f   libvcruntime:winapi_downlevel.obj
 0001:000058c0       ___vcrt_InitializeCriticalSectionEx 100068c0 f   libvcruntime:winapi_downlevel.obj
 0001:00005907       ___vcrt_initialize_winapi_thunks 10006907 f   libvcruntime:winapi_downlevel.obj
 0001:00005930       ___vcrt_uninitialize_winapi_thunks 10006930 f   libvcruntime:winapi_downlevel.obj
 0001:00005962       ___vcrt_initialize_pure_virtual_call_handler 10006962 f   libvcruntime:purevirt_data.obj
 0001:00005970       __global_unwind2           10006970 f   libvcruntime:_exsup_.obj
 0001:000059d6       __local_unwind2            100069d6 f   libvcruntime:_exsup_.obj
 0001:00005a5a       __abnormal_termination     10006a5a f   libvcruntime:_exsup_.obj
 0001:00005a80       __NLG_Notify1              10006a80 f   libvcruntime:_exsup_.obj
 0001:00005a8c       __NLG_Notify               10006a8c f   libvcruntime:_exsup_.obj
 0001:00005aa3       __NLG_Dispatch             10006aa3     libvcruntime:_exsup_.obj
 0001:00005aa3       __NLG_Dispatch2            10006aa3     libvcruntime:_exsup_.obj
 0001:00005aab       __NLG_Call                 10006aab f   libvcruntime:_exsup_.obj
 0001:00005aad       __NLG_Return2              10006aad     libvcruntime:_exsup_.obj
 0001:00005ab0       _memcpy                    10006ab0 f   libvcruntime:memcpy.obj
 0001:00006030       __CallSettingFrame@12      10007030 f   libvcruntime:lowhelpr.obj
 0001:00006057       __NLG_Return               10007057     libvcruntime:lowhelpr.obj
 0001:0000607c       ___DestructExceptionObject 1000707c f   libvcruntime:ehhelpers.obj
 0001:00006112       ?_CallMemberFunction0@@YGXQAX0@Z 10007112 f i libvcruntime:ehhelpers.obj
 0001:0000611f       ??$is_overflow_condition@K@__crt_strtox@@YA_NIK@Z 1000711f f i libucrt:strtox.obj
 0001:00006152       ??$make_c_string_character_source@_WPAPA_W@__crt_strtox@@YA?AV?$c_string_character_source@_W@0@QB_WQAPA_W@Z 10007152 f i libucrt:strtox.obj
 0001:00006152       ??$make_c_string_character_source@DPAPAD@__crt_strtox@@YA?AV?$c_string_character_source@D@0@QBDQAPAD@Z 10007152 f i libucrt:strtox.obj
 0001:0000616d       ??$parse_integer@KV?$c_string_character_source@D@__crt_strtox@@@__crt_strtox@@YAKQAU__crt_locale_pointers@@V?$c_string_character_source@D@0@H_N@Z 1000716d f i libucrt:strtox.obj
 0001:00006395       ??$parse_integer@KV?$c_string_character_source@_W@__crt_strtox@@@__crt_strtox@@YAKQAU__crt_locale_pointers@@V?$c_string_character_source@_W@0@H_N@Z 10007395 f i libucrt:strtox.obj
 0001:00006a7a       ??0_LocaleUpdate@@QAE@QAU__crt_locale_pointers@@@Z 10007a7a f i libucrt:strtox.obj
 0001:00006afd       ?unget@?$c_string_character_source@D@__crt_strtox@@QAEXD@Z 10007afd f i libucrt:strtox.obj
 0001:00006b25       ?unget@?$c_string_character_source@_W@__crt_strtox@@QAEX_W@Z 10007b25 f i libucrt:strtox.obj
 0001:00006b51       ?validate@?$c_string_character_source@_W@__crt_strtox@@QBE_NXZ 10007b51 f i libucrt:strtox.obj
 0001:00006b51       ?validate@?$string_output_adapter@_W@__crt_stdio_output@@QBE_NXZ 10007b51 f i libucrt:output.obj
 0001:00006b51       ?validate@?$c_string_character_source@D@__crt_strtox@@QBE_NXZ 10007b51 f i libucrt:strtox.obj
 0001:00006b6c       __chvalidchk_l             10007b6c f i libucrt:strtox.obj
 0001:00006b96       __ischartype_l             10007b96 f i libucrt:strtox.obj
 0001:00006bc9       _strtoul                   10007bc9 f   libucrt:strtox.obj
 0001:00006bf5       _wcstol                    10007bf5 f   libucrt:strtox.obj
 0001:00006c21       _wcstoul                   10007c21 f   libucrt:strtox.obj
 0001:00006dd2       ??$count@D@formatting_buffer@__crt_stdio_output@@QBEIXZ 10007dd2 f i libucrt:output.obj
 0001:00006dea       ??$ensure_buffer_is_big_enough@D@formatting_buffer@__crt_stdio_output@@QAE_NI@Z 10007dea f i libucrt:output.obj
 0001:00006e70       ??$is_wide_character_specifier@_W@__crt_stdio_output@@YA_N_K_WW4length_modifier@0@@Z 10007e70 f i libucrt:output.obj
 0001:00006ebf       ??$scratch_data@D@formatting_buffer@__crt_stdio_output@@QAEPADXZ 10007ebf f i libucrt:output.obj
 0001:00006edd       ??$type_case_integer_parse_into_buffer@I@?$output_processor@_WV?$string_output_adapter@_W@__crt_stdio_output@@V?$standard_base@_WV?$string_output_adapter@_W@__crt_stdio_output@@@2@@__crt_stdio_output@@AAEXII_N@Z 10007edd f i libucrt:output.obj
 0001:00006f52       ??$type_case_integer_parse_into_buffer@_K@?$output_processor@_WV?$string_output_adapter@_W@__crt_stdio_output@@V?$standard_base@_WV?$string_output_adapter@_W@__crt_stdio_output@@@2@@__crt_stdio_output@@AAEX_KI_N@Z 10007f52 f i libucrt:output.obj
 0001:00006fda       ??$write_multiple_characters@V?$string_output_adapter@_W@__crt_stdio_output@@D@__crt_stdio_output@@YAXABV?$string_output_adapter@_W@0@DHQAH@Z 10007fda f i libucrt:output.obj
 0001:0000700b       ??0?$common_data@_W@__crt_stdio_output@@IAE@XZ 1000800b f i libucrt:output.obj
 0001:00007057       ??0?$output_adapter_data@_WV?$string_output_adapter@_W@__crt_stdio_output@@@__crt_stdio_output@@IAE@ABV?$string_output_adapter@_W@1@_KQB_WQAU__crt_locale_pointers@@QAD@Z 10008057 f i libucrt:output.obj
 0001:00007093       ??0?$output_processor@_WV?$string_output_adapter@_W@__crt_stdio_output@@V?$standard_base@_WV?$string_output_adapter@_W@__crt_stdio_output@@@2@@__crt_stdio_output@@QAE@ABV?$string_output_adapter@_W@1@_KQB_WQAU__crt_locale_pointers@@QAD@Z 10008093 f i libucrt:output.obj
 0001:000070c8       ??1formatting_buffer@__crt_stdio_output@@QAE@XZ 100080c8 f i libucrt:output.obj
 0001:000070e2       ??4?$__crt_unique_heap_ptr@DU__crt_internal_free_policy@@@@QAEAAV0@$$QAV0@@Z 100080e2 f i libucrt:output.obj
 0001:00007106       ?crop_zeroes@__crt_stdio_output@@YAXPADQAU__crt_locale_pointers@@@Z 10008106 f i libucrt:output.obj
 0001:0000715d       ?find_next_state@?$output_processor@_WV?$string_output_adapter@_W@__crt_stdio_output@@V?$standard_base@_WV?$string_output_adapter@_W@__crt_stdio_output@@@2@@__crt_stdio_output@@ABE?AW4state@2@_WW432@@Z 1000815d f i libucrt:output.obj
 0001:00007191       ?force_decimal_point@__crt_stdio_output@@YAXPADQAU__crt_locale_pointers@@@Z 10008191 f i libucrt:output.obj
 0001:000071ed       ?parse_int_from_format_string@?$output_processor@_WV?$string_output_adapter@_W@__crt_stdio_output@@V?$standard_base@_WV?$string_output_adapter@_W@__crt_stdio_output@@@2@@__crt_stdio_output@@AAE_NQAH@Z 100081ed f i libucrt:output.obj
 0001:0000724b       ?process@?$output_processor@_WV?$string_output_adapter@_W@__crt_stdio_output@@V?$standard_base@_WV?$string_output_adapter@_W@__crt_stdio_output@@@2@@__crt_stdio_output@@QAEHXZ 1000824b f i libucrt:output.obj
 0001:0000736b       ?state_case_flag@?$output_processor@_WV?$string_output_adapter@_W@__crt_stdio_output@@V?$standard_base@_WV?$string_output_adapter@_W@__crt_stdio_output@@@2@@__crt_stdio_output@@AAE_NXZ 1000836b f i libucrt:output.obj
 0001:000073a8       ?state_case_normal@?$output_processor@_WV?$string_output_adapter@_W@__crt_stdio_output@@V?$standard_base@_WV?$string_output_adapter@_W@__crt_stdio_output@@@2@@__crt_stdio_output@@AAE_NXZ 100083a8 f i libucrt:output.obj
 0001:000073c7       ?state_case_normal_common@?$output_processor@_WV?$string_output_adapter@_W@__crt_stdio_output@@V?$standard_base@_WV?$string_output_adapter@_W@__crt_stdio_output@@@2@@__crt_stdio_output@@AAE_NXZ 100083c7 f i libucrt:output.obj
 0001:000073e2       ?state_case_precision@?$output_processor@_WV?$string_output_adapter@_W@__crt_stdio_output@@V?$standard_base@_WV?$string_output_adapter@_W@__crt_stdio_output@@@2@@__crt_stdio_output@@AAE_NXZ 100083e2 f i libucrt:output.obj
 0001:0000740b       ?state_case_size@?$output_processor@_WV?$string_output_adapter@_W@__crt_stdio_output@@V?$standard_base@_WV?$string_output_adapter@_W@__crt_stdio_output@@@2@@__crt_stdio_output@@AAE_NXZ 1000840b f i libucrt:output.obj
 0001:00007587       ?state_case_type@?$output_processor@_WV?$string_output_adapter@_W@__crt_stdio_output@@V?$standard_base@_WV?$string_output_adapter@_W@__crt_stdio_output@@@2@@__crt_stdio_output@@AAE_NXZ 10008587 f i libucrt:output.obj
 0001:000077e4       ?state_case_width@?$output_processor@_WV?$string_output_adapter@_W@__crt_stdio_output@@V?$standard_base@_WV?$string_output_adapter@_W@__crt_stdio_output@@@2@@__crt_stdio_output@@AAE_NXZ 100087e4 f i libucrt:output.obj
 0001:00007810       ?to_integer_size@__crt_stdio_output@@YAIW4length_modifier@1@@Z 10008810 f i libucrt:output.obj
 0001:0000786c       ?type_case_Z@?$output_processor@_WV?$string_output_adapter@_W@__crt_stdio_output@@V?$standard_base@_WV?$string_output_adapter@_W@__crt_stdio_output@@@2@@__crt_stdio_output@@AAE_NXZ 1000886c f i libucrt:output.obj
 0001:000078cf       ?type_case_a@?$output_processor@_WV?$string_output_adapter@_W@__crt_stdio_output@@V?$standard_base@_WV?$string_output_adapter@_W@__crt_stdio_output@@@2@@__crt_stdio_output@@AAE_NXZ 100088cf f i libucrt:output.obj
 0001:00007a41       ?type_case_c_tchar@?$output_processor@_WV?$string_output_adapter@_W@__crt_stdio_output@@V?$standard_base@_WV?$string_output_adapter@_W@__crt_stdio_output@@@2@@__crt_stdio_output@@AAE_N_W@Z 10008a41 f i libucrt:output.obj
 0001:00007ad9       ?type_case_integer@?$output_processor@_WV?$string_output_adapter@_W@__crt_stdio_output@@V?$standard_base@_WV?$string_output_adapter@_W@__crt_stdio_output@@@2@@__crt_stdio_output@@AAE_NI_N@Z 10008ad9 f i libucrt:output.obj
 0001:00007c23       ?type_case_n@?$output_processor@_WV?$string_output_adapter@_W@__crt_stdio_output@@V?$standard_base@_WV?$string_output_adapter@_W@__crt_stdio_output@@@2@@__crt_stdio_output@@AAE_NXZ 10008c23 f i libucrt:output.obj
 0001:00007c97       ?type_case_o@?$output_processor@_WV?$string_output_adapter@_W@__crt_stdio_output@@V?$standard_base@_WV?$string_output_adapter@_W@__crt_stdio_output@@@2@@__crt_stdio_output@@AAE_NXZ 10008c97 f i libucrt:output.obj
 0001:00007cb6       ?type_case_p@?$output_processor@_WV?$string_output_adapter@_W@__crt_stdio_output@@V?$standard_base@_WV?$string_output_adapter@_W@__crt_stdio_output@@@2@@__crt_stdio_output@@AAE_NXZ 10008cb6 f i libucrt:output.obj
 0001:00007cce       ?type_case_s@?$output_processor@_WV?$string_output_adapter@_W@__crt_stdio_output@@V?$standard_base@_WV?$string_output_adapter@_W@__crt_stdio_output@@@2@@__crt_stdio_output@@AAE_NXZ 10008cce f i libucrt:output.obj
 0001:00007d42       ?type_case_s_compute_narrow_string_length@?$output_processor@_WV?$string_output_adapter@_W@__crt_stdio_output@@V?$standard_base@_WV?$string_output_adapter@_W@__crt_stdio_output@@@2@@__crt_stdio_output@@ABEHH_W@Z 10008d42 f i libucrt:output.obj
 0001:00007d82       ?write_character@?$string_output_adapter@_W@__crt_stdio_output@@QBE_N_WQAH@Z 10008d82 f i libucrt:output.obj
 0001:00007dc7       ?write_stored_string_tchar@?$output_processor@_WV?$string_output_adapter@_W@__crt_stdio_output@@V?$standard_base@_WV?$string_output_adapter@_W@__crt_stdio_output@@@2@@__crt_stdio_output@@AAE_N_W@Z 10008dc7 f i libucrt:output.obj
 0001:00007e52       ?write_string@?$string_output_adapter@_W@__crt_stdio_output@@QBEXQB_WHQAH1@Z 10008e52 f i libucrt:output.obj
 0001:00007eec       ___stdio_common_vswprintf  10008eec f   libucrt:output.obj
 0001:00007f10       _wcsncmp                   10008f10 f   libucrt:wcsncmp.obj
 0001:00007f4a       __initterm                 10008f4a f   libucrt:initterm.obj
 0001:00007fa6       __initterm_e               10008fa6 f   libucrt:initterm.obj
 0001:00007feb       __seh_filter_dll           10008feb f   libucrt:exception_filter.obj
 0001:0000800b       __seh_filter_exe           1000900b f   libucrt:exception_filter.obj
 0001:00008399       ___acrt_initialize_thread_local_exit_callback 10009399 f   libucrt:exit.obj
 0001:000083a8       __cexit                    100093a8 f   libucrt:exit.obj
 0001:000083b7       __exit                     100093b7 f   libucrt:exit.obj
 0001:000083cd       __is_c_termination_complete 100093cd f   libucrt:exit.obj
 0001:0000866c       ___acrt_allocate_buffer_for_argv 1000966c f   libucrt:argv_parsing.obj
 0001:000086c1       __configure_narrow_argv    100096c1 f   libucrt:argv_parsing.obj
 0001:00008825       ??$uninitialize@A6AXAAPAPAD@Z@?$dual_state_global@PAPAD@__crt_state_management@@QAEXA6AXAAPAPAD@Z@Z 10009825 f i libucrt:environment_initialization.obj
 0001:00008825       ??$uninitialize@A6AXAAPAPA_W@Z@?$dual_state_global@PAPA_W@__crt_state_management@@QAEXA6AXAAPAPA_W@Z@Z 10009825 f i libucrt:environment_initialization.obj
 0001:0000889b       ?initialize@?$dual_state_global@PAU__crt_locale_data@@@__crt_state_management@@QAEXQAU__crt_locale_data@@@Z 1000989b f i libucrt:initialization.obj
 0001:0000889b       ?initialize@?$dual_state_global@P6AHI@Z@__crt_state_management@@QAEXQ6AHI@Z@Z 1000989b f i libucrt:new_handler.obj
 0001:0000889b       ?initialize@?$dual_state_global@P6AXH@Z@__crt_state_management@@QAEXQ6AXH@Z@Z 1000989b f i libucrt:signal.obj
 0001:0000889b       ?initialize@?$dual_state_global@P6AXPB_W00II@Z@__crt_state_management@@QAEXQ6AXPB_W00II@Z@Z 1000989b f i libucrt:invalid_parameter.obj
 0001:0000889b       ?initialize@?$dual_state_global@PAPAD@__crt_state_management@@QAEXQAPAD@Z 1000989b f i libucrt:environment_initialization.obj
 0001:0000889b       ?initialize@?$dual_state_global@P6AHPAU_exception@@@Z@__crt_state_management@@QAEXQ6AHPAU_exception@@@Z@Z 1000989b f i libucrt:matherr.obj
 0001:000088cc       ___dcrt_uninitialize_environments_nolock 100098cc f   libucrt:environment_initialization.obj
 0001:00008903       __initialize_narrow_environment 10009903 f   libucrt:environment_initialization.obj
 0001:00008908       ??$?RV<lambda_995298e7d72eb4c2aab26c0585b3abe5>@@AAV<lambda_275893d493268fdec8709772e3fcec0e>@@V<lambda_293819299cbf9a7022e18b56a874bb5c>@@@?$__crt_seh_guarded_call@H@@QAEH$$QAV<lambda_995298e7d72eb4c2aab26c0585b3abe5>@@AAV<lambda_275893d493268fdec8709772e3fcec0e>@@$$QAV<lambda_293819299cbf9a7022e18b56a874bb5c>@@@Z 10009908 f i libucrt:onexit.obj
 0001:00008959       ??$__acrt_lock_and_call@V<lambda_275893d493268fdec8709772e3fcec0e>@@@@YAHW4__acrt_lock_id@@$$QAV<lambda_275893d493268fdec8709772e3fcec0e>@@@Z 10009959 f i libucrt:onexit.obj
 0001:00008aa1       __execute_onexit_table     10009aa1 f   libucrt:onexit.obj
 0001:00008abe       __initialize_onexit_table  10009abe f   libucrt:onexit.obj
 0001:00008b27       ___acrt_uninitialize_command_line 10009b27 f   libucrt:argv_data.obj
 0001:00008bef       ___acrt_initialize         10009bef f   libucrt:initialization.obj
 0001:00008c01       ___acrt_thread_attach      10009c01 f   libucrt:initialization.obj
 0001:00008c0c       ___acrt_thread_detach      10009c0c f   libucrt:initialization.obj
 0001:00008c14       ___acrt_uninitialize       10009c14 f   libucrt:initialization.obj
 0001:00008c26       ___acrt_uninitialize_critical 10009c26 f   libucrt:initialization.obj
 0001:00008c38       _terminate                 10009c38 f   libucrt:terminate.obj
 0001:00008c74       _free                      10009c74 f   libucrt:free.obj
 0001:00008c79       _strcpy_s                  10009c79 f   libucrt:strcpy_s.obj
 0001:00008ce0       _strncmp                   10009ce0 f   libucrt:strncmp.obj
 0001:00008d58       _abort                     10009d58 f   libucrt:abort.obj
 0001:00008d9b       _calloc                    10009d9b f   libucrt:calloc.obj
 0001:00008da6       ___acrt_call_reportfault   10009da6 f   libucrt:invalid_parameter.obj
 0001:00008ee1       ___acrt_initialize_invalid_parameter_handler 10009ee1 f   libucrt:invalid_parameter.obj
 0001:00008ef5       __invalid_parameter        10009ef5 f   libucrt:invalid_parameter.obj
 0001:00008f70       __invalid_parameter_noinfo 10009f70 f   libucrt:invalid_parameter.obj
 0001:00008f80       __invoke_watson            10009f80 f   libucrt:invalid_parameter.obj
 0001:00008fb3       ___acrt_errno_from_os_error 10009fb3 f   libucrt:errno.obj
 0001:00008ff6       ___acrt_errno_map_os_error 10009ff6 f   libucrt:errno.obj
 0001:00009019       ___doserrno                1000a019 f   libucrt:errno.obj
 0001:0000902c       __errno                    1000a02c f   libucrt:errno.obj
 0001:0000903f       ___pctype_func             1000a03f f   libucrt:ctype.obj
 0001:00009065       _iswctype                  1000a065 f   libucrt:iswctype.obj
 0001:000090c4       __isctype_l                1000a0c4 f   libucrt:isctype.obj
 0001:00009196       ??$?RV<lambda_3518db117f0e7cdb002338c5d3c47b6c>@@AAV<lambda_b2ea41f6bbb362cd97d94c6828d90b61>@@V<lambda_abdedf541bb04549bc734292b4a045d4>@@@?$__crt_seh_guarded_call@X@@QAEX$$QAV<lambda_3518db117f0e7cdb002338c5d3c47b6c>@@AAV<lambda_b2ea41f6bbb362cd97d94c6828d90b61>@@$$QAV<lambda_abdedf541bb04549bc734292b4a045d4>@@@Z 1000a196 f i libucrt:per_thread_data.obj
 0001:000091e6       ??$?RV<lambda_51b6e8b1eb166f2a3faf91f424b38130>@@AAV<lambda_6250bd4b2a391816dd638c3bf72b0bcb>@@V<lambda_0b5a4a3e68152e1d9b943535f5f47bed>@@@?$__crt_seh_guarded_call@X@@QAEX$$QAV<lambda_51b6e8b1eb166f2a3faf91f424b38130>@@AAV<lambda_6250bd4b2a391816dd638c3bf72b0bcb>@@$$QAV<lambda_0b5a4a3e68152e1d9b943535f5f47bed>@@@Z 1000a1e6 f i libucrt:per_thread_data.obj
 0001:00009247       ??$?RV<lambda_5b71d36f03204c0beab531769a5b5694>@@AAV<lambda_be2b3da3f62db62e9dad5dc70221a656>@@V<lambda_8f9ce462984622f9bf76b59e2aaaf805>@@@?$__crt_seh_guarded_call@X@@QAEX$$QAV<lambda_5b71d36f03204c0beab531769a5b5694>@@AAV<lambda_be2b3da3f62db62e9dad5dc70221a656>@@$$QAV<lambda_8f9ce462984622f9bf76b59e2aaaf805>@@@Z 1000a247 f i libucrt:per_thread_data.obj
 0001:00009292       ??$?RV<lambda_9df27f884b057bc3edfc946cb5b7cf47>@@AAV<lambda_e69574bed617af4e071282c136b37893>@@V<lambda_cc0d902bcbbeb830f749456577db4721>@@@?$__crt_seh_guarded_call@X@@QAEX$$QAV<lambda_9df27f884b057bc3edfc946cb5b7cf47>@@AAV<lambda_e69574bed617af4e071282c136b37893>@@$$QAV<lambda_cc0d902bcbbeb830f749456577db4721>@@@Z 1000a292 f i libucrt:per_thread_data.obj
 0001:000092da       ??$__acrt_lock_and_call@V<lambda_6250bd4b2a391816dd638c3bf72b0bcb>@@@@YAXW4__acrt_lock_id@@$$QAV<lambda_6250bd4b2a391816dd638c3bf72b0bcb>@@@Z 1000a2da f i libucrt:per_thread_data.obj
 0001:00009302       ??$__acrt_lock_and_call@V<lambda_b2ea41f6bbb362cd97d94c6828d90b61>@@@@YAXW4__acrt_lock_id@@$$QAV<lambda_b2ea41f6bbb362cd97d94c6828d90b61>@@@Z 1000a302 f i libucrt:per_thread_data.obj
 0001:0000932a       ??$__acrt_lock_and_call@V<lambda_be2b3da3f62db62e9dad5dc70221a656>@@@@YAXW4__acrt_lock_id@@$$QAV<lambda_be2b3da3f62db62e9dad5dc70221a656>@@@Z 1000a32a f i libucrt:per_thread_data.obj
 0001:00009352       ??$__acrt_lock_and_call@V<lambda_e69574bed617af4e071282c136b37893>@@@@YAXW4__acrt_lock_id@@$$QAV<lambda_e69574bed617af4e071282c136b37893>@@@Z 1000a352 f i libucrt:per_thread_data.obj
 0001:00009508       ___acrt_freeptd            1000a508 f   libucrt:per_thread_data.obj
 0001:00009534       ___acrt_getptd             1000a534 f   libucrt:per_thread_data.obj
 0001:000095b8       ___acrt_getptd_noexit      1000a5b8 f   libucrt:per_thread_data.obj
 0001:0000963d       ___acrt_initialize_ptd     1000a63d f   libucrt:per_thread_data.obj
 0001:00009669       ___acrt_uninitialize_ptd   1000a669 f   libucrt:per_thread_data.obj
 0001:00009683       ___acrt_update_locale_info 1000a683 f   libucrt:locale_update.obj
 0001:000096b0       ___acrt_update_multibyte_info 1000a6b0 f   libucrt:locale_update.obj
 0001:000096dd       ___acrt_set_locale_changed 1000a6dd f   libucrt:wsetlocale.obj
 0001:000096e8       ___acrt_uninitialize_locale 1000a6e8 f   libucrt:wsetlocale.obj
 0001:0000973a       __isdigit_l                1000a73a f i libucrt:_ctype.obj
 0001:00009772       _isdigit                   1000a772 f i libucrt:_ctype.obj
 0001:00009906       __tolower_l                1000a906 f   libucrt:tolower_toupper.obj
 0001:00009920       _tolower                   1000a920 f   libucrt:tolower_toupper.obj
 0001:00009950       __free_base                1000a950 f   libucrt:free_base.obj
 0001:0000998a       __malloc_base              1000a98a f   libucrt:malloc_base.obj
 0001:000099d8       __mbtowc_l                 1000a9d8 f   libucrt:mbtowc.obj
 0001:00009ad2       _mbtowc                    1000aad2 f   libucrt:mbtowc.obj
 0001:00009aec       _wcsnlen                   1000aaec f   libucrt:strnlen.obj
 0001:00009ca3       ?__acrt_fp_classify@@YA?AW4__acrt_fp_class@@ABN@Z 1000aca3 f i libucrt:cvt.obj
 0001:00009d0f       ?__acrt_fp_is_negative@@YA_NABN@Z 1000ad0f f i libucrt:cvt.obj
 0001:0000a56e       ___acrt_fp_format          1000b56e f   libucrt:cvt.obj
 0001:0000a6b8       __fileno                   1000b6b8 f   libucrt:fileno.obj
 0001:0000a6de       ___acrt_initialize_stdio   1000b6de f   libucrt:_file.obj
 0001:0000a7a6       ___acrt_uninitialize_stdio 1000b7a6 f   libucrt:_file.obj
 0001:0000a7f2       __lock_file                1000b7f2 f   libucrt:_file.obj
 0001:0000a806       __unlock_file              1000b806 f   libucrt:_file.obj
 0001:0000a81a       __get_printf_count_output  1000b81a f   libucrt:printf_count_output.obj
 0001:0000a99b       ___acrt_initialize_lowio   1000b99b f   libucrt:ioinit.obj
 0001:0000a9f1       ___acrt_uninitialize_lowio 1000b9f1 f   libucrt:ioinit.obj
 0001:0000aa1d       ___acrt_initialize_locks   1000ba1d f   libucrt:locks.obj
 0001:0000aa5e       ___acrt_lock               1000ba5e f   libucrt:locks.obj
 0001:0000aa75       ___acrt_uninitialize_locks 1000ba75 f   libucrt:locks.obj
 0001:0000aaa6       ___acrt_unlock             1000baa6 f   libucrt:locks.obj
 0001:0000abd4       ___acrt_FlsAlloc@4         1000bbd4 f   libucrt:winapi_thunks.obj
 0001:0000ac2a       ___acrt_FlsFree@4          1000bc2a f   libucrt:winapi_thunks.obj
 0001:0000ac80       ___acrt_FlsGetValue@4      1000bc80 f   libucrt:winapi_thunks.obj
 0001:0000acd6       ___acrt_FlsSetValue@8      1000bcd6 f   libucrt:winapi_thunks.obj
 0001:0000ad2f       ___acrt_InitializeCriticalSectionEx@12 1000bd2f f   libucrt:winapi_thunks.obj
 0001:0000ad91       ___acrt_LCMapStringEx@36   1000bd91 f   libucrt:winapi_thunks.obj
 0001:0000ae19       ___acrt_LocaleNameToLCID@8 1000be19 f   libucrt:winapi_thunks.obj
 0001:0000ae75       ___acrt_initialize_winapi_thunks 1000be75 f   libucrt:winapi_thunks.obj
 0001:0000ae9b       ___acrt_is_packaged_app    1000be9b f   libucrt:winapi_thunks.obj
 0001:0000af22       ___acrt_uninitialize_winapi_thunks 1000bf22 f   libucrt:winapi_thunks.obj
 0001:0000af58       __calloc_base              1000bf58 f   libucrt:calloc_base.obj
 0001:0000b377       ??1?$argument_list@D@?A0xb0e4b824@@QAE@XZ 1000c377 f i libucrt:argv_wildcards.obj
 0001:0000b39c       ?append@?$argument_list@D@?A0xb0e4b824@@QAEHQAD@Z 1000c39c f i libucrt:argv_wildcards.obj
 0001:0000b3d1       ?expand_if_necessary@?$argument_list@D@?A0xb0e4b824@@AAEHXZ 1000c3d1 f i libucrt:argv_wildcards.obj
 0001:0000b458       ___acrt_expand_narrow_argv_wildcards 1000c458 f   libucrt:argv_wildcards.obj
 0001:0000b463       ??$?RV<lambda_978dc153c237d78434369da87b74ff60>@@AAV<lambda_ad1ced32f4ac17aa236e5ef05d6b3b7c>@@V<lambda_4a8533e2866a575feecb8298ce776b0d>@@@?$__crt_seh_guarded_call@X@@QAEX$$QAV<lambda_978dc153c237d78434369da87b74ff60>@@AAV<lambda_ad1ced32f4ac17aa236e5ef05d6b3b7c>@@$$QAV<lambda_4a8533e2866a575feecb8298ce776b0d>@@@Z 1000c463 f i libucrt:mbctype.obj
 0001:0000b4a6       ??$__acrt_lock_and_call@V<lambda_ad1ced32f4ac17aa236e5ef05d6b3b7c>@@@@YAXW4__acrt_lock_id@@$$QAV<lambda_ad1ced32f4ac17aa236e5ef05d6b3b7c>@@@Z 1000c4a6 f i libucrt:mbctype.obj
 0001:0000b93d       ___acrt_initialize_multibyte 1000c93d f   libucrt:mbctype.obj
 0001:0000b95b       ___acrt_update_thread_multibyte_data 1000c95b f   libucrt:mbctype.obj
 0001:0000b9fd       __setmbcp_nolock           1000c9fd f   libucrt:mbctype.obj
 0001:0000bcc8       __ismbblead                1000ccc8 f   libucrt:ismbbyte.obj
 0001:0000bce0       ___acrt_initialize_command_line 1000cce0 f   libucrt:argv_data.obj
 0001:0000bd30       ___dcrt_get_narrow_environment_from_os 1000cd30 f   libucrt:get_environment_from_os.obj
 0001:0000bdb3       __recalloc                 1000cdb3 f   libucrt:recalloc.obj
 0001:0000bdbe       __recalloc_base            1000cdbe f   libucrt:recalloc.obj
 0001:0000be2b       ___acrt_initialize_heap    1000ce2b f   libucrt:heap_handle.obj
 0001:0000be3c       ___acrt_uninitialize_heap  1000ce3c f   libucrt:heap_handle.obj
 0001:0000be46       ___acrt_execute_initializers 1000ce46 f   libucrt:shared_initialization.obj
 0001:0000bec9       ___acrt_execute_uninitializers 1000cec9 f   libucrt:shared_initialization.obj
 0001:0000bf16       ___acrt_initialize_new_handler 1000cf16 f   libucrt:new_handler.obj
 0001:0000bf2a       __callnewh                 1000cf2a f   libucrt:new_handler.obj
 0001:0000bf6e       __query_new_handler        1000cf6e f   libucrt:new_handler.obj
 0001:0000bfc0       ??$?RV<lambda_a048d3beccc847880fc8490e18b82769>@@AAV<lambda_ec61778202f4f5fc7e7711acc23c3bca>@@V<lambda_f7496a158712204296dd6628a163878e>@@@?$__crt_seh_guarded_call@P6AXH@Z@@QAEP6AXH@Z$$QAV<lambda_a048d3beccc847880fc8490e18b82769>@@AAV<lambda_ec61778202f4f5fc7e7711acc23c3bca>@@$$QAV<lambda_f7496a158712204296dd6628a163878e>@@@Z 1000cfc0 f i libucrt:signal.obj
 0001:0000c01a       ??$__acrt_lock_and_call@V<lambda_ec61778202f4f5fc7e7711acc23c3bca>@@@@YAP6AXH@ZW4__acrt_lock_id@@$$QAV<lambda_ec61778202f4f5fc7e7711acc23c3bca>@@@Z 1000d01a f i libucrt:signal.obj
 0001:0000c0ac       ___acrt_get_sigabrt_handler 1000d0ac f   libucrt:signal.obj
 0001:0000c0c3       ___acrt_initialize_signal_handlers 1000d0c3 f   libucrt:signal.obj
 0001:0000c0fe       ___fpecode                 1000d0fe f   libucrt:signal.obj
 0001:0000c107       _raise                     1000d107 f   libucrt:signal.obj
 0001:0000c30f       ___acrt_has_user_matherr   1000d30f f   libucrt:matherr.obj
 0001:0000c328       ___acrt_initialize_user_matherr 1000d328 f   libucrt:matherr.obj
 0001:0000c33c       ___acrt_invoke_user_matherr 1000d33c f   libucrt:matherr.obj
 0001:0000c385       __isleadbyte_l             1000d385 f i libucrt:_wctype.obj
 0001:0000c3be       ___acrt_GetStringTypeA     1000d3be f   libucrt:getstringtypea.obj
 0001:0000c4db       __freea_crt                1000d4db f i libucrt:getstringtypea.obj
 0001:0000c4fb       ___acrt_add_locale_ref     1000d4fb f   libucrt:locale_refcounting.obj
 0001:0000c578       ___acrt_free_locale        1000d578 f   libucrt:locale_refcounting.obj
 0001:0000c6c2       ___acrt_locale_add_lc_time_reference 1000d6c2 f   libucrt:locale_refcounting.obj
 0001:0000c6eb       ___acrt_locale_free_lc_time_if_unreferenced 1000d6eb f   libucrt:locale_refcounting.obj
 0001:0000c71b       ___acrt_locale_release_lc_time_reference 1000d71b f   libucrt:locale_refcounting.obj
 0001:0000c744       ___acrt_release_locale_ref 1000d744 f   libucrt:locale_refcounting.obj
 0001:0000c7c5       ___acrt_update_thread_locale_data 1000d7c5 f   libucrt:locale_refcounting.obj
 0001:0000c83c       __updatetlocinfoEx_nolock  1000d83c f   libucrt:locale_refcounting.obj
 0001:0000c88c       ___acrt_locale_free_monetary 1000d88c f   libucrt:initmon.obj
 0001:0000c98a       ___acrt_locale_free_numeric 1000d98a f   libucrt:initnum.obj
 0001:0000ca2f       ___acrt_locale_free_time   1000da2f f   libucrt:inittime.obj
 0001:0000cd30       ___acrt_LCMapStringA       1000dd30 f   libucrt:lcmapstringa.obj
 0001:0000cd7b       __query_new_mode           1000dd7b f   libucrt:new_mode.obj
 0001:0000cd81       ___acrt_fp_strflt_to_string 1000dd81 f   libucrt:_fptostr.obj
 0001:0000ce3d       ??0scoped_fp_state_reset@?A0x48fbfdd4@@QAE@XZ 1000de3d f i libucrt:cfout.obj
 0001:0000ce70       ?divide@__crt_strtox@@YA_KAAUbig_integer@1@ABU21@@Z 1000de70 f i libucrt:cfout.obj
 0001:0000d31e       ___acrt_fltout             1000e31e f   libucrt:cfout.obj
 0001:0000e6ba       __fcloseall                1000f6ba f   libucrt:closeall.obj
 0001:0000e75a       ___acrt_stdio_flush_nolock 1000f75a f   libucrt:fflush.obj
 0001:0000e7c0       __fflush_nolock            1000f7c0 f   libucrt:fflush.obj
 0001:0000e807       __flushall                 1000f807 f   libucrt:fflush.obj
 0001:0000e8e8       ___acrt_stdio_free_buffer_nolock 1000f8e8 f   libucrt:_freebuf.obj
 0001:0000e926       __isatty                   1000f926 f   libucrt:isatty.obj
 0001:0000e97c       ___acrt_lowio_create_handle_array 1000f97c f   libucrt:osfinfo.obj
 0001:0000e9f6       ___acrt_lowio_destroy_handle_array 1000f9f6 f   libucrt:osfinfo.obj
 0001:0000ea2b       ___acrt_lowio_ensure_fh_exists 1000fa2b f   libucrt:osfinfo.obj
 0001:0000eac3       ___acrt_lowio_lock_fh      1000fac3 f   libucrt:osfinfo.obj
 0001:0000eae6       ___acrt_lowio_unlock_fh    1000fae6 f   libucrt:osfinfo.obj
 0001:0000eb09       __free_osfhnd              1000fb09 f   libucrt:osfinfo.obj
 0001:0000eb9a       __get_osfhandle            1000fb9a f   libucrt:osfinfo.obj
 0001:0000ecc0       ___acrt_DownlevelLocaleNameToLCID 1000fcc0 f   libucrt:lcidtoname_downlevel.obj
 0001:0000edd0       _qsort                     1000fdd0 f   libucrt:qsort.obj
 0001:0000f21b       _strncpy_s                 1001021b f   libucrt:strncpy_s.obj
 0001:0000f230       _strpbrk                   10010230 f   libucrt:strpbrk.obj
 0001:0000f270       __mbsdec                   10010270 f   libucrt:mbsdec.obj
 0001:0000f287       __mbsdec_l                 10010287 f   libucrt:mbsdec.obj
 0001:0000f323       __msize                    10010323 f   libucrt:msize.obj
 0001:0000f356       __realloc_base             10010356 f   libucrt:realloc_base.obj
 0001:0000f3bf       ___strncnt                 100103bf f   libucrt:strncnt.obj
 0001:0000f3db       _fegetenv                  100103db f   libucrt:fegetenv.obj
 0001:0000f3f8       _fesetenv                  100103f8 f   libucrt:fesetenv.obj
 0001:0000f441       _feholdexcept              10010441 f   libucrt:feholdexcept.obj
 0001:0000f490       _log10                     10010490 f   libucrt:log10.obj
 0001:0000f4d0       __CIlog10                  100104d0 f   libucrt:log10.obj
 0001:0000f50b       __CIlog10_default          1001050b f   libucrt:log10.obj
 0001:0000f51f       __log10_default            1001051f     libucrt:log10.obj
 0001:0000f5e0       _ceil                      100105e0 f   libucrt:ceil_pentium4.obj
 0001:0000f620       __ceil_pentium4            10010620 f   libucrt:ceil_pentium4.obj
 0001:0000fc8d       __write                    10010c8d f   libucrt:write.obj
 0001:0000fd78       __write_nolock             10010d78 f   libucrt:write.obj
 0001:00010002       __lseeki64_nolock          10011002 f   libucrt:lseek.obj
 0001:0001001d       __fclose_nolock            1001101d f   libucrt:fclose.obj
 0001:00010093       _fclose                    10011093 f   libucrt:fclose.obj
 0001:00010113       ??$?RV<lambda_61cee617f5178ae960314fd4d05640a0>@@AAV<lambda_6978c1fb23f02e42e1d9e99668cc68aa>@@V<lambda_9cd88cf8ad10232537feb2133f08c833>@@@?$__crt_seh_guarded_call@H@@QAEH$$QAV<lambda_61cee617f5178ae960314fd4d05640a0>@@AAV<lambda_6978c1fb23f02e42e1d9e99668cc68aa>@@$$QAV<lambda_9cd88cf8ad10232537feb2133f08c833>@@@Z 10011113 f i libucrt:commit.obj
 0001:000101ab       ??$__acrt_lowio_lock_fh_and_call@V<lambda_6978c1fb23f02e42e1d9e99668cc68aa>@@@@YAHH$$QAV<lambda_6978c1fb23f02e42e1d9e99668cc68aa>@@@Z 100111ab f i libucrt:commit.obj
 0001:000101d3       __commit                   100111d3 f   libucrt:commit.obj
 0001:00010242       __query_app_type           10011242 f   libucrt:report_runtime_error.obj
 0001:000104eb       __getfpcontrolword         100114eb f   libucrt:_fenvutils.obj
 0001:0001052e       __getfpstatusword          1001152e f   libucrt:_fenvutils.obj
 0001:000105d6       __setfpcontrolword         100115d6 f   libucrt:_fenvutils.obj
 0001:00010656       __setfpstatusword          10011656 f   libucrt:_fenvutils.obj
 0001:000106d6       __clearfp                  100116d6 f   libucrt:ieee87.obj
 0001:000107b4       ___acrt_initialize_sse2    100117b4 f   libucrt:mathfcns.obj
 0001:000107d0       __CIlog10_pentium4         100117d0 f   libucrt:log10_pentium4.obj
 0001:000107e8       __log10_pentium4           100117e8     libucrt:log10_pentium4.obj
 0001:00010a71       __fFEXP                    10011a71     libucrt:87tran.obj
 0001:00010ac8       __rtinfpopse               10011ac8     libucrt:87tran.obj
 0001:00010aca       __rtinfnpopse              10011aca     libucrt:87tran.obj
 0001:00010ada       __fFLN                     10011ada     libucrt:87tran.obj
 0001:00010b8f       __rtinfpop                 10011b8f     libucrt:87tran.obj
 0001:00010b91       __rtinfnpop                10011b91     libucrt:87tran.obj
 0001:00010bae       __ffexpm1                  10011bae     libucrt:87tran.obj
 0001:00010c60       __trandisp1                10011c60 f   libucrt:87disp.obj
 0001:00010cc7       __trandisp2                10011cc7 f   libucrt:87disp.obj
 0001:00010d53       __rttospopde               10011d53     libucrt:87disp.obj
 0001:00010d58       __rttospop                 10011d58     libucrt:87disp.obj
 0001:00010d5a       __rtnospop                 10011d5a     libucrt:87disp.obj
 0001:00010d5c       __rttosnpop                10011d5c     libucrt:87disp.obj
 0001:00010d5d       __rtnospopde               10011d5d     libucrt:87disp.obj
 0001:00010d64       __rtzeropop                10011d64     libucrt:87disp.obj
 0001:00010d66       __rtzeronpop               10011d66     libucrt:87disp.obj
 0001:00010d6b       __rtzerospop               10011d6b     libucrt:87disp.obj
 0001:00010d78       __rtonepop                 10011d78     libucrt:87disp.obj
 0001:00010d7a       __rtonenpop                10011d7a     libucrt:87disp.obj
 0001:00010d7f       __tosnan1                  10011d7f     libucrt:87disp.obj
 0001:00010daa       __nosnan2                  10011daa     libucrt:87disp.obj
 0001:00010dac       __tosnan2                  10011dac     libucrt:87disp.obj
 0001:00010dd4       __nan2                     10011dd4     libucrt:87disp.obj
 0001:00010e13       __rtindfpop                10011e13     libucrt:87disp.obj
 0001:00010e15       __rtindfnpop               10011e15     libucrt:87disp.obj
 0001:00010e26       __rttosnpopde              10011e26     libucrt:87disp.obj
 0001:00010e30       __rtatan2inf               10011e30     libucrt:87disp.obj
 0001:00010e4d       __rtchsifneg               10011e4d     libucrt:87disp.obj
 0001:00010e60       __twoToTOS                 10011e60 f   libucrt:common.obj
 0001:00010e75       __load_CW                  10011e75 f   libucrt:common.obj
 0001:00010e8c       __convertTOStoQNaN         10011e8c f   libucrt:common.obj
 0001:00010ea5       __fload_withFB             10011ea5 f   libucrt:common.obj
 0001:00010ee8       __checkTOS_withFB          10011ee8 f   libucrt:common.obj
 0001:00010efe       __fast_exit                10011efe f   libucrt:common.obj
 0001:00010f0b       __math_exit                10011f0b f   libucrt:common.obj
 0001:00010f35       __check_overflow_exit      10011f35 f   libucrt:common.obj
 0001:00010f49       __check_range_exit         10011f49 f   libucrt:common.obj
 0001:00010ff0       __startTwoArgErrorHandling 10011ff0 f   libucrt:genexcep.obj
 0001:00011007       __startOneArgErrorHandling 10012007 f   libucrt:genexcep.obj
 0001:00011043       ___libm_error_support      10012043 f   libucrt:libm_error.obj
 0001:0001125b       __ceil_default             1001225b f   libucrt:ceil.obj
 0001:00011314       __putwch_nolock            10012314 f   libucrt:putwch.obj
 0001:00011359       ??$?RV<lambda_123407a5e2ac06da108355a851863b7a>@@AAV<lambda_2fe9b910cf3cbf4a0ab98a02ba45b3ec>@@V<lambda_ae55bdf541ad94d75914d381c370e64d>@@@?$__crt_seh_guarded_call@H@@QAEH$$QAV<lambda_123407a5e2ac06da108355a851863b7a>@@AAV<lambda_2fe9b910cf3cbf4a0ab98a02ba45b3ec>@@$$QAV<lambda_ae55bdf541ad94d75914d381c370e64d>@@@Z 10012359 f i libucrt:close.obj
 0001:000113db       ??$__acrt_lowio_lock_fh_and_call@V<lambda_2fe9b910cf3cbf4a0ab98a02ba45b3ec>@@@@YAHH$$QAV<lambda_2fe9b910cf3cbf4a0ab98a02ba45b3ec>@@@Z 100123db f i libucrt:close.obj
 0001:00011403       __close                    10012403 f   libucrt:close.obj
 0001:00011482       __close_nolock             10012482 f   libucrt:close.obj
 0001:0001151e       ?__acrt_stdio_free_stream@@YAXV__crt_stdio_stream@@@Z 1001251e f   libucrt:stream.obj
 0001:00011560       ___ascii_strnicmp          10012560 f   libucrt:_strnicm.obj
 0001:000115c1       __clrfp                    100125c1 f   libucrt:fpctrl.obj
 0001:000115d4       __ctrlfp                   100125d4 f   libucrt:fpctrl.obj
 0001:00011600       __set_statfp               10012600 f   libucrt:fpctrl.obj
 0001:0001165b       __statfp                   1001265b f   libucrt:fpctrl.obj
 0001:0001166d       __d_inttype                1001266d f   libucrt:powhlp.obj
 0001:000116d7       __powhlp                   100126d7 f   libucrt:powhlp.obj
 0001:00011802       __87except                 10012802 f   libucrt:87except.obj
 0001:0001190d       __frnd                     1001290d f   libucrt:frnd.obj
 0001:00011923       __errcode                  10012923 f   libucrt:fpexcept.obj
 0001:00011957       __except1                  10012957 f   libucrt:fpexcept.obj
 0001:00011a25       __handle_exc               10012a25 f   libucrt:fpexcept.obj
 0001:00011c05       __raise_exc                10012c05 f   libucrt:fpexcept.obj
 0001:00011c28       __raise_exc_ex             10012c28 f   libucrt:fpexcept.obj
 0001:00011f19       __set_errno_from_matherr   10012f19 f   libucrt:fpexcept.obj
 0001:00011f48       __umatherr                 10012f48 f   libucrt:fpexcept.obj
 0001:00011fea       __decomp                   10012fea f   libucrt:util.obj
 0001:000120be       __set_exp                  100130be f   libucrt:util.obj
 0001:000120ed       __sptype                   100130ed f   libucrt:util.obj
 0001:0001214b       ___dcrt_lowio_initialize_console_output 1001314b f   libucrt:initcon.obj
 0001:0001216a       ___dcrt_terminate_console_output 1001316a f   libucrt:initcon.obj
 0001:00012181       __fpclass                  10013181 f   libucrt:ieeemisc.obj
 0001:00012225       _IsProcessorFeaturePresent@4 10013225 f   kernel32:KERNEL32.dll
 0001:00012230       __FindPESection            10013230 f   LIBCMT:pesect.obj
 0001:00012280       __IsNonwritableInCurrentImage 10013280 f   LIBCMT:pesect.obj
 0001:00012340       __ValidateImageBase        10013340 f   LIBCMT:pesect.obj
 0001:00012380       __aulldvrm                 10013380 f   LIBCMT:ulldvrm.obj
 0001:00012420       __allmul                   10013420 f   LIBCMT:llmul.obj
 0001:00012460       __SEH_prolog4_GS           10013460 f   LIBCMT:_sehprolg4gs_.obj
 0001:000124a9       __SEH_epilog4_GS           100134a9 f   LIBCMT:_sehprolg4gs_.obj
 0001:000124c0       __alldvrm                  100134c0 f   LIBCMT:lldvrm.obj
 0001:000125a0       __aullshr                  100135a0 f   LIBCMT:ullshr.obj
 0001:000125c0       __alloca_probe_16          100135c0 f   LIBCMT:alloca16.obj
 0001:000125d6       __alloca_probe_8           100135d6     LIBCMT:alloca16.obj
 0001:000125f0       __allshl                   100135f0 f   LIBCMT:llshl.obj
 0001:00012610       __ftol2_sse                10013610 f   LIBCMT:_ftol2_.obj
 0001:00012619       __ftol2_pentium4           10013619 f   LIBCMT:_ftol2_.obj
 0001:0001262c       __ftol2_sse_excpt          1001362c f   LIBCMT:_ftol2_.obj
 0001:00012650       __ftol2                    10013650 f   LIBCMT:_ftol2_.obj
 0001:000126d0       _strrchr                   100136d0 f   libvcruntime:strrchr.obj
 0001:00012810       _strchr                    10013810 f   libvcruntime:strchr.obj
 0001:0001287e       ___from_strstr_to_strchr   1001387e     libvcruntime:strchr.obj
 0002:00000000       __imp__RegQueryValueExW@24 10014000     advapi32:ADVAPI32.dll
 0002:00000004       __imp__RegOpenKeyExW@20    10014004     advapi32:ADVAPI32.dll
 0002:00000008       __imp__RegCreateKeyExW@36  10014008     advapi32:ADVAPI32.dll
 0002:0000000c       __imp__RegCloseKey@4       1001400c     advapi32:ADVAPI32.dll
 0002:00000010       __imp__RegSetValueExW@24   10014010     advapi32:ADVAPI32.dll
 0002:00000014       \177ADVAPI32_NULL_THUNK_DATA 10014014     advapi32:ADVAPI32.dll
 0002:00000018       __imp__SelectObject@8      10014018     gdi32:GDI32.dll
 0002:0000001c       __imp__LineTo@12           1001401c     gdi32:GDI32.dll
 0002:00000020       __imp__DeleteObject@4      10014020     gdi32:GDI32.dll
 0002:00000024       __imp__CreateSolidBrush@4  10014024     gdi32:GDI32.dll
 0002:00000028       __imp__CreatePen@12        10014028     gdi32:GDI32.dll
 0002:0000002c       __imp__MoveToEx@16         1001402c     gdi32:GDI32.dll
 0002:00000030       \177GDI32_NULL_THUNK_DATA  10014030     gdi32:GDI32.dll
 0002:00000034       __imp__MultiByteToWideChar@24 10014034     kernel32:KERNEL32.dll
 0002:00000038       __imp__lstrlenA@4          10014038     kernel32:KERNEL32.dll
 0002:0000003c       __imp__WriteConsoleW@20    1001403c     kernel32:KERNEL32.dll
 0002:00000040       __imp__DecodePointer@4     10014040     kernel32:KERNEL32.dll
 0002:00000044       __imp__FlushFileBuffers@4  10014044     kernel32:KERNEL32.dll
 0002:00000048       __imp__lstrcpyA@8          10014048     kernel32:KERNEL32.dll
 0002:0000004c       __imp__lstrcpynA@12        1001404c     kernel32:KERNEL32.dll
 0002:00000050       __imp__lstrcpynW@12        10014050     kernel32:KERNEL32.dll
 0002:00000054       __imp__GetModuleFileNameW@12 10014054     kernel32:KERNEL32.dll
 0002:00000058       __imp__lstrlenW@4          10014058     kernel32:KERNEL32.dll
 0002:0000005c       __imp__GetLastError@0      1001405c     kernel32:KERNEL32.dll
 0002:00000060       __imp__lstrcpyW@8          10014060     kernel32:KERNEL32.dll
 0002:00000064       __imp__VirtualProtect@16   10014064     kernel32:KERNEL32.dll
 0002:00000068       __imp__CloseHandle@4       10014068     kernel32:KERNEL32.dll
 0002:0000006c       __imp__DeleteCriticalSection@4 1001406c     kernel32:KERNEL32.dll
 0002:00000070       __imp__DebugBreak@0        10014070     kernel32:KERNEL32.dll
 0002:00000074       __imp__HeapCreate@12       10014074     kernel32:KERNEL32.dll
 0002:00000078       __imp__HeapDestroy@4       10014078     kernel32:KERNEL32.dll
 0002:0000007c       __imp__HeapAlloc@12        1001407c     kernel32:KERNEL32.dll
 0002:00000080       __imp__HeapReAlloc@16      10014080     kernel32:KERNEL32.dll
 0002:00000084       __imp__HeapFree@12         10014084     kernel32:KERNEL32.dll
 0002:00000088       __imp__UnhandledExceptionFilter@4 10014088     kernel32:KERNEL32.dll
 0002:0000008c       __imp__SetUnhandledExceptionFilter@4 1001408c     kernel32:KERNEL32.dll
 0002:00000090       __imp__GetCurrentProcess@0 10014090     kernel32:KERNEL32.dll
 0002:00000094       __imp__TerminateProcess@8  10014094     kernel32:KERNEL32.dll
 0002:00000098       __imp__IsProcessorFeaturePresent@4 10014098     kernel32:KERNEL32.dll
 0002:0000009c       __imp__QueryPerformanceCounter@4 1001409c     kernel32:KERNEL32.dll
 0002:000000a0       __imp__GetCurrentProcessId@0 100140a0     kernel32:KERNEL32.dll
 0002:000000a4       __imp__GetCurrentThreadId@0 100140a4     kernel32:KERNEL32.dll
 0002:000000a8       __imp__GetSystemTimeAsFileTime@4 100140a8     kernel32:KERNEL32.dll
 0002:000000ac       __imp__InitializeSListHead@4 100140ac     kernel32:KERNEL32.dll
 0002:000000b0       __imp__IsDebuggerPresent@0 100140b0     kernel32:KERNEL32.dll
 0002:000000b4       __imp__GetStartupInfoW@4   100140b4     kernel32:KERNEL32.dll
 0002:000000b8       __imp__GetModuleHandleW@4  100140b8     kernel32:KERNEL32.dll
 0002:000000bc       __imp__InterlockedFlushSList@4 100140bc     kernel32:KERNEL32.dll
 0002:000000c0       __imp__RtlUnwind@16        100140c0     kernel32:KERNEL32.dll
 0002:000000c4       __imp__SetLastError@4      100140c4     kernel32:KERNEL32.dll
 0002:000000c8       __imp__EnterCriticalSection@4 100140c8     kernel32:KERNEL32.dll
 0002:000000cc       __imp__LeaveCriticalSection@4 100140cc     kernel32:KERNEL32.dll
 0002:000000d0       __imp__CreateFileW@28      100140d0     kernel32:KERNEL32.dll
 0002:000000d4       __imp__InitializeCriticalSectionAndSpinCount@8 100140d4     kernel32:KERNEL32.dll
 0002:000000d8       __imp__TlsAlloc@0          100140d8     kernel32:KERNEL32.dll
 0002:000000dc       __imp__TlsGetValue@4       100140dc     kernel32:KERNEL32.dll
 0002:000000e0       __imp__TlsSetValue@8       100140e0     kernel32:KERNEL32.dll
 0002:000000e4       __imp__TlsFree@4           100140e4     kernel32:KERNEL32.dll
 0002:000000e8       __imp__FreeLibrary@4       100140e8     kernel32:KERNEL32.dll
 0002:000000ec       __imp__GetProcAddress@8    100140ec     kernel32:KERNEL32.dll
 0002:000000f0       __imp__LoadLibraryExW@12   100140f0     kernel32:KERNEL32.dll
 0002:000000f4       __imp__RaiseException@16   100140f4     kernel32:KERNEL32.dll
 0002:000000f8       __imp__ExitProcess@4       100140f8     kernel32:KERNEL32.dll
 0002:000000fc       __imp__GetModuleHandleExW@12 100140fc     kernel32:KERNEL32.dll
 0002:00000100       __imp__GetModuleFileNameA@12 10014100     kernel32:KERNEL32.dll
 0002:00000104       __imp__WideCharToMultiByte@32 10014104     kernel32:KERNEL32.dll
 0002:00000108       __imp__GetStringTypeW@16   10014108     kernel32:KERNEL32.dll
 0002:0000010c       __imp__GetACP@0            1001410c     kernel32:KERNEL32.dll
 0002:00000110       __imp__GetStdHandle@4      10014110     kernel32:KERNEL32.dll
 0002:00000114       __imp__GetFileType@4       10014114     kernel32:KERNEL32.dll
 0002:00000118       __imp__LCMapStringW@24     10014118     kernel32:KERNEL32.dll
 0002:0000011c       __imp__FindClose@4         1001411c     kernel32:KERNEL32.dll
 0002:00000120       __imp__FindFirstFileExA@24 10014120     kernel32:KERNEL32.dll
 0002:00000124       __imp__FindNextFileA@8     10014124     kernel32:KERNEL32.dll
 0002:00000128       __imp__IsValidCodePage@4   10014128     kernel32:KERNEL32.dll
 0002:0000012c       __imp__GetOEMCP@0          1001412c     kernel32:KERNEL32.dll
 0002:00000130       __imp__GetCPInfo@8         10014130     kernel32:KERNEL32.dll
 0002:00000134       __imp__GetCommandLineA@0   10014134     kernel32:KERNEL32.dll
 0002:00000138       __imp__GetCommandLineW@0   10014138     kernel32:KERNEL32.dll
 0002:0000013c       __imp__GetEnvironmentStringsW@0 1001413c     kernel32:KERNEL32.dll
 0002:00000140       __imp__FreeEnvironmentStringsW@4 10014140     kernel32:KERNEL32.dll
 0002:00000144       __imp__GetProcessHeap@0    10014144     kernel32:KERNEL32.dll
 0002:00000148       __imp__SetStdHandle@8      10014148     kernel32:KERNEL32.dll
 0002:0000014c       __imp__HeapSize@12         1001414c     kernel32:KERNEL32.dll
 0002:00000150       __imp__WriteFile@20        10014150     kernel32:KERNEL32.dll
 0002:00000154       __imp__GetConsoleCP@0      10014154     kernel32:KERNEL32.dll
 0002:00000158       __imp__GetConsoleMode@8    10014158     kernel32:KERNEL32.dll
 0002:0000015c       __imp__SetFilePointerEx@20 1001415c     kernel32:KERNEL32.dll
 0002:00000160       \177KERNEL32_NULL_THUNK_DATA 10014160     kernel32:KERNEL32.dll
 0002:00000164       __imp__wsprintfW           10014164     user32:USER32.dll
 0002:00000168       __imp__FillRect@12         10014168     user32:USER32.dll
 0002:0000016c       __imp__wsprintfA           1001416c     user32:USER32.dll
 0002:00000170       \177USER32_NULL_THUNK_DATA 10014170     user32:USER32.dll
 0002:00000174       __imp__VerQueryValueW@16   10014174     version:VERSION.dll
 0002:00000178       __imp__GetFileVersionInfoW@16 10014178     version:VERSION.dll
 0002:0000017c       __imp__GetFileVersionInfoSizeW@8 1001417c     version:VERSION.dll
 0002:00000180       \177VERSION_NULL_THUNK_DATA 10014180     version:VERSION.dll
 0002:00000184       ___guard_check_icall_fptr  10014184     LIBCMT:guard_support.obj
 0002:00000188       ___xc_a                    10014188     LIBCMT:initializers.obj
 0002:0000018c       ___xc_z                    1001418c     LIBCMT:initializers.obj
 0002:00000190       ___xi_a                    10014190     LIBCMT:initializers.obj
 0002:00000194       ___acrt_stdio_initializer  10014194     libucrt:stdio_initializer.obj
 0002:00000198       ___acrt_multibyte_initializer 10014198     libucrt:multibyte_initializer.obj
 0002:0000019c       ___acrt_tran_sse2_initializer 1001419c     libucrt:sse2_initializer.obj
 0002:000001a0       ___xi_z                    100141a0     LIBCMT:initializers.obj
 0002:000001a4       ___xp_a                    100141a4     LIBCMT:initializers.obj
 0002:000001a8       ___acrt_locale_terminator  100141a8     libucrt:locale_initializer.obj
 0002:000001ac       ___dcrt_console_output_terminator 100141ac     libucrt:console_output_initializer.obj
 0002:000001b0       ___acrt_stdio_terminator   100141b0     libucrt:stdio_initializer.obj
 0002:000001b4       ___xp_z                    100141b4     LIBCMT:initializers.obj
 0002:000001b8       ___xt_a                    100141b8     LIBCMT:initializers.obj
 0002:000001bc       ___xt_z                    100141bc     LIBCMT:initializers.obj
 0002:000001c0       ??_C@_1BM@GCLEPEKO@?$AAP?$AAl?$AAu?$AAg?$AAi?$AAn?$AAE?$AAn?$AAa?$AAb?$AAl?$AAe?$AAd?$AA?$AA@ 100141c0     ConEmuLn.obj
 0002:000001dc       ??_C@_1BG@GKMEIIHO@?$AAL?$AAi?$AAn?$AAe?$AAs?$AAP?$AAa?$AAn?$AAe?$AAl?$AA?$AA@ 100141dc     ConEmuLn.obj
 0002:000001f4       ??_C@_1BG@FMPDIDHG@?$AAL?$AAi?$AAn?$AAe?$AAs?$AAC?$AAo?$AAl?$AAo?$AAr?$AA?$AA@ 100141f4     ConEmuLn.obj
 0002:0000020c       ??_C@_1BI@DNACCAMK@?$AAL?$AAi?$AAn?$AAe?$AAs?$AAE?$AAd?$AAi?$AAt?$AAo?$AAr?$AA?$AA@ 1001420c     ConEmuLn.obj
 0002:00000224       ??_C@_1CC@LODMIFLF@?$AAL?$AAi?$AAn?$AAe?$AAs?$AAE?$AAd?$AAi?$AAt?$AAo?$AAr?$AAC?$AAo?$AAl?$AAo?$AAr?$AA?$AA@ 10014224     ConEmuLn.obj
 0002:00000248       ??_C@_1BI@IMFGPMJI@?$AAL?$AAi?$AAn?$AAe?$AAs?$AAV?$AAi?$AAe?$AAw?$AAe?$AAr?$AA?$AA@ 10014248     ConEmuLn.obj
 0002:00000260       ??_C@_1CC@KGIANIMF@?$AAL?$AAi?$AAn?$AAe?$AAs?$AAV?$AAi?$AAe?$AAw?$AAe?$AAr?$AAC?$AAo?$AAl?$AAo?$AAr?$AA?$AA@ 10014260     ConEmuLn.obj
 0002:00000284       ??_C@_1BI@PPOFOFEE@?$AAH?$AAi?$AAl?$AAi?$AAg?$AAh?$AAt?$AAT?$AAy?$AAp?$AAe?$AA?$AA@ 10014284     ConEmuLn.obj
 0002:0000029c       ??_C@_1BO@FGCOGFB@?$AAH?$AAi?$AAl?$AAi?$AAg?$AAh?$AAt?$AAP?$AAl?$AAu?$AAg?$AAi?$AAn?$AAs?$AA?$AA@ 1001429c     ConEmuLn.obj
 0002:000002bc       ??_C@_1CA@GLKFLGCI@?$AAH?$AAi?$AAl?$AAi?$AAg?$AAh?$AAt?$AAP?$AAl?$AAu?$AAg?$AAB?$AAa?$AAc?$AAk?$AA?$AA@ 100142bc     ConEmuLn.obj
 0002:000002dc       ??_C@_08BCACMCCB@ExitFARW?$AA@ 100142dc     ConEmuLn.obj
 0002:000002e8       ??_C@_0L@DJCGGOCO@ConfigureW?$AA@ 100142e8     ConEmuLn.obj
 0002:000002f4       ??_C@_11LOCGONAA@?$AA?$AA@ 100142f4     ConEmuLn.obj
 0002:000002f8       ??_C@_13FPGAJAPJ@?$AA?2?$AA?$AA@ 100142f8     ConEmuLn.obj
 0002:00000300       ??_C@_1FG@DPPGENBC@?$AAL?$AAo?$AAa?$AAd?$AAA?$AAp?$AAp?$AAV?$AAe?$AAr?$AAs?$AAi?$AAo?$AAn?$AA?4?$AAV?$AAe?$AAr?$AAQ?$AAu?$AAe?$AAr?$AAy?$AAV?$AAa?$AAl?$AAu?$AAe?$AA?$CI?$AA?$CC?$AA?2?$AA?$CC@ 10014300     ConEmuLn.obj
 0002:00000358       ??_C@_1FK@HILEEFML@?$AAL?$AAo?$AAa?$AAd?$AAA?$AAp?$AAp?$AAV?$AAe?$AAr?$AAs?$AAi?$AAo?$AAn?$AA?4?$AAG?$AAe?$AAt?$AAF?$AAi?$AAl?$AAe?$AAV?$AAe?$AAr?$AAs?$AAi?$AAo?$AAn?$AAI?$AAn?$AAf@ 10014358     ConEmuLn.obj
 0002:000003b8       ??_C@_1GC@BINFLBDC@?$AAL?$AAo?$AAa?$AAd?$AAA?$AAp?$AAp?$AAV?$AAe?$AAr?$AAs?$AAi?$AAo?$AAn?$AA?5?$AAf?$AAa?$AAi?$AAl?$AAe?$AAd?$AA?$CB?$AA?5?$AAC?$AAa?$AAn?$AA?8?$AAt?$AA?5?$AAa?$AAl?$AAl@ 100143b8     ConEmuLn.obj
 0002:00000420       ??_C@_1GC@CPPHDKJK@?$AAL?$AAo?$AAa?$AAd?$AAA?$AAp?$AAp?$AAV?$AAe?$AAr?$AAs?$AAi?$AAo?$AAn?$AA?4?$AAG?$AAe?$AAt?$AAF?$AAi?$AAl?$AAe?$AAV?$AAe?$AAr?$AAs?$AAi?$AAo?$AAn?$AAI?$AAn?$AAf@ 10014420     ConEmuLn.obj
 0002:00000488       ??_C@_1EG@IINOBDEG@?$AAI?$AAn?$AAv?$AAa?$AAl?$AAi?$AAd?$AA?5?$AAa?$AAs?$AAM?$AAo?$AAd?$AAu?$AAl?$AAe?$AAP?$AAa?$AAt?$AAh?$AA?5?$AAw?$AAa?$AAs?$AA?5?$AAs?$AAp?$AAe?$AAc?$AAi?$AAf?$AAi@ 10014488     ConEmuLn.obj
 0002:000004d0       ??_C@_1CA@GGFPMHLH@?$AA?6?$AAE?$AAr?$AAr?$AAC?$AAo?$AAd?$AAe?$AA?$DN?$AA0?$AAx?$AA?$CF?$AA0?$AA8?$AAX?$AA?$AA@ 100144d0     ConEmuLn.obj
 0002:000004f0       ??_C@_1FG@LNADFPCE@?$AAL?$AAo?$AAa?$AAd?$AAF?$AAa?$AAr?$AAV?$AAe?$AAr?$AAs?$AAi?$AAo?$AAn?$AA?4?$AAG?$AAe?$AAt?$AAM?$AAo?$AAd?$AAu?$AAl?$AAe?$AAF?$AAi?$AAl?$AAe?$AAN?$AAa?$AAm?$AAe@ 100144f0     ConEmuLn.obj
 0002:00000548       ??_C@_1BC@KLDFICIN@?$AA0?$AAx?$AAX?$AAX?$AAX?$AAX?$AAX?$AAX?$AA?$AA@ 10014548     ConEmuLn1900.obj
 0002:0000055c       ??_C@_19OMFGMPJN@?$AA?$CF?$AA0?$AA6?$AAX?$AA?$AA@ 1001455c     ConEmuLn1900.obj
 0002:00000570       __xmm@00000000000000030000000500000008 10014570     ConEmuLn1900.obj
 0002:00000580       __xmm@00000000000000050000000500000009 10014580     ConEmuLn1900.obj
 0002:00000590       __xmm@00000000000000070000000500000008 10014590     ConEmuLn1900.obj
 0002:000005a0       __xmm@00000000000000080000000500000008 100145a0     ConEmuLn1900.obj
 0002:000005b0       __xmm@00000000000000090000000500000008 100145b0     ConEmuLn1900.obj
 0002:000005c0       __xmm@000000000000000b0000000500000008 100145c0     ConEmuLn1900.obj
 0002:000005d0       __xmm@000000000000000c0000000500000000 100145d0     ConEmuLn1900.obj
 0002:000005e0       __xmm@000000000000000e0000000000000000 100145e0     ConEmuLn1900.obj
 0002:000005f0       __xmm@000000000000000f0000000000000007 100145f0     ConEmuLn1900.obj
 0002:00000600       __xmm@00000024000000070000001d00000006 10014600     ConEmuLn1900.obj
 0002:00000610       __xmm@00000024000000080000001d00000006 10014610     ConEmuLn1900.obj
 0002:00000620       __xmm@00000024000000090000001d00000006 10014620     ConEmuLn1900.obj
 0002:00000630       __xmm@000000240000000c0000001d00000006 10014630     ConEmuLn1900.obj
 0002:00000640       __xmm@00000026000000010000000300000003 10014640     ConEmuLn1900.obj
 0002:00000650       ??_C@_1CE@PCHJHFGJ@?$AAC?$AAo?$AAn?$AAE?$AAm?$AAu?$AA?5?$AAU?$AAn?$AAd?$AAe?$AAr?$AAl?$AAi?$AAn?$AAe?$AAs?$AA?$AA@ 10014650     ConEmuLn2800.obj
 0002:00000678       ??_C@_1GC@KMIACAL@?$AAP?$AAa?$AAi?$AAn?$AAt?$AA?5?$AAu?$AAn?$AAd?$AAe?$AAr?$AAl?$AAi?$AAn?$AAe?$AAd?$AA?5?$AAb?$AAa?$AAc?$AAk?$AAg?$AAr?$AAo?$AAu?$AAn?$AAd?$AA?5?$AAi?$AAn?$AA?5?$AAt@ 10014678     ConEmuLn2800.obj
 0002:000006dc       ??_C@_1DE@DJEAMLPH@?$AAC?$AAo?$AAn?$AAE?$AAm?$AAu?$AA?4?$AAM?$AAa?$AAx?$AAi?$AAm?$AAu?$AAs?$AA5?$AA?$EA?$AAg?$AAm?$AAa?$AAi?$AAl?$AA?4?$AAc?$AAo?$AAm?$AA?$AA@ 100146dc     ConEmuLn2800.obj
 0002:00000710       ??_C@_1BE@MMJMCNIO@?$AAC?$AAo?$AAn?$AAE?$AAm?$AAu?$AAL?$AAn?$AA?2?$AA?$AA@ 10014710     ConEmuLn995.obj
 0002:00000724       ??_C@_08KOICIHPP@0xXXXXXX?$AA@ 10014724     ConEmuLnA.obj
 0002:00000730       ??_C@_04JCFDBOEJ@?$CF06X?$AA@ 10014730     ConEmuLnA.obj
 0002:00000738       __pRawDllMain              10014738     LIBCMT:dll_dllmain.obj
 0002:00000738       __pDefaultRawDllMain       10014738     LIBCMT:dll_dllmain.obj
 0002:000008e0       ??_C@_08EHJDFFNH@__based?$CI?$AA@ 100148e0     libvcruntime:undname.obj
 0002:000008ec       ??_C@_07KOLFKCDI@__cdecl?$AA@ 100148ec     libvcruntime:undname.obj
 0002:000008f4       ??_C@_08GHMPAG@__pascal?$AA@ 100148f4     libvcruntime:undname.obj
 0002:00000900       ??_C@_09IFJBGAPI@__stdcall?$AA@ 10014900     libvcruntime:undname.obj
 0002:0000090c       ??_C@_0L@NPHFGOKO@__thiscall?$AA@ 1001490c     libvcruntime:undname.obj
 0002:00000918       ??_C@_0L@JMKHOMEK@__fastcall?$AA@ 10014918     libvcruntime:undname.obj
 0002:00000924       ??_C@_0N@BCKKPABJ@__vectorcall?$AA@ 10014924     libvcruntime:undname.obj
 0002:00000934       ??_C@_09HIJEGCPM@__clrcall?$AA@ 10014934     libvcruntime:undname.obj
 0002:00000940       ??_C@_06GHPCKEAG@__eabi?$AA@ 10014940     libvcruntime:undname.obj
 0002:00000948       ??_C@_07EECFKIPL@__swift?$AA@ 10014948     libvcruntime:undname.obj
 0002:00000950       ??_C@_07JOMMBBKO@__ptr64?$AA@ 10014950     libvcruntime:undname.obj
 0002:00000958       ??_C@_0L@PILCLIHE@__restrict?$AA@ 10014958     libvcruntime:undname.obj
 0002:00000964       ??_C@_0M@GFIIJFMG@__unaligned?$AA@ 10014964     libvcruntime:undname.obj
 0002:00000970       ??_C@_09DHDLOLLB@restrict?$CI?$AA@ 10014970     libvcruntime:undname.obj
 0002:0000097a       ??_C@_00CNPNBAHC@?$AA@     1001497a     libvcruntime:undname.obj
 0002:0000097c       ??_C@_04NIHEBCM@?5new?$AA@ 1001497c     libvcruntime:undname.obj
 0002:00000984       ??_C@_07FPCDHGMM@?5delete?$AA@ 10014984     libvcruntime:undname.obj
 0002:0000098c       ??_C@_01NEMOKFLO@?$DN?$AA@ 1001498c     libvcruntime:undname.obj
 0002:00000990       ??_C@_02GPIOPFAK@?$DO?$DO?$AA@ 10014990     libvcruntime:undname.obj
 0002:00000994       ??_C@_02FODMEDOG@?$DM?$DM?$AA@ 10014994     libvcruntime:undname.obj
 0002:00000998       ??_C@_01DCLJPIOD@?$CB?$AA@ 10014998     libvcruntime:undname.obj
 0002:0000099c       ??_C@_02EGOFBIJA@?$DN?$DN?$AA@ 1001499c     libvcruntime:undname.obj
 0002:000009a0       ??_C@_02FDNJECIE@?$CB?$DN?$AA@ 100149a0     libvcruntime:undname.obj
 0002:000009a4       ??_C@_02GPECMEKF@?$FL?$FN?$AA@ 100149a4     libvcruntime:undname.obj
 0002:000009a8       ??_C@_08LHJFAFGD@operator?$AA@ 100149a8     libvcruntime:undname.obj
 0002:000009b4       ??_C@_02HBOOOICD@?9?$DO?$AA@ 100149b4     libvcruntime:undname.obj
 0002:000009b8       ??_C@_01NBENCBCI@?$CK?$AA@ 100149b8     libvcruntime:undname.obj
 0002:000009bc       ??_C@_02ECNGHCIF@?$CL?$CL?$AA@ 100149bc     libvcruntime:undname.obj
 0002:000009c0       ??_C@_02BAABKJLB@?9?9?$AA@ 100149c0     libvcruntime:undname.obj
 0002:000009c4       ??_C@_01JOAMLHOP@?9?$AA@   100149c4     libvcruntime:undname.obj
 0002:000009c8       ??_C@_01MIFGBAGJ@?$CL?$AA@ 100149c8     libvcruntime:undname.obj
 0002:000009cc       ??_C@_01HNPIGOCE@?$CG?$AA@ 100149cc     libvcruntime:undname.obj
 0002:000009d0       ??_C@_03MNHNFDLC@?9?$DO?$CK?$AA@ 100149d0     libvcruntime:undname.obj
 0002:000009d4       ??_C@_01KMDKNFGN@?1?$AA@   100149d4     libvcruntime:undname.obj
 0002:000009d8       ??_C@_01FGNFDNOH@?$CF?$AA@ 100149d8     libvcruntime:undname.obj
 0002:000009dc       ??_C@_01MNNFJEPP@?$DM?$AA@ 100149dc     libvcruntime:undname.obj
 0002:000009e0       ??_C@_02EHCHHCKH@?$DM?$DN?$AA@ 100149e0     libvcruntime:undname.obj
 0002:000009e4       ??_C@_01PPODPGHN@?$DO?$AA@ 100149e4     libvcruntime:undname.obj
 0002:000009e8       ??_C@_02EEKDKGMJ@?$DO?$DN?$AA@ 100149e8     libvcruntime:undname.obj
 0002:000009ec       ??_C@_01IHBHIGKO@?0?$AA@   100149ec     libvcruntime:undname.obj
 0002:000009f0       ??_C@_02HCKGKOFO@?$CI?$CJ?$AA@ 100149f0     libvcruntime:undname.obj
 0002:000009f4       ??_C@_01PJKLJHI@?$HO?$AA@  100149f4     libvcruntime:undname.obj
 0002:000009f8       ??_C@_01JKBOJNNK@?$FO?$AA@ 100149f8     libvcruntime:undname.obj
 0002:000009fc       ??_C@_01DNKMNLPK@?$HM?$AA@ 100149fc     libvcruntime:undname.obj
 0002:00000a00       ??_C@_02PPKAJPJL@?$CG?$CG?$AA@ 10014a00     libvcruntime:undname.obj
 0002:00000a04       ??_C@_02NONPIBCD@?$HM?$HM?$AA@ 10014a04     libvcruntime:undname.obj
 0002:00000a08       ??_C@_02FPIMKNGF@?$CK?$DN?$AA@ 10014a08     libvcruntime:undname.obj
 0002:00000a0c       ??_C@_02FOEOMHFC@?$CL?$DN?$AA@ 10014a0c     libvcruntime:undname.obj
 0002:00000a10       ??_C@_02FKMDLLOA@?9?$DN?$AA@ 10014a10     libvcruntime:undname.obj
 0002:00000a14       ??_C@_02FJEHGPIO@?1?$DN?$AA@ 10014a14     libvcruntime:undname.obj
 0002:00000a18       ??_C@_02FENAOKFI@?$CF?$DN?$AA@ 10014a18     libvcruntime:undname.obj
 0002:00000a1c       ??_C@_03IKFCCPFF@?$DO?$DO?$DN?$AA@ 10014a1c     libvcruntime:undname.obj
 0002:00000a20       ??_C@_03CDNPDDLA@?$DM?$DM?$DN?$AA@ 10014a20     libvcruntime:undname.obj
 0002:00000a24       ??_C@_02FGJGFEAB@?$CG?$DN?$AA@ 10014a24     libvcruntime:undname.obj
 0002:00000a28       ??_C@_02DHLNPPGH@?$HM?$DN?$AA@ 10014a28     libvcruntime:undname.obj
 0002:00000a2c       ??_C@_02MHEGNOJ@?$FO?$DN?$AA@ 10014a2c     libvcruntime:undname.obj
 0002:00000a30       ??_C@_09IFPLHPGF@?$GAvftable?8?$AA@ 10014a30     libvcruntime:undname.obj
 0002:00000a3c       ??_C@_09BLBHBJP@?$GAvbtable?8?$AA@ 10014a3c     libvcruntime:undname.obj
 0002:00000a48       ??_C@_07FEEIOKP@?$GAvcall?8?$AA@ 10014a48     libvcruntime:undname.obj
 0002:00000a50       ??_C@_08LLFFHHDJ@?$GAtypeof?8?$AA@ 10014a50     libvcruntime:undname.obj
 0002:00000a5c       ??_C@_0BF@KDPPACIK@?$GAlocal?5static?5guard?8?$AA@ 10014a5c     libvcruntime:undname.obj
 0002:00000a74       ??_C@_08OBABFOLI@?$GAstring?8?$AA@ 10014a74     libvcruntime:undname.obj
 0002:00000a80       ??_C@_0BD@JDLKDPAB@?$GAvbase?5destructor?8?$AA@ 10014a80     libvcruntime:undname.obj
 0002:00000a94       ??_C@_0BN@DEGPLNFK@?$GAvector?5deleting?5destructor?8?$AA@ 10014a94     libvcruntime:undname.obj
 0002:00000ab4       ??_C@_0BO@OBMKPJIG@?$GAdefault?5constructor?5closure?8?$AA@ 10014ab4     libvcruntime:undname.obj
 0002:00000ad4       ??_C@_0BN@IMDCHIKM@?$GAscalar?5deleting?5destructor?8?$AA@ 10014ad4     libvcruntime:undname.obj
 0002:00000af4       ??_C@_0BO@PFGOCPJJ@?$GAvector?5constructor?5iterator?8?$AA@ 10014af4     libvcruntime:undname.obj
 0002:00000b14       ??_C@_0BN@LFPFMEDL@?$GAvector?5destructor?5iterator?8?$AA@ 10014b14     libvcruntime:undname.obj
 0002:00000b34       ??_C@_0CE@IKBNEHA@?$GAvector?5vbase?5constructor?5iterat@ 10014b34     libvcruntime:undname.obj
 0002:00000b58       ??_C@_0BL@NILFHHPC@?$GAvirtual?5displacement?5map?8?$AA@ 10014b58     libvcruntime:undname.obj
 0002:00000b74       ??_C@_0CB@JONCMFFK@?$GAeh?5vector?5constructor?5iterator?8@ 10014b74     libvcruntime:undname.obj
 0002:00000b98       ??_C@_0CA@GCEOPDGL@?$GAeh?5vector?5destructor?5iterator?8?$AA@ 10014b98     libvcruntime:undname.obj
 0002:00000bb8       ??_C@_0CH@OOJPLCPH@?$GAeh?5vector?5vbase?5constructor?5ite@ 10014bb8     libvcruntime:undname.obj
 0002:00000be0       ??_C@_0BL@LLKPOHJI@?$GAcopy?5constructor?5closure?8?$AA@ 10014be0     libvcruntime:undname.obj
 0002:00000bfc       ??_C@_0BA@KBCDOMBN@?$GAudt?5returning?8?$AA@ 10014bfc     libvcruntime:undname.obj
 0002:00000c0c       ??_C@_03KLGMFNMG@?$GAEH?$AA@ 10014c0c     libvcruntime:undname.obj
 0002:00000c10       ??_C@_05KHLCHHI@?$GARTTI?$AA@ 10014c10     libvcruntime:undname.obj
 0002:00000c18       ??_C@_0BA@KKLDJDLB@?$GAlocal?5vftable?8?$AA@ 10014c18     libvcruntime:undname.obj
 0002:00000c28       ??_C@_0CE@IIHCMGGL@?$GAlocal?5vftable?5constructor?5closu@ 10014c28     libvcruntime:undname.obj
 0002:00000c4c       ??_C@_06FHBGPFGH@?5new?$FL?$FN?$AA@ 10014c4c     libvcruntime:undname.obj
 0002:00000c54       ??_C@_09LBNFPBCA@?5delete?$FL?$FN?$AA@ 10014c54     libvcruntime:undname.obj
 0002:00000c60       ??_C@_0P@HJKNJFNN@?$GAomni?5callsig?8?$AA@ 10014c60     libvcruntime:undname.obj
 0002:00000c70       ??_C@_0BL@CNOONJFP@?$GAplacement?5delete?5closure?8?$AA@ 10014c70     libvcruntime:undname.obj
 0002:00000c8c       ??_C@_0BN@CKNJLHMB@?$GAplacement?5delete?$FL?$FN?5closure?8?$AA@ 10014c8c     libvcruntime:undname.obj
 0002:00000cac       ??_C@_0CG@CFDHKGGD@?$GAmanaged?5vector?5constructor?5iter@ 10014cac     libvcruntime:undname.obj
 0002:00000cd4       ??_C@_0CF@IMGKMJNO@?$GAmanaged?5vector?5destructor?5itera@ 10014cd4     libvcruntime:undname.obj
 0002:00000cfc       ??_C@_0CG@HLDDJMAG@?$GAeh?5vector?5copy?5constructor?5iter@ 10014cfc     libvcruntime:undname.obj
 0002:00000d24       ??_C@_0CM@FCBBDIGB@?$GAeh?5vector?5vbase?5copy?5constructo@ 10014d24     libvcruntime:undname.obj
 0002:00000d50       ??_C@_0BL@CLIPGLGB@?$GAdynamic?5initializer?5for?5?8?$AA@ 10014d50     libvcruntime:undname.obj
 0002:00000d6c       ??_C@_0CB@PDBIFEP@?$GAdynamic?5atexit?5destructor?5for?5?8@ 10014d6c     libvcruntime:undname.obj
 0002:00000d90       ??_C@_0CD@CGAJBKEJ@?$GAvector?5copy?5constructor?5iterato@ 10014d90     libvcruntime:undname.obj
 0002:00000db4       ??_C@_0CJ@GJELGAMM@?$GAvector?5vbase?5copy?5constructor?5i@ 10014db4     libvcruntime:undname.obj
 0002:00000de0       ??_C@_0CL@FGIJHLCE@?$GAmanaged?5vector?5copy?5constructor@ 10014de0     libvcruntime:undname.obj
 0002:00000e0c       ??_C@_0BM@PMGGMLDN@?$GAlocal?5static?5thread?5guard?8?$AA@ 10014e0c     libvcruntime:undname.obj
 0002:00000e28       ??_C@_0N@BDNMDMOL@operator?5?$CC?$CC?5?$AA@ 10014e28     libvcruntime:undname.obj
 0002:00000e38       ??_C@_0BC@GGEBGALA@operator?5co_await?$AA@ 10014e38     libvcruntime:undname.obj
 0002:00000e4c       ??_C@_0BC@DAFEJGAK@?5Type?5Descriptor?8?$AA@ 10014e4c     libvcruntime:undname.obj
 0002:00000e60       ??_C@_0BM@LDKODKLH@?5Base?5Class?5Descriptor?5at?5?$CI?$AA@ 10014e60     libvcruntime:undname.obj
 0002:00000e7c       ??_C@_0BD@LGICGFMM@?5Base?5Class?5Array?8?$AA@ 10014e7c     libvcruntime:undname.obj
 0002:00000e90       ??_C@_0BN@MECKDCOJ@?5Class?5Hierarchy?5Descriptor?8?$AA@ 10014e90     libvcruntime:undname.obj
 0002:00000eb0       ??_C@_0BK@CFCOFLF@?5Complete?5Object?5Locator?8?$AA@ 10014eb0     libvcruntime:undname.obj
 0002:00000ed8       ??_C@_1DM@KHCHBNEB@?$AAa?$AAp?$AAi?$AA?9?$AAm?$AAs?$AA?9?$AAw?$AAi?$AAn?$AA?9?$AAc?$AAo?$AAr?$AAe?$AA?9?$AAf?$AAi?$AAb?$AAe?$AAr?$AAs?$AA?9?$AAl?$AA1?$AA?9?$AA1?$AA?9?$AA1?$AA?$AA@ 10014ed8     libvcruntime:winapi_downlevel.obj
 0002:00000f14       ??_C@_1DK@LPPGFMPP@?$AAa?$AAp?$AAi?$AA?9?$AAm?$AAs?$AA?9?$AAw?$AAi?$AAn?$AA?9?$AAc?$AAo?$AAr?$AAe?$AA?9?$AAs?$AAy?$AAn?$AAc?$AAh?$AA?9?$AAl?$AA1?$AA?9?$AA2?$AA?9?$AA0?$AA?$AA@ 10014f14     libvcruntime:winapi_downlevel.obj
 0002:00000f50       ??_C@_1BC@GDMECMAK@?$AAk?$AAe?$AAr?$AAn?$AAe?$AAl?$AA3?$AA2?$AA?$AA@ 10014f50     libvcruntime:winapi_downlevel.obj
 0002:00000f64       ??_C@_1BA@PFFKHIOG@?$AAa?$AAp?$AAi?$AA?9?$AAm?$AAs?$AA?9?$AA?$AA@ 10014f64     libvcruntime:winapi_downlevel.obj
 0002:00000f74       ??_C@_1BA@IAIFMGEF@?$AAe?$AAx?$AAt?$AA?9?$AAm?$AAs?$AA?9?$AA?$AA@ 10014f74     libvcruntime:winapi_downlevel.obj
 0002:00000f8c       ??_C@_08KNHFBNJ@FlsAlloc?$AA@ 10014f8c     libvcruntime:winapi_downlevel.obj
 0002:00000fa0       ??_C@_07PEJMOBNF@FlsFree?$AA@ 10014fa0     libvcruntime:winapi_downlevel.obj
 0002:00000fb0       ??_C@_0M@GDNOONDI@FlsGetValue?$AA@ 10014fb0     libvcruntime:winapi_downlevel.obj
 0002:00000fc4       ??_C@_0M@JCPCPOEF@FlsSetValue?$AA@ 10014fc4     libvcruntime:winapi_downlevel.obj
 0002:00000fd8       ??_C@_0BM@HCFOFFN@InitializeCriticalSectionEx?$AA@ 10014fd8     libvcruntime:winapi_downlevel.obj
 0002:00000ff4       __pDestructExceptionObject 10014ff4     libvcruntime:ehhelpers.obj
 0002:00000ff8       _standard_lookup_table     10014ff8     libucrt:output.obj
 0002:00001054       ??_C@_06OJHGLDPL@?$CInull?$CJ?$AA@ 10015054     libucrt:output.obj
 0002:0000105c       ??_C@_1O@CEDCILHN@?$AA?$CI?$AAn?$AAu?$AAl?$AAl?$AA?$CJ?$AA?$AA@ 1001505c     libucrt:output.obj
 0002:00001070       ___acrt_exception_action_table 10015070     libucrt:exception_filter.obj
 0002:00001100       ___acrt_signal_action_table_count 10015100     libucrt:exception_filter.obj
 0002:00001104       ___acrt_signal_action_first_fpe_index 10015104     libucrt:exception_filter.obj
 0002:00001108       ___acrt_signal_action_fpe_count 10015108     libucrt:exception_filter.obj
 0002:0000110c       ??_C@_1BI@BGOHAHKC@?$AAm?$AAs?$AAc?$AAo?$AAr?$AAe?$AAe?$AA?4?$AAd?$AAl?$AAl?$AA?$AA@ 1001510c     libucrt:exit.obj
 0002:00001124       ??_C@_0P@MIGLKIOC@CorExitProcess?$AA@ 10015124     libucrt:exit.obj
 0002:00001318       __wctype                   10015318     libucrt:ctype.obj
 0002:00001520       ___newctype                10015520     libucrt:ctype.obj
 0002:00001820       ___newclmap                10015820     libucrt:ctype.obj
 0002:000019a0       ___newcumap                100159a0     libucrt:ctype.obj
 0002:00001b20       ??_C@_03KOEHGMDN@Sun?$AA@  10015b20     libucrt:nlsdata.obj
 0002:00001b24       ??_C@_03PDAGKDH@Mon?$AA@   10015b24     libucrt:nlsdata.obj
 0002:00001b28       ??_C@_03NAGEINEP@Tue?$AA@  10015b28     libucrt:nlsdata.obj
 0002:00001b2c       ??_C@_03MHOMLAJA@Wed?$AA@  10015b2c     libucrt:nlsdata.obj
 0002:00001b30       ??_C@_03IOFIKPDN@Thu?$AA@  10015b30     libucrt:nlsdata.obj
 0002:00001b34       ??_C@_03IDIOELNC@Fri?$AA@  10015b34     libucrt:nlsdata.obj
 0002:00001b38       ??_C@_03FEFJNEK@Sat?$AA@   10015b38     libucrt:nlsdata.obj
 0002:00001b3c       ??_C@_06OOPIFAJ@Sunday?$AA@ 10015b3c     libucrt:nlsdata.obj
 0002:00001b44       ??_C@_06JLEDEDGH@Monday?$AA@ 10015b44     libucrt:nlsdata.obj
 0002:00001b4c       ??_C@_07BAAGCFCM@Tuesday?$AA@ 10015b4c     libucrt:nlsdata.obj
 0002:00001b54       ??_C@_09DLIGFAKA@Wednesday?$AA@ 10015b54     libucrt:nlsdata.obj
 0002:00001b60       ??_C@_08HACCIKIA@Thursday?$AA@ 10015b60     libucrt:nlsdata.obj
 0002:00001b6c       ??_C@_06JECMNKMI@Friday?$AA@ 10015b6c     libucrt:nlsdata.obj
 0002:00001b74       ??_C@_08INBOOONO@Saturday?$AA@ 10015b74     libucrt:nlsdata.obj
 0002:00001b80       ??_C@_03JIHJHPIE@Jan?$AA@  10015b80     libucrt:nlsdata.obj
 0002:00001b84       ??_C@_03HJBDCHOM@Feb?$AA@  10015b84     libucrt:nlsdata.obj
 0002:00001b88       ??_C@_03ODNJBKGA@Mar?$AA@  10015b88     libucrt:nlsdata.obj
 0002:00001b8c       ??_C@_03LEOLGMJP@Apr?$AA@  10015b8c     libucrt:nlsdata.obj
 0002:00001b90       ??_C@_03CNMDKL@May?$AA@    10015b90     libucrt:nlsdata.obj
 0002:00001b94       ??_C@_03IDFGHECI@Jun?$AA@  10015b94     libucrt:nlsdata.obj
 0002:00001b98       ??_C@_03LBGABGKK@Jul?$AA@  10015b98     libucrt:nlsdata.obj
 0002:00001b9c       ??_C@_03IFJFEIGA@Aug?$AA@  10015b9c     libucrt:nlsdata.obj
 0002:00001ba0       ??_C@_03GGCAPAJC@Sep?$AA@  10015ba0     libucrt:nlsdata.obj
 0002:00001ba4       ??_C@_03BMAOKBAD@Oct?$AA@  10015ba4     libucrt:nlsdata.obj
 0002:00001ba8       ??_C@_03JPJOFNIA@Nov?$AA@  10015ba8     libucrt:nlsdata.obj
 0002:00001bac       ??_C@_03MKABNOCG@Dec?$AA@  10015bac     libucrt:nlsdata.obj
 0002:00001bb0       ??_C@_07CGJPFGJA@January?$AA@ 10015bb0     libucrt:nlsdata.obj
 0002:00001bb8       ??_C@_08GNJGEPFN@February?$AA@ 10015bb8     libucrt:nlsdata.obj
 0002:00001bc4       ??_C@_05HPCKOFNC@March?$AA@ 10015bc4     libucrt:nlsdata.obj
 0002:00001bcc       ??_C@_05DMJDNLEJ@April?$AA@ 10015bcc     libucrt:nlsdata.obj
 0002:00001bd4       ??_C@_04CNLMGBGM@June?$AA@ 10015bd4     libucrt:nlsdata.obj
 0002:00001bdc       ??_C@_04MIEPOIFP@July?$AA@ 10015bdc     libucrt:nlsdata.obj
 0002:00001be4       ??_C@_06LBBHFDDG@August?$AA@ 10015be4     libucrt:nlsdata.obj
 0002:00001bec       ??_C@_09BHHEALKD@September?$AA@ 10015bec     libucrt:nlsdata.obj
 0002:00001bf8       ??_C@_07JJNFCEND@October?$AA@ 10015bf8     libucrt:nlsdata.obj
 0002:00001c00       ??_C@_08HCHEGEOA@November?$AA@ 10015c00     libucrt:nlsdata.obj
 0002:00001c0c       ??_C@_08EDHMEBNP@December?$AA@ 10015c0c     libucrt:nlsdata.obj
 0002:00001c18       ??_C@_02DEDBPAFC@AM?$AA@   10015c18     libucrt:nlsdata.obj
 0002:00001c1c       ??_C@_02CJNFDJBF@PM?$AA@   10015c1c     libucrt:nlsdata.obj
 0002:00001c20       ??_C@_08BPBNCDIB@MM?1dd?1yy?$AA@ 10015c20     libucrt:nlsdata.obj
 0002:00001c2c       ??_C@_0BE@CKGJFCPC@dddd?0?5MMMM?5dd?0?5yyyy?$AA@ 10015c2c     libucrt:nlsdata.obj
 0002:00001c40       ??_C@_08JCCMCCIL@HH?3mm?3ss?$AA@ 10015c40     libucrt:nlsdata.obj
 0002:00001c4c       ??_C@_17MBGCMIPB@?$AAS?$AAu?$AAn?$AA?$AA@ 10015c4c     libucrt:nlsdata.obj
 0002:00001c54       ??_C@_17KBOMKBF@?$AAM?$AAo?$AAn?$AA?$AA@ 10015c54     libucrt:nlsdata.obj
 0002:00001c5c       ??_C@_17BMKGEGOJ@?$AAT?$AAu?$AAe?$AA?$AA@ 10015c5c     libucrt:nlsdata.obj
 0002:00001c64       ??_C@_17CJEDCEPE@?$AAW?$AAe?$AAd?$AA?$AA@ 10015c64     libucrt:nlsdata.obj
 0002:00001c6c       ??_C@_17PDPHAADD@?$AAT?$AAh?$AAu?$AA?$AA@ 10015c6c     libucrt:nlsdata.obj
 0002:00001c74       ??_C@_17HFOLPPLP@?$AAF?$AAr?$AAi?$AA?$AA@ 10015c74     libucrt:nlsdata.obj
 0002:00001c7c       ??_C@_17GGIBDPIH@?$AAS?$AAa?$AAt?$AA?$AA@ 10015c7c     libucrt:nlsdata.obj
 0002:00001c84       ??_C@_1O@IHNHDHPB@?$AAS?$AAu?$AAn?$AAd?$AAa?$AAy?$AA?$AA@ 10015c84     libucrt:nlsdata.obj
 0002:00001c94       ??_C@_1O@MMNBFLIA@?$AAM?$AAo?$AAn?$AAd?$AAa?$AAy?$AA?$AA@ 10015c94     libucrt:nlsdata.obj
 0002:00001ca4       ??_C@_1BA@ENFBFFEK@?$AAT?$AAu?$AAe?$AAs?$AAd?$AAa?$AAy?$AA?$AA@ 10015ca4     libucrt:nlsdata.obj
 0002:00001cb4       ??_C@_1BE@EBOGMDOH@?$AAW?$AAe?$AAd?$AAn?$AAe?$AAs?$AAd?$AAa?$AAy?$AA?$AA@ 10015cb4     libucrt:nlsdata.obj
 0002:00001cc8       ??_C@_1BC@HHMNLIHE@?$AAT?$AAh?$AAu?$AAr?$AAs?$AAd?$AAa?$AAy?$AA?$AA@ 10015cc8     libucrt:nlsdata.obj
 0002:00001cdc       ??_C@_1O@PDICJHAG@?$AAF?$AAr?$AAi?$AAd?$AAa?$AAy?$AA?$AA@ 10015cdc     libucrt:nlsdata.obj
 0002:00001cec       ??_C@_1BC@ENMNNPAJ@?$AAS?$AAa?$AAt?$AAu?$AAr?$AAd?$AAa?$AAy?$AA?$AA@ 10015cec     libucrt:nlsdata.obj
 0002:00001d00       ??_C@_17DKNBKCHM@?$AAJ?$AAa?$AAn?$AA?$AA@ 10015d00     libucrt:nlsdata.obj
 0002:00001d08       ??_C@_17LMDJEKJN@?$AAF?$AAe?$AAb?$AA?$AA@ 10015d08     libucrt:nlsdata.obj
 0002:00001d10       ??_C@_17CKNLEDEC@?$AAM?$AAa?$AAr?$AA?$AA@ 10015d10     libucrt:nlsdata.obj
 0002:00001d18       ??_C@_17LFPOIHDD@?$AAA?$AAp?$AAr?$AA?$AA@ 10015d18     libucrt:nlsdata.obj
 0002:00001d20       ??_C@_17PNNKMEED@?$AAM?$AAa?$AAy?$AA?$AA@ 10015d20     libucrt:nlsdata.obj
 0002:00001d28       ??_C@_17KCJGOCPB@?$AAJ?$AAu?$AAn?$AA?$AA@ 10015d28     libucrt:nlsdata.obj
 0002:00001d30       ??_C@_17IJPCKHK@?$AAJ?$AAu?$AAl?$AA?$AA@ 10015d30     libucrt:nlsdata.obj
 0002:00001d38       ??_C@_17ICPELBCN@?$AAA?$AAu?$AAg?$AA?$AA@ 10015d38     libucrt:nlsdata.obj
 0002:00001d40       ??_C@_17HCHCOKMG@?$AAS?$AAe?$AAp?$AA?$AA@ 10015d40     libucrt:nlsdata.obj
 0002:00001d48       ??_C@_17FNLKOI@?$AAO?$AAc?$AAt?$AA?$AA@ 10015d48     libucrt:nlsdata.obj
 0002:00001d50       ??_C@_17BBDMLCIG@?$AAN?$AAo?$AAv?$AA?$AA@ 10015d50     libucrt:nlsdata.obj
 0002:00001d58       ??_C@_17EGKACKIF@?$AAD?$AAe?$AAc?$AA?$AA@ 10015d58     libucrt:nlsdata.obj
 0002:00001d60       ??_C@_1BA@EFMEIEBA@?$AAJ?$AAa?$AAn?$AAu?$AAa?$AAr?$AAy?$AA?$AA@ 10015d60     libucrt:nlsdata.obj
 0002:00001d70       ??_C@_1BC@JGDDFFAM@?$AAF?$AAe?$AAb?$AAr?$AAu?$AAa?$AAr?$AAy?$AA?$AA@ 10015d70     libucrt:nlsdata.obj
 0002:00001d84       ??_C@_1M@IKEENEDF@?$AAM?$AAa?$AAr?$AAc?$AAh?$AA?$AA@ 10015d84     libucrt:nlsdata.obj
 0002:00001d90       ??_C@_1M@GJNLMHFD@?$AAA?$AAp?$AAr?$AAi?$AAl?$AA?$AA@ 10015d90     libucrt:nlsdata.obj
 0002:00001d9c       ??_C@_19EPFLPGAP@?$AAJ?$AAu?$AAn?$AAe?$AA?$AA@ 10015d9c     libucrt:nlsdata.obj
 0002:00001da8       ??_C@_19BIFMLPCD@?$AAJ?$AAu?$AAl?$AAy?$AA?$AA@ 10015da8     libucrt:nlsdata.obj
 0002:00001db4       ??_C@_1O@PAHLKOAC@?$AAA?$AAu?$AAg?$AAu?$AAs?$AAt?$AA?$AA@ 10015db4     libucrt:nlsdata.obj
 0002:00001dc4       ??_C@_1BE@DKAAMBJL@?$AAS?$AAe?$AAp?$AAt?$AAe?$AAm?$AAb?$AAe?$AAr?$AA?$AA@ 10015dc4     libucrt:nlsdata.obj
 0002:00001dd8       ??_C@_1BA@EPANDLNG@?$AAO?$AAc?$AAt?$AAo?$AAb?$AAe?$AAr?$AA?$AA@ 10015dd8     libucrt:nlsdata.obj
 0002:00001de8       ??_C@_1BC@BGLIFPF@?$AAN?$AAo?$AAv?$AAe?$AAm?$AAb?$AAe?$AAr?$AA?$AA@ 10015de8     libucrt:nlsdata.obj
 0002:00001dfc       ??_C@_1BC@FEMKIFH@?$AAD?$AAe?$AAc?$AAe?$AAm?$AAb?$AAe?$AAr?$AA?$AA@ 10015dfc     libucrt:nlsdata.obj
 0002:00001e10       ??_C@_15ODEHAHHF@?$AAA?$AAM?$AA?$AA@ 10015e10     libucrt:nlsdata.obj
 0002:00001e18       ??_C@_15CLMNNGEL@?$AAP?$AAM?$AA?$AA@ 10015e18     libucrt:nlsdata.obj
 0002:00001e20       ??_C@_1BC@IEBCMHCM@?$AAM?$AAM?$AA?1?$AAd?$AAd?$AA?1?$AAy?$AAy?$AA?$AA@ 10015e20     libucrt:nlsdata.obj
 0002:00001e34       ??_C@_1CI@KNAKOEBC@?$AAd?$AAd?$AAd?$AAd?$AA?0?$AA?5?$AAM?$AAM?$AAM?$AAM?$AA?5?$AAd?$AAd?$AA?0?$AA?5?$AAy?$AAy?$AAy?$AAy?$AA?$AA@ 10015e34     libucrt:nlsdata.obj
 0002:00001e5c       ??_C@_1BC@GDGBMEMK@?$AAH?$AAH?$AA?3?$AAm?$AAm?$AA?3?$AAs?$AAs?$AA?$AA@ 10015e5c     libucrt:nlsdata.obj
 0002:00001e70       ??_C@_1M@BMHNFIME@?$AAe?$AAn?$AA?9?$AAU?$AAS?$AA?$AA@ 10015e70     libucrt:nlsdata.obj
 0002:00001e80       ___lc_time_c               10015e80     libucrt:nlsdata.obj
 0002:00001fe4       ??_C@_03OEIAHPBN@INF?$AA@  10015fe4     libucrt:cvt.obj
 0002:00001fe8       ??_C@_03OJHLLCGB@inf?$AA@  10015fe8     libucrt:cvt.obj
 0002:00001fec       ??_C@_03LKNCIKJB@NAN?$AA@  10015fec     libucrt:cvt.obj
 0002:00001ff0       ??_C@_03LHCJEHON@nan?$AA@  10015ff0     libucrt:cvt.obj
 0002:00001ff4       ??_C@_09OFJJIMPC@NAN?$CISNAN?$CJ?$AA@ 10015ff4     libucrt:cvt.obj
 0002:00002000       ??_C@_09IPFBKMDL@nan?$CIsnan?$CJ?$AA@ 10016000     libucrt:cvt.obj
 0002:0000200c       ??_C@_08IKHNHAJ@NAN?$CIIND?$CJ?$AA@ 1001600c     libucrt:cvt.obj
 0002:00002018       ??_C@_08OFCDMILK@nan?$CIind?$CJ?$AA@ 10016018     libucrt:cvt.obj
 0002:00002024       ??_C@_05KLBDPFGC@e?$CL000?$AA@ 10016024     libucrt:cvt.obj
 0002:00002080       ??_C@_1EG@CNNIPFIM@?$AAa?$AAp?$AAi?$AA?9?$AAm?$AAs?$AA?9?$AAw?$AAi?$AAn?$AA?9?$AAa?$AAp?$AAp?$AAm?$AAo?$AAd?$AAe?$AAl?$AA?9?$AAr?$AAu?$AAn?$AAt?$AAi?$AAm?$AAe?$AA?9?$AAl?$AA1?$AA?9?$AA1@ 10016080     libucrt:winapi_thunks.obj
 0002:000020c8       ??_C@_1EA@JGEFHKEI@?$AAa?$AAp?$AAi?$AA?9?$AAm?$AAs?$AA?9?$AAw?$AAi?$AAn?$AA?9?$AAc?$AAo?$AAr?$AAe?$AA?9?$AAd?$AAa?$AAt?$AAe?$AAt?$AAi?$AAm?$AAe?$AA?9?$AAl?$AA1?$AA?9?$AA1?$AA?9?$AA1?$AA?$AA@ 100160c8     libucrt:winapi_thunks.obj
 0002:00002108       ??_C@_1DI@GCIAAENM@?$AAa?$AAp?$AAi?$AA?9?$AAm?$AAs?$AA?9?$AAw?$AAi?$AAn?$AA?9?$AAc?$AAo?$AAr?$AAe?$AA?9?$AAf?$AAi?$AAl?$AAe?$AA?9?$AAl?$AA2?$AA?9?$AA1?$AA?9?$AA1?$AA?$AA@ 10016108     libucrt:winapi_thunks.obj
 0002:00002140       ??_C@_1EI@MPIAOHOC@?$AAa?$AAp?$AAi?$AA?9?$AAm?$AAs?$AA?9?$AAw?$AAi?$AAn?$AA?9?$AAc?$AAo?$AAr?$AAe?$AA?9?$AAl?$AAo?$AAc?$AAa?$AAl?$AAi?$AAz?$AAa?$AAt?$AAi?$AAo?$AAn?$AA?9?$AAl?$AA1?$AA?9@ 10016140     libucrt:winapi_thunks.obj
 0002:00002188       ??_C@_1FK@FPHCKFIE@?$AAa?$AAp?$AAi?$AA?9?$AAm?$AAs?$AA?9?$AAw?$AAi?$AAn?$AA?9?$AAc?$AAo?$AAr?$AAe?$AA?9?$AAl?$AAo?$AAc?$AAa?$AAl?$AAi?$AAz?$AAa?$AAt?$AAi?$AAo?$AAn?$AA?9?$AAo?$AAb?$AAs@ 10016188     libucrt:winapi_thunks.obj
 0002:000021e8       ??_C@_1EM@DILCGIIO@?$AAa?$AAp?$AAi?$AA?9?$AAm?$AAs?$AA?9?$AAw?$AAi?$AAn?$AA?9?$AAc?$AAo?$AAr?$AAe?$AA?9?$AAp?$AAr?$AAo?$AAc?$AAe?$AAs?$AAs?$AAt?$AAh?$AAr?$AAe?$AAa?$AAd?$AAs?$AA?9?$AAl@ 100161e8     libucrt:winapi_thunks.obj
 0002:00002234       ??_C@_1DM@LNCGDDPN@?$AAa?$AAp?$AAi?$AA?9?$AAm?$AAs?$AA?9?$AAw?$AAi?$AAn?$AA?9?$AAc?$AAo?$AAr?$AAe?$AA?9?$AAs?$AAt?$AAr?$AAi?$AAn?$AAg?$AA?9?$AAl?$AA1?$AA?9?$AA1?$AA?9?$AA0?$AA?$AA@ 10016234     libucrt:winapi_thunks.obj
 0002:00002270       ??_C@_1DO@FPAPJEMD@?$AAa?$AAp?$AAi?$AA?9?$AAm?$AAs?$AA?9?$AAw?$AAi?$AAn?$AA?9?$AAc?$AAo?$AAr?$AAe?$AA?9?$AAs?$AAy?$AAs?$AAi?$AAn?$AAf?$AAo?$AA?9?$AAl?$AA1?$AA?9?$AA2?$AA?9?$AA1?$AA?$AA@ 10016270     libucrt:winapi_thunks.obj
 0002:000022b0       ??_C@_1DK@NDHNAHIO@?$AAa?$AAp?$AAi?$AA?9?$AAm?$AAs?$AA?9?$AAw?$AAi?$AAn?$AA?9?$AAc?$AAo?$AAr?$AAe?$AA?9?$AAw?$AAi?$AAn?$AAr?$AAt?$AA?9?$AAl?$AA1?$AA?9?$AA1?$AA?9?$AA0?$AA?$AA@ 100162b0     libucrt:winapi_thunks.obj
 0002:000022ec       ??_C@_1DM@KGHDGBCM@?$AAa?$AAp?$AAi?$AA?9?$AAm?$AAs?$AA?9?$AAw?$AAi?$AAn?$AA?9?$AAc?$AAo?$AAr?$AAe?$AA?9?$AAx?$AAs?$AAt?$AAa?$AAt?$AAe?$AA?9?$AAl?$AA2?$AA?9?$AA1?$AA?9?$AA0?$AA?$AA@ 100162ec     libucrt:winapi_thunks.obj
 0002:00002328       ??_C@_1EO@IJIOEFOH@?$AAa?$AAp?$AAi?$AA?9?$AAm?$AAs?$AA?9?$AAw?$AAi?$AAn?$AA?9?$AAr?$AAt?$AAc?$AAo?$AAr?$AAe?$AA?9?$AAn?$AAt?$AAu?$AAs?$AAe?$AAr?$AA?9?$AAw?$AAi?$AAn?$AAd?$AAo?$AAw?$AA?9@ 10016328     libucrt:winapi_thunks.obj
 0002:00002378       ??_C@_1FG@HHGEKANL@?$AAa?$AAp?$AAi?$AA?9?$AAm?$AAs?$AA?9?$AAw?$AAi?$AAn?$AA?9?$AAs?$AAe?$AAc?$AAu?$AAr?$AAi?$AAt?$AAy?$AA?9?$AAs?$AAy?$AAs?$AAt?$AAe?$AAm?$AAf?$AAu?$AAn?$AAc?$AAt?$AAi@ 10016378     libucrt:winapi_thunks.obj
 0002:000023d0       ??_C@_1FG@NCKKOLKO@?$AAe?$AAx?$AAt?$AA?9?$AAm?$AAs?$AA?9?$AAw?$AAi?$AAn?$AA?9?$AAk?$AAe?$AAr?$AAn?$AAe?$AAl?$AA3?$AA2?$AA?9?$AAp?$AAa?$AAc?$AAk?$AAa?$AAg?$AAe?$AA?9?$AAc?$AAu?$AAr?$AAr@ 100163d0     libucrt:winapi_thunks.obj
 0002:00002428       ??_C@_1EG@DBIOJECG@?$AAe?$AAx?$AAt?$AA?9?$AAm?$AAs?$AA?9?$AAw?$AAi?$AAn?$AA?9?$AAn?$AAt?$AAu?$AAs?$AAe?$AAr?$AA?9?$AAd?$AAi?$AAa?$AAl?$AAo?$AAg?$AAb?$AAo?$AAx?$AA?9?$AAl?$AA1?$AA?9?$AA1@ 10016428     libucrt:winapi_thunks.obj
 0002:00002470       ??_C@_1EO@FIHMJCLF@?$AAe?$AAx?$AAt?$AA?9?$AAm?$AAs?$AA?9?$AAw?$AAi?$AAn?$AA?9?$AAn?$AAt?$AAu?$AAs?$AAe?$AAr?$AA?9?$AAw?$AAi?$AAn?$AAd?$AAo?$AAw?$AAs?$AAt?$AAa?$AAt?$AAi?$AAo?$AAn?$AA?9@ 10016470     libucrt:winapi_thunks.obj
 0002:000024c0       ??_C@_1BC@DNHGCMLG@?$AAa?$AAd?$AAv?$AAa?$AAp?$AAi?$AA3?$AA2?$AA?$AA@ 100164c0     libucrt:winapi_thunks.obj
 0002:000024d4       ??_C@_1O@BCCLBEOE@?$AAu?$AAs?$AAe?$AAr?$AA3?$AA2?$AA?$AA@ 100164d4     libucrt:winapi_thunks.obj
 0002:0000250c       ??_C@_0BE@JOGNEJCI@GetCurrentPackageId?$AA@ 1001650c     libucrt:winapi_thunks.obj
 0002:00002530       ??_C@_0O@KKBNKAPF@LCMapStringEx?$AA@ 10016530     libucrt:winapi_thunks.obj
 0002:00002548       ??_C@_0BB@HBDEELFH@LocaleNameToLCID?$AA@ 10016548     libucrt:winapi_thunks.obj
 0002:0000256c       ??_C@_1M@HPNHIDJI@?$AAj?$AAa?$AA?9?$AAJ?$AAP?$AA?$AA@ 1001656c     libucrt:mbctype.obj
 0002:00002578       ??_C@_1M@BIBDDEMK@?$AAz?$AAh?$AA?9?$AAC?$AAN?$AA?$AA@ 10016578     libucrt:mbctype.obj
 0002:00002584       ??_C@_1M@JLOOOEGK@?$AAk?$AAo?$AA?9?$AAK?$AAR?$AA?$AA@ 10016584     libucrt:mbctype.obj
 0002:00002590       ??_C@_1M@CLNBBOPM@?$AAz?$AAh?$AA?9?$AAT?$AAW?$AA?$AA@ 10016590     libucrt:mbctype.obj
 0002:0000259c       ??_C@_15PJPFLCCM@?$AAu?$AAk?$AA?$AA@ 1001659c     libucrt:get_qualified_locale.obj
 0002:000025a8       ?large_power_data@?1??multiply_by_power_of_ten@__crt_strtox@@YA_NAAUbig_integer@2@I@Z@4QBIB 100165a8     libucrt:cfout.obj
 0002:00002eb0       ?large_power_indices@?1??multiply_by_power_of_ten@__crt_strtox@@YA_NAAUbig_integer@2@I@Z@4QBUunpack_index@?1??12@YA_N0I@Z@B 10016eb0     libucrt:cfout.obj
 0002:00002f48       ?small_powers_of_ten@?6??multiply_by_power_of_ten@__crt_strtox@@YA_NAAUbig_integer@2@I@Z@4QBIB 10016f48     libucrt:cfout.obj
 0002:00002f6c       ??_C@_01GBGANLPD@0?$AA@    10016f6c     libucrt:cfout.obj
 0002:00002f70       ??_C@_05DNEBIAHO@1?$CDINF?$AA@ 10016f70     libucrt:cfout.obj
 0002:00002f78       ??_C@_06IMKFLFPG@1?$CDQNAN?$AA@ 10016f78     libucrt:cfout.obj
 0002:00002f80       ??_C@_06PGGFOGJG@1?$CDSNAN?$AA@ 10016f80     libucrt:cfout.obj
 0002:00002f88       ??_C@_05PHHOCPM@1?$CDIND?$AA@ 10016f88     libucrt:cfout.obj
 0002:000036b0       ??_C@_15EMKDOKLE@?$AAa?$AAr?$AA?$AA@ 100176b0     libucrt:lcidtoname_downlevel.obj
 0002:000036b8       ??_C@_15KNPADPLH@?$AAb?$AAg?$AA?$AA@ 100176b8     libucrt:lcidtoname_downlevel.obj
 0002:000036c0       ??_C@_15EDMHLDMO@?$AAc?$AAa?$AA?$AA@ 100176c0     libucrt:lcidtoname_downlevel.obj
 0002:000036c8       ??_C@_1O@BPEAJADD@?$AAz?$AAh?$AA?9?$AAC?$AAH?$AAS?$AA?$AA@ 100176c8     libucrt:lcidtoname_downlevel.obj
 0002:000036d8       ??_C@_15LJNHCMNK@?$AAc?$AAs?$AA?$AA@ 100176d8     libucrt:lcidtoname_downlevel.obj
 0002:000036e0       ??_C@_15FOMCIDHG@?$AAd?$AAa?$AA?$AA@ 100176e0     libucrt:lcidtoname_downlevel.obj
 0002:000036e8       ??_C@_15NBKABECB@?$AAd?$AAe?$AA?$AA@ 100176e8     libucrt:lcidtoname_downlevel.obj
 0002:000036f0       ??_C@_15GHPEIIAO@?$AAe?$AAl?$AA?$AA@ 100176f0     libucrt:lcidtoname_downlevel.obj
 0002:000036f8       ??_C@_15MNPNEAIF@?$AAe?$AAn?$AA?$AA@ 100176f8     libucrt:lcidtoname_downlevel.obj
 0002:00003700       ??_C@_15GPIOMPMH@?$AAe?$AAs?$AA?$AA@ 10017700     libucrt:lcidtoname_downlevel.obj
 0002:00003708       ??_C@_15NGLOAKJC@?$AAf?$AAi?$AA?$AA@ 10017708     libucrt:lcidtoname_downlevel.obj
 0002:00003710       ??_C@_15FBKGNKAM@?$AAf?$AAr?$AA?$AA@ 10017710     libucrt:lcidtoname_downlevel.obj
 0002:00003718       ??_C@_15KGGCNEFK@?$AAh?$AAe?$AA?$AA@ 10017718     libucrt:lcidtoname_downlevel.obj
 0002:00003720       ??_C@_15PGHLIDMF@?$AAh?$AAu?$AA?$AA@ 10017720     libucrt:lcidtoname_downlevel.obj
 0002:00003728       ??_C@_15BIEMAPLM@?$AAi?$AAs?$AA?$AA@ 10017728     libucrt:lcidtoname_downlevel.obj
 0002:00003730       ??_C@_15IFJLDHAF@?$AAi?$AAt?$AA?$AA@ 10017730     libucrt:lcidtoname_downlevel.obj
 0002:00003738       ??_C@_15GEMIOCAG@?$AAj?$AAa?$AA?$AA@ 10017738     libucrt:lcidtoname_downlevel.obj
 0002:00003740       ??_C@_15EPELEGJA@?$AAk?$AAo?$AA?$AA@ 10017740     libucrt:lcidtoname_downlevel.obj
 0002:00003748       ??_C@_15NDDHIMN@?$AAn?$AAl?$AA?$AA@ 10017748     libucrt:lcidtoname_downlevel.obj
 0002:00003750       ??_C@_15BPIGNHCD@?$AAn?$AAo?$AA?$AA@ 10017750     libucrt:lcidtoname_downlevel.obj
 0002:00003758       ??_C@_15DEOPBLCG@?$AAp?$AAl?$AA?$AA@ 10017758     libucrt:lcidtoname_downlevel.obj
 0002:00003760       ??_C@_15KBECGEFG@?$AAp?$AAt?$AA?$AA@ 10017760     libucrt:lcidtoname_downlevel.obj
 0002:00003768       ??_C@_15GLJCBFMD@?$AAr?$AAo?$AA?$AA@ 10017768     libucrt:lcidtoname_downlevel.obj
 0002:00003770       ??_C@_15FEDGKCDI@?$AAr?$AAu?$AA?$AA@ 10017770     libucrt:lcidtoname_downlevel.obj
 0002:00003778       ??_C@_15GLKMLLHM@?$AAh?$AAr?$AA?$AA@ 10017778     libucrt:lcidtoname_downlevel.obj
 0002:00003780       ??_C@_15CPKMFBDB@?$AAs?$AAk?$AA?$AA@ 10017780     libucrt:lcidtoname_downlevel.obj
 0002:00003788       ??_C@_15BAAIOGMK@?$AAs?$AAq?$AA?$AA@ 10017788     libucrt:lcidtoname_downlevel.obj
 0002:00003790       ??_C@_15INNPNOHD@?$AAs?$AAv?$AA?$AA@ 10017790     libucrt:lcidtoname_downlevel.obj
 0002:00003798       ??_C@_15CABMMOGH@?$AAt?$AAh?$AA?$AA@ 10017798     libucrt:lcidtoname_downlevel.obj
 0002:000037a0       ??_C@_15BPLIHJJM@?$AAt?$AAr?$AA?$AA@ 100177a0     libucrt:lcidtoname_downlevel.obj
 0002:000037a8       ??_C@_15NEOEKKDJ@?$AAu?$AAr?$AA?$AA@ 100177a8     libucrt:lcidtoname_downlevel.obj
 0002:000037b0       ??_C@_15NFICGAJK@?$AAi?$AAd?$AA?$AA@ 100177b0     libucrt:lcidtoname_downlevel.obj
 0002:000037b8       ??_C@_15HPJPHDM@?$AAb?$AAe?$AA?$AA@ 100177b8     libucrt:lcidtoname_downlevel.obj
 0002:000037c0       ??_C@_15LCHLGJII@?$AAs?$AAl?$AA?$AA@ 100177c0     libucrt:lcidtoname_downlevel.obj
 0002:000037c8       ??_C@_15PCFJPHHO@?$AAe?$AAt?$AA?$AA@ 100177c8     libucrt:lcidtoname_downlevel.obj
 0002:000037d0       ??_C@_15HPFPGODN@?$AAl?$AAv?$AA?$AA@ 100177d0     libucrt:lcidtoname_downlevel.obj
 0002:000037d8       ??_C@_15NFFGKGLG@?$AAl?$AAt?$AA?$AA@ 100177d8     libucrt:lcidtoname_downlevel.obj
 0002:000037e0       ??_C@_15BDAKCCHN@?$AAf?$AAa?$AA?$AA@ 100177e0     libucrt:lcidtoname_downlevel.obj
 0002:000037e8       ??_C@_15NFGIAIAJ@?$AAv?$AAi?$AA?$AA@ 100177e8     libucrt:lcidtoname_downlevel.obj
 0002:000037f0       ??_C@_15LMKNDMHN@?$AAh?$AAy?$AA?$AA@ 100177f0     libucrt:lcidtoname_downlevel.obj
 0002:000037f8       ??_C@_15IJBHMCFL@?$AAa?$AAz?$AA?$AA@ 100177f8     libucrt:lcidtoname_downlevel.obj
 0002:00003800       ??_C@_15EKOFJABL@?$AAe?$AAu?$AA?$AA@ 10017800     libucrt:lcidtoname_downlevel.obj
 0002:00003808       ??_C@_15BGHADCNK@?$AAm?$AAk?$AA?$AA@ 10017808     libucrt:lcidtoname_downlevel.obj
 0002:00003810       ??_C@_15JDNICKHM@?$AAa?$AAf?$AA?$AA@ 10017810     libucrt:lcidtoname_downlevel.obj
 0002:00003818       ??_C@_15KPJEDBKD@?$AAk?$AAa?$AA?$AA@ 10017818     libucrt:lcidtoname_downlevel.obj
 0002:00003820       ??_C@_15PDNFFFEO@?$AAf?$AAo?$AA?$AA@ 10017820     libucrt:lcidtoname_downlevel.obj
 0002:00003828       ??_C@_15OMLEGLOC@?$AAh?$AAi?$AA?$AA@ 10017828     libucrt:lcidtoname_downlevel.obj
 0002:00003830       ??_C@_15IDNNENKK@?$AAm?$AAs?$AA?$AA@ 10017830     libucrt:lcidtoname_downlevel.obj
 0002:00003838       ??_C@_15MACJNBMH@?$AAk?$AAk?$AA?$AA@ 10017838     libucrt:lcidtoname_downlevel.obj
 0002:00003840       ??_C@_15DKDJEOND@?$AAk?$AAy?$AA?$AA@ 10017840     libucrt:lcidtoname_downlevel.obj
 0002:00003848       ??_C@_15DFGDLJBG@?$AAs?$AAw?$AA?$AA@ 10017848     libucrt:lcidtoname_downlevel.obj
 0002:00003850       ??_C@_15BBFAICNG@?$AAu?$AAz?$AA?$AA@ 10017850     libucrt:lcidtoname_downlevel.obj
 0002:00003858       ??_C@_15DKNDCGEA@?$AAt?$AAt?$AA?$AA@ 10017858     libucrt:lcidtoname_downlevel.obj
 0002:00003860       ??_C@_15MGIFMDPL@?$AAp?$AAa?$AA?$AA@ 10017860     libucrt:lcidtoname_downlevel.obj
 0002:00003868       ??_C@_15HCNDBBA@?$AAg?$AAu?$AA?$AA@ 10017868     libucrt:lcidtoname_downlevel.obj
 0002:00003870       ??_C@_15FNBEIBON@?$AAt?$AAa?$AA?$AA@ 10017870     libucrt:lcidtoname_downlevel.obj
 0002:00003878       ??_C@_15NCHGBGLK@?$AAt?$AAe?$AA?$AA@ 10017878     libucrt:lcidtoname_downlevel.obj
 0002:00003880       ??_C@_15PHPHCBPF@?$AAk?$AAn?$AA?$AA@ 10017880     libucrt:lcidtoname_downlevel.obj
 0002:00003888       ??_C@_15DLGBCKMP@?$AAm?$AAr?$AA?$AA@ 10017888     libucrt:lcidtoname_downlevel.obj
 0002:00003890       ??_C@_15EABBLBFF@?$AAs?$AAa?$AA?$AA@ 10017890     libucrt:lcidtoname_downlevel.obj
 0002:00003898       ??_C@_15CBKOMCOI@?$AAm?$AAn?$AA?$AA@ 10017898     libucrt:lcidtoname_downlevel.obj
 0002:000038a0       ??_C@_15CKDMCJAF@?$AAg?$AAl?$AA?$AA@ 100178a0     libucrt:lcidtoname_downlevel.obj
 0002:000038a8       ??_C@_17CNJFBPG@?$AAk?$AAo?$AAk?$AA?$AA@ 100178a8     libucrt:lcidtoname_downlevel.obj
 0002:000038b0       ??_C@_17FFBJICPL@?$AAs?$AAy?$AAr?$AA?$AA@ 100178b0     libucrt:lcidtoname_downlevel.obj
 0002:000038b8       ??_C@_17KPNDCPAF@?$AAd?$AAi?$AAv?$AA?$AA@ 100178b8     libucrt:lcidtoname_downlevel.obj
 0002:000038c0       ??_C@_1M@OKAHONE@?$AAa?$AAr?$AA?9?$AAS?$AAA?$AA?$AA@ 100178c0     libucrt:lcidtoname_downlevel.obj
 0002:000038cc       ??_C@_1M@FFFIGIGK@?$AAb?$AAg?$AA?9?$AAB?$AAG?$AA?$AA@ 100178cc     libucrt:lcidtoname_downlevel.obj
 0002:000038d8       ??_C@_1M@BJNKEDC@?$AAc?$AAa?$AA?9?$AAE?$AAS?$AA?$AA@ 100178d8     libucrt:lcidtoname_downlevel.obj
 0002:000038e4       ??_C@_1M@IJJHFJHA@?$AAc?$AAs?$AA?9?$AAC?$AAZ?$AA?$AA@ 100178e4     libucrt:lcidtoname_downlevel.obj
 0002:000038f0       ??_C@_1M@CLPEOBGI@?$AAd?$AAa?$AA?9?$AAD?$AAK?$AA?$AA@ 100178f0     libucrt:lcidtoname_downlevel.obj
 0002:000038fc       ??_C@_1M@MCMADGCB@?$AAd?$AAe?$AA?9?$AAD?$AAE?$AA?$AA@ 100178fc     libucrt:lcidtoname_downlevel.obj
 0002:00003908       ??_C@_1M@OOCKEMAM@?$AAe?$AAl?$AA?9?$AAG?$AAR?$AA?$AA@ 10017908     libucrt:lcidtoname_downlevel.obj
 0002:00003914       ??_C@_1M@DDNJFGID@?$AAf?$AAi?$AA?9?$AAF?$AAI?$AA?$AA@ 10017914     libucrt:lcidtoname_downlevel.obj
 0002:00003920       ??_C@_1M@GLIPPMAC@?$AAf?$AAr?$AA?9?$AAF?$AAR?$AA?$AA@ 10017920     libucrt:lcidtoname_downlevel.obj
 0002:0000392c       ??_C@_1M@GFMCHPE@?$AAh?$AAe?$AA?9?$AAI?$AAL?$AA?$AA@ 1001792c     libucrt:lcidtoname_downlevel.obj
 0002:00003938       ??_C@_1M@MHLPGNKM@?$AAh?$AAu?$AA?9?$AAH?$AAU?$AA?$AA@ 10017938     libucrt:lcidtoname_downlevel.obj
 0002:00003944       ??_C@_1M@LPDDNNPN@?$AAi?$AAs?$AA?9?$AAI?$AAS?$AA?$AA@ 10017944     libucrt:lcidtoname_downlevel.obj
 0002:00003950       ??_C@_1M@MADIPODN@?$AAi?$AAt?$AA?9?$AAI?$AAT?$AA?$AA@ 10017950     libucrt:lcidtoname_downlevel.obj
 0002:0000395c       ??_C@_1M@IHBJJGG@?$AAn?$AAl?$AA?9?$AAN?$AAL?$AA?$AA@ 1001795c     libucrt:lcidtoname_downlevel.obj
 0002:00003968       ??_C@_1M@EANAGDL@?$AAn?$AAb?$AA?9?$AAN?$AAO?$AA?$AA@ 10017968     libucrt:lcidtoname_downlevel.obj
 0002:00003974       ??_C@_1M@NEIEMEGP@?$AAp?$AAl?$AA?9?$AAP?$AAL?$AA?$AA@ 10017974     libucrt:lcidtoname_downlevel.obj
 0002:00003980       ??_C@_1M@BOCFIGEP@?$AAp?$AAt?$AA?9?$AAB?$AAR?$AA?$AA@ 10017980     libucrt:lcidtoname_downlevel.obj
 0002:0000398c       ??_C@_1M@IMPFOPBG@?$AAr?$AAo?$AA?9?$AAR?$AAO?$AA?$AA@ 1001798c     libucrt:lcidtoname_downlevel.obj
 0002:00003998       ??_C@_1M@IDNNEJMM@?$AAr?$AAu?$AA?9?$AAR?$AAU?$AA?$AA@ 10017998     libucrt:lcidtoname_downlevel.obj
 0002:000039a4       ??_C@_1M@LILEEOGM@?$AAh?$AAr?$AA?9?$AAH?$AAR?$AA?$AA@ 100179a4     libucrt:lcidtoname_downlevel.obj
 0002:000039b0       ??_C@_1M@FKIFEHPB@?$AAs?$AAk?$AA?9?$AAS?$AAK?$AA?$AA@ 100179b0     libucrt:lcidtoname_downlevel.obj
 0002:000039bc       ??_C@_1M@LJMAMNPJ@?$AAs?$AAq?$AA?9?$AAA?$AAL?$AA?$AA@ 100179bc     libucrt:lcidtoname_downlevel.obj
 0002:000039c8       ??_C@_1M@GIAKDKJK@?$AAs?$AAv?$AA?9?$AAS?$AAE?$AA?$AA@ 100179c8     libucrt:lcidtoname_downlevel.obj
 0002:000039d4       ??_C@_1M@MKJKIKCL@?$AAt?$AAh?$AA?9?$AAT?$AAH?$AA?$AA@ 100179d4     libucrt:lcidtoname_downlevel.obj
 0002:000039e0       ??_C@_1M@MFLCCMPB@?$AAt?$AAr?$AA?9?$AAT?$AAR?$AA?$AA@ 100179e0     libucrt:lcidtoname_downlevel.obj
 0002:000039ec       ??_C@_1M@OIJHDKJN@?$AAu?$AAr?$AA?9?$AAP?$AAK?$AA?$AA@ 100179ec     libucrt:lcidtoname_downlevel.obj
 0002:000039f8       ??_C@_1M@LHIPCIEK@?$AAi?$AAd?$AA?9?$AAI?$AAD?$AA?$AA@ 100179f8     libucrt:lcidtoname_downlevel.obj
 0002:00003a04       ??_C@_1M@MFMOBGI@?$AAu?$AAk?$AA?9?$AAU?$AAA?$AA?$AA@ 10017a04     libucrt:lcidtoname_downlevel.obj
 0002:00003a10       ??_C@_1M@OBGLJIPL@?$AAb?$AAe?$AA?9?$AAB?$AAY?$AA?$AA@ 10017a10     libucrt:lcidtoname_downlevel.obj
 0002:00003a1c       ??_C@_1M@BCFAJEAD@?$AAs?$AAl?$AA?9?$AAS?$AAI?$AA?$AA@ 10017a1c     libucrt:lcidtoname_downlevel.obj
 0002:00003a28       ??_C@_1M@FKFFEDDN@?$AAe?$AAt?$AA?9?$AAE?$AAE?$AA?$AA@ 10017a28     libucrt:lcidtoname_downlevel.obj
 0002:00003a34       ??_C@_1M@KGKKAACI@?$AAl?$AAv?$AA?9?$AAL?$AAV?$AA?$AA@ 10017a34     libucrt:lcidtoname_downlevel.obj
 0002:00003a40       ??_C@_1M@IFGBIJO@?$AAl?$AAt?$AA?9?$AAL?$AAT?$AA?$AA@ 10017a40     libucrt:lcidtoname_downlevel.obj
 0002:00003a4c       ??_C@_1M@FGEAHEDM@?$AAf?$AAa?$AA?9?$AAI?$AAR?$AA?$AA@ 10017a4c     libucrt:lcidtoname_downlevel.obj
 0002:00003a58       ??_C@_1M@KBMAIBFN@?$AAv?$AAi?$AA?9?$AAV?$AAN?$AA?$AA@ 10017a58     libucrt:lcidtoname_downlevel.obj
 0002:00003a64       ??_C@_1M@GPCBKDJK@?$AAh?$AAy?$AA?9?$AAA?$AAM?$AA?$AA@ 10017a64     libucrt:lcidtoname_downlevel.obj
 0002:00003a70       ??_C@_1BG@BECMDDJB@?$AAa?$AAz?$AA?9?$AAA?$AAZ?$AA?9?$AAL?$AAa?$AAt?$AAn?$AA?$AA@ 10017a70     libucrt:lcidtoname_downlevel.obj
 0002:00003a88       ??_C@_1M@MAOFCAEA@?$AAe?$AAu?$AA?9?$AAE?$AAS?$AA?$AA@ 10017a88     libucrt:lcidtoname_downlevel.obj
 0002:00003a94       ??_C@_1M@IGHABKPI@?$AAm?$AAk?$AA?9?$AAM?$AAK?$AA?$AA@ 10017a94     libucrt:lcidtoname_downlevel.obj
 0002:00003aa0       ??_C@_1M@IAIGNEJG@?$AAt?$AAn?$AA?9?$AAZ?$AAA?$AA?$AA@ 10017aa0     libucrt:lcidtoname_downlevel.obj
 0002:00003aac       ??_C@_1M@IIJCOJFA@?$AAx?$AAh?$AA?9?$AAZ?$AAA?$AA?$AA@ 10017aac     libucrt:lcidtoname_downlevel.obj
 0002:00003ab8       ??_C@_1M@LGPJHNJH@?$AAz?$AAu?$AA?9?$AAZ?$AAA?$AA?$AA@ 10017ab8     libucrt:lcidtoname_downlevel.obj
 0002:00003ac4       ??_C@_1M@HOKAOIO@?$AAa?$AAf?$AA?9?$AAZ?$AAA?$AA?$AA@ 10017ac4     libucrt:lcidtoname_downlevel.obj
 0002:00003ad0       ??_C@_1M@DPCLHLIE@?$AAk?$AAa?$AA?9?$AAG?$AAE?$AA?$AA@ 10017ad0     libucrt:lcidtoname_downlevel.obj
 0002:00003adc       ??_C@_1M@BLKMHJBI@?$AAf?$AAo?$AA?9?$AAF?$AAO?$AA?$AA@ 10017adc     libucrt:lcidtoname_downlevel.obj
 0002:00003ae8       ??_C@_1M@LGGJAPPB@?$AAh?$AAi?$AA?9?$AAI?$AAN?$AA?$AA@ 10017ae8     libucrt:lcidtoname_downlevel.obj
 0002:00003af4       ??_C@_1M@FIKPIHFE@?$AAm?$AAt?$AA?9?$AAM?$AAT?$AA?$AA@ 10017af4     libucrt:lcidtoname_downlevel.obj
 0002:00003b00       ??_C@_1M@HEGGPBFA@?$AAs?$AAe?$AA?9?$AAN?$AAO?$AA?$AA@ 10017b00     libucrt:lcidtoname_downlevel.obj
 0002:00003b0c       ??_C@_1M@EIBJEEPA@?$AAm?$AAs?$AA?9?$AAM?$AAY?$AA?$AA@ 10017b0c     libucrt:lcidtoname_downlevel.obj
 0002:00003b18       ??_C@_1M@FHLBGMPP@?$AAk?$AAk?$AA?9?$AAK?$AAZ?$AA?$AA@ 10017b18     libucrt:lcidtoname_downlevel.obj
 0002:00003b24       ??_C@_1M@NGJJLCGI@?$AAk?$AAy?$AA?9?$AAK?$AAG?$AA?$AA@ 10017b24     libucrt:lcidtoname_downlevel.obj
 0002:00003b30       ??_C@_1M@GIENNBFC@?$AAs?$AAw?$AA?9?$AAK?$AAE?$AA?$AA@ 10017b30     libucrt:lcidtoname_downlevel.obj
 0002:00003b3c       ??_C@_1BG@NDGMJIMJ@?$AAu?$AAz?$AA?9?$AAU?$AAZ?$AA?9?$AAL?$AAa?$AAt?$AAn?$AA?$AA@ 10017b3c     libucrt:lcidtoname_downlevel.obj
 0002:00003b54       ??_C@_1M@IDCCIHBC@?$AAt?$AAt?$AA?9?$AAR?$AAU?$AA?$AA@ 10017b54     libucrt:lcidtoname_downlevel.obj
 0002:00003b60       ??_C@_1M@LOICPMOJ@?$AAb?$AAn?$AA?9?$AAI?$AAN?$AA?$AA@ 10017b60     libucrt:lcidtoname_downlevel.obj
 0002:00003b6c       ??_C@_1M@KPKKNEAH@?$AAp?$AAa?$AA?9?$AAI?$AAN?$AA?$AA@ 10017b6c     libucrt:lcidtoname_downlevel.obj
 0002:00003b78       ??_C@_1M@PJGPPBOG@?$AAg?$AAu?$AA?9?$AAI?$AAN?$AA?$AA@ 10017b78     libucrt:lcidtoname_downlevel.obj
 0002:00003b84       ??_C@_1M@KMKMOPHI@?$AAt?$AAa?$AA?9?$AAI?$AAN?$AA?$AA@ 10017b84     libucrt:lcidtoname_downlevel.obj
 0002:00003b90       ??_C@_1M@KFEHEPAC@?$AAt?$AAe?$AA?9?$AAI?$AAN?$AA?$AA@ 10017b90     libucrt:lcidtoname_downlevel.obj
 0002:00003b9c       ??_C@_1M@CDCLMGHI@?$AAk?$AAn?$AA?9?$AAI?$AAN?$AA?$AA@ 10017b9c     libucrt:lcidtoname_downlevel.obj
 0002:00003ba8       ??_C@_1M@MIODLDKF@?$AAm?$AAl?$AA?9?$AAI?$AAN?$AA?$AA@ 10017ba8     libucrt:lcidtoname_downlevel.obj
 0002:00003bb4       ??_C@_1M@PBIEACPO@?$AAm?$AAr?$AA?9?$AAI?$AAN?$AA?$AA@ 10017bb4     libucrt:lcidtoname_downlevel.obj
 0002:00003bc0       ??_C@_1M@NIDEAGPH@?$AAs?$AAa?$AA?9?$AAI?$AAN?$AA?$AA@ 10017bc0     libucrt:lcidtoname_downlevel.obj
 0002:00003bcc       ??_C@_1M@FHIHCBIO@?$AAm?$AAn?$AA?9?$AAM?$AAN?$AA?$AA@ 10017bcc     libucrt:lcidtoname_downlevel.obj
 0002:00003bd8       ??_C@_1M@JAIJPENP@?$AAc?$AAy?$AA?9?$AAG?$AAB?$AA?$AA@ 10017bd8     libucrt:lcidtoname_downlevel.obj
 0002:00003be4       ??_C@_1M@PHGFBEPN@?$AAg?$AAl?$AA?9?$AAE?$AAS?$AA?$AA@ 10017be4     libucrt:lcidtoname_downlevel.obj
 0002:00003bf0       ??_C@_1O@KPIPDNCP@?$AAk?$AAo?$AAk?$AA?9?$AAI?$AAN?$AA?$AA@ 10017bf0     libucrt:lcidtoname_downlevel.obj
 0002:00003c00       ??_C@_1O@KNHJLDJA@?$AAs?$AAy?$AAr?$AA?9?$AAS?$AAY?$AA?$AA@ 10017c00     libucrt:lcidtoname_downlevel.obj
 0002:00003c10       ??_C@_1O@MKEKBLAH@?$AAd?$AAi?$AAv?$AA?9?$AAM?$AAV?$AA?$AA@ 10017c10     libucrt:lcidtoname_downlevel.obj
 0002:00003c20       ??_C@_1O@OHDCKDDF@?$AAq?$AAu?$AAz?$AA?9?$AAB?$AAO?$AA?$AA@ 10017c20     libucrt:lcidtoname_downlevel.obj
 0002:00003c30       ??_C@_1M@LEPJNLFD@?$AAn?$AAs?$AA?9?$AAZ?$AAA?$AA?$AA@ 10017c30     libucrt:lcidtoname_downlevel.obj
 0002:00003c3c       ??_C@_1M@OMLEIIJB@?$AAm?$AAi?$AA?9?$AAN?$AAZ?$AA?$AA@ 10017c3c     libucrt:lcidtoname_downlevel.obj
 0002:00003c48       ??_C@_1M@PMPEAILG@?$AAa?$AAr?$AA?9?$AAI?$AAQ?$AA?$AA@ 10017c48     libucrt:lcidtoname_downlevel.obj
 0002:00003c54       ??_C@_1M@CNKPNOEE@?$AAd?$AAe?$AA?9?$AAC?$AAH?$AA?$AA@ 10017c54     libucrt:lcidtoname_downlevel.obj
 0002:00003c60       ??_C@_1M@LKMGMLKO@?$AAe?$AAn?$AA?9?$AAG?$AAB?$AA?$AA@ 10017c60     libucrt:lcidtoname_downlevel.obj
 0002:00003c6c       ??_C@_1M@PGKJFFGL@?$AAe?$AAs?$AA?9?$AAM?$AAX?$AA?$AA@ 10017c6c     libucrt:lcidtoname_downlevel.obj
 0002:00003c78       ??_C@_1M@DNNANBDC@?$AAf?$AAr?$AA?9?$AAB?$AAE?$AA?$AA@ 10017c78     libucrt:lcidtoname_downlevel.obj
 0002:00003c84       ??_C@_1M@HLGMDFHM@?$AAi?$AAt?$AA?9?$AAC?$AAH?$AA?$AA@ 10017c84     libucrt:lcidtoname_downlevel.obj
 0002:00003c90       ??_C@_1M@CLLBGJH@?$AAn?$AAl?$AA?9?$AAB?$AAE?$AA?$AA@ 10017c90     libucrt:lcidtoname_downlevel.obj
 0002:00003c9c       ??_C@_1M@BODBOGLF@?$AAn?$AAn?$AA?9?$AAN?$AAO?$AA?$AA@ 10017c9c     libucrt:lcidtoname_downlevel.obj
 0002:00003ca8       ??_C@_1M@HFFAHKAD@?$AAp?$AAt?$AA?9?$AAP?$AAT?$AA?$AA@ 10017ca8     libucrt:lcidtoname_downlevel.obj
 0002:00003cb4       ??_C@_1BG@LNOAKHIE@?$AAs?$AAr?$AA?9?$AAS?$AAP?$AA?9?$AAL?$AAa?$AAt?$AAn?$AA?$AA@ 10017cb4     libucrt:lcidtoname_downlevel.obj
 0002:00003ccc       ??_C@_1M@HBMHBGAK@?$AAs?$AAv?$AA?9?$AAF?$AAI?$AA?$AA@ 10017ccc     libucrt:lcidtoname_downlevel.obj
 0002:00003cd8       ??_C@_1BG@DGCJGJBE@?$AAa?$AAz?$AA?9?$AAA?$AAZ?$AA?9?$AAC?$AAy?$AAr?$AAl?$AA?$AA@ 10017cd8     libucrt:lcidtoname_downlevel.obj
 0002:00003cf0       ??_C@_1M@KEJDAAHB@?$AAs?$AAe?$AA?9?$AAS?$AAE?$AA?$AA@ 10017cf0     libucrt:lcidtoname_downlevel.obj
 0002:00003cfc       ??_C@_1M@HEIBJJAD@?$AAm?$AAs?$AA?9?$AAB?$AAN?$AA?$AA@ 10017cfc     libucrt:lcidtoname_downlevel.obj
 0002:00003d08       ??_C@_1BG@PBGJMCEM@?$AAu?$AAz?$AA?9?$AAU?$AAZ?$AA?9?$AAC?$AAy?$AAr?$AAl?$AA?$AA@ 10017d08     libucrt:lcidtoname_downlevel.obj
 0002:00003d20       ??_C@_1O@LAOBCMDF@?$AAq?$AAu?$AAz?$AA?9?$AAE?$AAC?$AA?$AA@ 10017d20     libucrt:lcidtoname_downlevel.obj
 0002:00003d30       ??_C@_1M@POEEMAIO@?$AAa?$AAr?$AA?9?$AAE?$AAG?$AA?$AA@ 10017d30     libucrt:lcidtoname_downlevel.obj
 0002:00003d3c       ??_C@_1M@EFAKDEDL@?$AAz?$AAh?$AA?9?$AAH?$AAK?$AA?$AA@ 10017d3c     libucrt:lcidtoname_downlevel.obj
 0002:00003d48       ??_C@_1M@HKKIJHGI@?$AAd?$AAe?$AA?9?$AAA?$AAT?$AA?$AA@ 10017d48     libucrt:lcidtoname_downlevel.obj
 0002:00003d54       ??_C@_1M@KBFBEHJF@?$AAe?$AAn?$AA?9?$AAA?$AAU?$AA?$AA@ 10017d54     libucrt:lcidtoname_downlevel.obj
 0002:00003d60       ??_C@_1M@MNPLFAAH@?$AAe?$AAs?$AA?9?$AAE?$AAS?$AA?$AA@ 10017d60     libucrt:lcidtoname_downlevel.obj
 0002:00003d6c       ??_C@_1M@HJOOJFMA@?$AAf?$AAr?$AA?9?$AAC?$AAA?$AA?$AA@ 10017d6c     libucrt:lcidtoname_downlevel.obj
 0002:00003d78       ??_C@_1BG@JPOFPNAB@?$AAs?$AAr?$AA?9?$AAS?$AAP?$AA?9?$AAC?$AAy?$AAr?$AAl?$AA?$AA@ 10017d78     libucrt:lcidtoname_downlevel.obj
 0002:00003d90       ??_C@_1M@LNFOCMOB@?$AAs?$AAe?$AA?9?$AAF?$AAI?$AA?$AA@ 10017d90     libucrt:lcidtoname_downlevel.obj
 0002:00003d9c       ??_C@_1O@MGJBOAMB@?$AAq?$AAu?$AAz?$AA?9?$AAP?$AAE?$AA?$AA@ 10017d9c     libucrt:lcidtoname_downlevel.obj
 0002:00003dac       ??_C@_1M@GJINLBOK@?$AAa?$AAr?$AA?9?$AAL?$AAY?$AA?$AA@ 10017dac     libucrt:lcidtoname_downlevel.obj
 0002:00003db8       ??_C@_1M@GGMNHJNL@?$AAz?$AAh?$AA?9?$AAS?$AAG?$AA?$AA@ 10017db8     libucrt:lcidtoname_downlevel.obj
 0002:00003dc4       ??_C@_1M@HOIKODND@?$AAd?$AAe?$AA?9?$AAL?$AAU?$AA?$AA@ 10017dc4     libucrt:lcidtoname_downlevel.obj
 0002:00003dd0       ??_C@_1M@DDOCCGFG@?$AAe?$AAn?$AA?9?$AAC?$AAA?$AA?$AA@ 10017dd0     libucrt:lcidtoname_downlevel.obj
 0002:00003ddc       ??_C@_1M@BNOEMJLF@?$AAe?$AAs?$AA?9?$AAG?$AAT?$AA?$AA@ 10017ddc     libucrt:lcidtoname_downlevel.obj
 0002:00003de8       ??_C@_1M@EOGNKEK@?$AAf?$AAr?$AA?9?$AAC?$AAH?$AA?$AA@ 10017de8     libucrt:lcidtoname_downlevel.obj
 0002:00003df4       ??_C@_1M@FLIDJFHL@?$AAh?$AAr?$AA?9?$AAB?$AAA?$AA?$AA@ 10017df4     libucrt:lcidtoname_downlevel.obj
 0002:00003e00       ??_C@_1O@FMCELNAJ@?$AAs?$AAm?$AAj?$AA?9?$AAN?$AAO?$AA?$AA@ 10017e00     libucrt:lcidtoname_downlevel.obj
 0002:00003e10       ??_C@_1M@JHGLJMGJ@?$AAa?$AAr?$AA?9?$AAD?$AAZ?$AA?$AA@ 10017e10     libucrt:lcidtoname_downlevel.obj
 0002:00003e1c       ??_C@_1M@JKKFDCNP@?$AAz?$AAh?$AA?9?$AAM?$AAO?$AA?$AA@ 10017e1c     libucrt:lcidtoname_downlevel.obj
 0002:00003e28       ??_C@_1M@GEEFALPE@?$AAd?$AAe?$AA?9?$AAL?$AAI?$AA?$AA@ 10017e28     libucrt:lcidtoname_downlevel.obj
 0002:00003e34       ??_C@_1M@IGEOFBG@?$AAe?$AAn?$AA?9?$AAN?$AAZ?$AA?$AA@ 10017e34     libucrt:lcidtoname_downlevel.obj
 0002:00003e40       ??_C@_1M@KDBONEHP@?$AAe?$AAs?$AA?9?$AAC?$AAR?$AA?$AA@ 10017e40     libucrt:lcidtoname_downlevel.obj
 0002:00003e4c       ??_C@_1M@FHMDOHNN@?$AAf?$AAr?$AA?9?$AAL?$AAU?$AA?$AA@ 10017e4c     libucrt:lcidtoname_downlevel.obj
 0002:00003e58       ??_C@_1BG@NFKKMAFG@?$AAb?$AAs?$AA?9?$AAB?$AAA?$AA?9?$AAL?$AAa?$AAt?$AAn?$AA?$AA@ 10017e58     libucrt:lcidtoname_downlevel.obj
 0002:00003e70       ??_C@_1O@IMNBEMCI@?$AAs?$AAm?$AAj?$AA?9?$AAS?$AAE?$AA?$AA@ 10017e70     libucrt:lcidtoname_downlevel.obj
 0002:00003e80       ??_C@_1M@DHHMBNDP@?$AAa?$AAr?$AA?9?$AAM?$AAA?$AA?$AA@ 10017e80     libucrt:lcidtoname_downlevel.obj
 0002:00003e8c       ??_C@_1M@BNBLJCGH@?$AAe?$AAn?$AA?9?$AAI?$AAE?$AA?$AA@ 10017e8c     libucrt:lcidtoname_downlevel.obj
 0002:00003e98       ??_C@_1M@GEPAFMDL@?$AAe?$AAs?$AA?9?$AAP?$AAA?$AA?$AA@ 10017e98     libucrt:lcidtoname_downlevel.obj
 0002:00003ea4       ??_C@_1M@OJONDMDL@?$AAf?$AAr?$AA?9?$AAM?$AAC?$AA?$AA@ 10017ea4     libucrt:lcidtoname_downlevel.obj
 0002:00003eb0       ??_C@_1BG@OBCNFJB@?$AAs?$AAr?$AA?9?$AAB?$AAA?$AA?9?$AAL?$AAa?$AAt?$AAn?$AA?$AA@ 10017eb0     libucrt:lcidtoname_downlevel.obj
 0002:00003ec8       ??_C@_1O@KEMEEGPO@?$AAs?$AAm?$AAa?$AA?9?$AAN?$AAO?$AA?$AA@ 10017ec8     libucrt:lcidtoname_downlevel.obj
 0002:00003ed8       ??_C@_1M@ELMGFODK@?$AAa?$AAr?$AA?9?$AAT?$AAN?$AA?$AA@ 10017ed8     libucrt:lcidtoname_downlevel.obj
 0002:00003ee4       ??_C@_1M@BHDLHFAF@?$AAe?$AAn?$AA?9?$AAZ?$AAA?$AA?$AA@ 10017ee4     libucrt:lcidtoname_downlevel.obj
 0002:00003ef0       ??_C@_1M@BMGIGLIF@?$AAe?$AAs?$AA?9?$AAD?$AAO?$AA?$AA@ 10017ef0     libucrt:lcidtoname_downlevel.obj
 0002:00003efc       ??_C@_1BG@CMBHIPBE@?$AAs?$AAr?$AA?9?$AAB?$AAA?$AA?9?$AAC?$AAy?$AAr?$AAl?$AA?$AA@ 10017efc     libucrt:lcidtoname_downlevel.obj
 0002:00003f14       ??_C@_1O@HEDBLHNP@?$AAs?$AAm?$AAa?$AA?9?$AAS?$AAE?$AA?$AA@ 10017f14     libucrt:lcidtoname_downlevel.obj
 0002:00003f24       ??_C@_1M@DAGCADIM@?$AAa?$AAr?$AA?9?$AAO?$AAM?$AA?$AA@ 10017f24     libucrt:lcidtoname_downlevel.obj
 0002:00003f30       ??_C@_1M@FODLMICG@?$AAe?$AAn?$AA?9?$AAJ?$AAM?$AA?$AA@ 10017f30     libucrt:lcidtoname_downlevel.obj
 0002:00003f3c       ??_C@_1M@DNMLCIHB@?$AAe?$AAs?$AA?9?$AAV?$AAE?$AA?$AA@ 10017f3c     libucrt:lcidtoname_downlevel.obj
 0002:00003f48       ??_C@_1O@EOKHMKJK@?$AAs?$AAm?$AAs?$AA?9?$AAF?$AAI?$AA?$AA@ 10017f48     libucrt:lcidtoname_downlevel.obj
 0002:00003f58       ??_C@_1M@CAFJMKOF@?$AAa?$AAr?$AA?9?$AAY?$AAE?$AA?$AA@ 10017f58     libucrt:lcidtoname_downlevel.obj
 0002:00003f64       ??_C@_1M@CBFHIJLI@?$AAe?$AAn?$AA?9?$AAC?$AAB?$AA?$AA@ 10017f64     libucrt:lcidtoname_downlevel.obj
 0002:00003f70       ??_C@_1M@BGNFLDN@?$AAe?$AAs?$AA?9?$AAC?$AAO?$AA?$AA@ 10017f70     libucrt:lcidtoname_downlevel.obj
 0002:00003f7c       ??_C@_1O@JMPHMAMC@?$AAs?$AAm?$AAn?$AA?9?$AAF?$AAI?$AA?$AA@ 10017f7c     libucrt:lcidtoname_downlevel.obj
 0002:00003f8c       ??_C@_1M@JLANABKE@?$AAa?$AAr?$AA?9?$AAS?$AAY?$AA?$AA@ 10017f8c     libucrt:lcidtoname_downlevel.obj
 0002:00003f98       ??_C@_1M@HPKGCFGN@?$AAe?$AAn?$AA?9?$AAB?$AAZ?$AA?$AA@ 10017f98     libucrt:lcidtoname_downlevel.obj
 0002:00003fa4       ??_C@_1M@OLJCMLGM@?$AAe?$AAs?$AA?9?$AAP?$AAE?$AA?$AA@ 10017fa4     libucrt:lcidtoname_downlevel.obj
 0002:00003fb0       ??_C@_1M@MKKGFKLE@?$AAa?$AAr?$AA?9?$AAJ?$AAO?$AA?$AA@ 10017fb0     libucrt:lcidtoname_downlevel.obj
 0002:00003fbc       ??_C@_1M@EKPGLDNI@?$AAe?$AAn?$AA?9?$AAT?$AAT?$AA?$AA@ 10017fbc     libucrt:lcidtoname_downlevel.obj
 0002:00003fc8       ??_C@_1M@OONGHFHE@?$AAe?$AAs?$AA?9?$AAA?$AAR?$AA?$AA@ 10017fc8     libucrt:lcidtoname_downlevel.obj
 0002:00003fd4       ??_C@_1M@OOJFGBHE@?$AAa?$AAr?$AA?9?$AAL?$AAB?$AA?$AA@ 10017fd4     libucrt:lcidtoname_downlevel.obj
 0002:00003fe0       ??_C@_1M@GCEJHNEG@?$AAe?$AAn?$AA?9?$AAZ?$AAW?$AA?$AA@ 10017fe0     libucrt:lcidtoname_downlevel.obj
 0002:00003fec       ??_C@_1M@JNOCAHJI@?$AAe?$AAs?$AA?9?$AAE?$AAC?$AA?$AA@ 10017fec     libucrt:lcidtoname_downlevel.obj
 0002:00003ff8       ??_C@_1M@JEFHPGGB@?$AAa?$AAr?$AA?9?$AAK?$AAW?$AA?$AA@ 10017ff8     libucrt:lcidtoname_downlevel.obj
 0002:00004004       ??_C@_1M@MLKIBJOJ@?$AAe?$AAn?$AA?9?$AAP?$AAH?$AA?$AA@ 10018004     libucrt:lcidtoname_downlevel.obj
 0002:00004010       ??_C@_1M@BDNIPEND@?$AAe?$AAs?$AA?9?$AAC?$AAL?$AA?$AA@ 10018010     libucrt:lcidtoname_downlevel.obj
 0002:0000401c       ??_C@_1M@MPNMEKBD@?$AAa?$AAr?$AA?9?$AAA?$AAE?$AA?$AA@ 1001801c     libucrt:lcidtoname_downlevel.obj
 0002:00004028       ??_C@_1M@KBJALCPI@?$AAe?$AAs?$AA?9?$AAU?$AAY?$AA?$AA@ 10018028     libucrt:lcidtoname_downlevel.obj
 0002:00004034       ??_C@_1M@LLCCOAGA@?$AAa?$AAr?$AA?9?$AAB?$AAH?$AA?$AA@ 10018034     libucrt:lcidtoname_downlevel.obj
 0002:00004040       ??_C@_1M@PBFNCDEL@?$AAe?$AAs?$AA?9?$AAP?$AAY?$AA?$AA@ 10018040     libucrt:lcidtoname_downlevel.obj
 0002:0000404c       ??_C@_1M@EDGINPNP@?$AAa?$AAr?$AA?9?$AAQ?$AAA?$AA?$AA@ 1001804c     libucrt:lcidtoname_downlevel.obj
 0002:00004058       ??_C@_1M@MKDBIIJI@?$AAe?$AAs?$AA?9?$AAB?$AAO?$AA?$AA@ 10018058     libucrt:lcidtoname_downlevel.obj
 0002:00004064       ??_C@_1M@CPKKEBLD@?$AAe?$AAs?$AA?9?$AAS?$AAV?$AA?$AA@ 10018064     libucrt:lcidtoname_downlevel.obj
 0002:00004070       ??_C@_1M@NDBGMMJL@?$AAe?$AAs?$AA?9?$AAH?$AAN?$AA?$AA@ 10018070     libucrt:lcidtoname_downlevel.obj
 0002:0000407c       ??_C@_1M@JIJIBHDP@?$AAe?$AAs?$AA?9?$AAN?$AAI?$AA?$AA@ 1001807c     libucrt:lcidtoname_downlevel.obj
 0002:00004088       ??_C@_1M@CGFMKEEK@?$AAe?$AAs?$AA?9?$AAP?$AAR?$AA?$AA@ 10018088     libucrt:lcidtoname_downlevel.obj
 0002:00004094       ??_C@_1O@ICJHKIIK@?$AAz?$AAh?$AA?9?$AAC?$AAH?$AAT?$AA?$AA@ 10018094     libucrt:lcidtoname_downlevel.obj
 0002:000040a4       ??_C@_15CLNEJCE@?$AAs?$AAr?$AA?$AA@ 100180a4     libucrt:lcidtoname_downlevel.obj
 0002:000047d0       ??_C@_1M@KAHEKEIG@?$AAa?$AAf?$AA?9?$AAz?$AAa?$AA?$AA@ 100187d0     libucrt:lcidtoname_downlevel.obj
 0002:000047dc       ??_C@_1M@GIECOABL@?$AAa?$AAr?$AA?9?$AAa?$AAe?$AA?$AA@ 100187dc     libucrt:lcidtoname_downlevel.obj
 0002:000047e8       ??_C@_1M@BMLMEKGI@?$AAa?$AAr?$AA?9?$AAb?$AAh?$AA?$AA@ 100187e8     libucrt:lcidtoname_downlevel.obj
 0002:000047f4       ??_C@_1M@DAPFDGGB@?$AAa?$AAr?$AA?9?$AAd?$AAz?$AA?$AA@ 100187f4     libucrt:lcidtoname_downlevel.obj
 0002:00004800       ??_C@_1M@FJNKGKIG@?$AAa?$AAr?$AA?9?$AAe?$AAg?$AA?$AA@ 10018800     libucrt:lcidtoname_downlevel.obj
 0002:0000480c       ??_C@_1M@FLGKKCLO@?$AAa?$AAr?$AA?9?$AAi?$AAq?$AA?$AA@ 1001880c     libucrt:lcidtoname_downlevel.obj
 0002:00004818       ??_C@_1M@GNDIPALM@?$AAa?$AAr?$AA?9?$AAj?$AAo?$AA?$AA@ 10018818     libucrt:lcidtoname_downlevel.obj
 0002:00004824       ??_C@_1M@DDMJFMGJ@?$AAa?$AAr?$AA?9?$AAk?$AAw?$AA?$AA@ 10018824     libucrt:lcidtoname_downlevel.obj
 0002:00004830       ??_C@_1M@EJALMLHM@?$AAa?$AAr?$AA?9?$AAl?$AAb?$AA?$AA@ 10018830     libucrt:lcidtoname_downlevel.obj
 0002:0000483c       ??_C@_1M@MOBDBLOC@?$AAa?$AAr?$AA?9?$AAl?$AAy?$AA?$AA@ 1001883c     libucrt:lcidtoname_downlevel.obj
 0002:00004848       ??_C@_1M@JAOCLHDH@?$AAa?$AAr?$AA?9?$AAm?$AAa?$AA?$AA@ 10018848     libucrt:lcidtoname_downlevel.obj
 0002:00004854       ??_C@_1M@JHPMKJIE@?$AAa?$AAr?$AA?9?$AAo?$AAm?$AA?$AA@ 10018854     libucrt:lcidtoname_downlevel.obj
 0002:00004860       ??_C@_1M@OEPGHFNH@?$AAa?$AAr?$AA?9?$AAq?$AAa?$AA?$AA@ 10018860     libucrt:lcidtoname_downlevel.obj
 0002:0000486c       ??_C@_1M@KJDONENM@?$AAa?$AAr?$AA?9?$AAs?$AAa?$AA?$AA@ 1001886c     libucrt:lcidtoname_downlevel.obj
 0002:00004878       ??_C@_1M@DMJDKLKM@?$AAa?$AAr?$AA?9?$AAs?$AAy?$AA?$AA@ 10018878     libucrt:lcidtoname_downlevel.obj
 0002:00004884       ??_C@_1M@OMFIPEDC@?$AAa?$AAr?$AA?9?$AAt?$AAn?$AA?$AA@ 10018884     libucrt:lcidtoname_downlevel.obj
 0002:00004890       ??_C@_1M@IHMHGAON@?$AAa?$AAr?$AA?9?$AAy?$AAe?$AA?$AA@ 10018890     libucrt:lcidtoname_downlevel.obj
 0002:0000489c       ??_C@_1BG@KDCPGJGB@?$AAa?$AAz?$AA?9?$AAa?$AAz?$AA?9?$AAc?$AAy?$AAr?$AAl?$AA?$AA@ 1001889c     libucrt:lcidtoname_downlevel.obj
 0002:000048b4       ??_C@_1BG@IBCKDDOE@?$AAa?$AAz?$AA?9?$AAa?$AAz?$AA?9?$AAl?$AAa?$AAt?$AAn?$AA?$AA@ 100188b4     libucrt:lcidtoname_downlevel.obj
 0002:000048cc       ??_C@_1M@EGPFDCPD@?$AAb?$AAe?$AA?9?$AAb?$AAy?$AA?$AA@ 100188cc     libucrt:lcidtoname_downlevel.obj
 0002:000048d8       ??_C@_1M@PCMGMCGC@?$AAb?$AAg?$AA?9?$AAb?$AAg?$AA?$AA@ 100188d8     libucrt:lcidtoname_downlevel.obj
 0002:000048e4       ??_C@_1M@BJBMFGOB@?$AAb?$AAn?$AA?9?$AAi?$AAn?$AA?$AA@ 100188e4     libucrt:lcidtoname_downlevel.obj
 0002:000048f0       ??_C@_1BG@EAKMMACD@?$AAb?$AAs?$AA?9?$AAb?$AAa?$AA?9?$AAl?$AAa?$AAt?$AAn?$AA?$AA@ 100188f0     libucrt:lcidtoname_downlevel.obj
 0002:00004908       ??_C@_1M@KGADAODK@?$AAc?$AAa?$AA?9?$AAe?$AAs?$AA?$AA@ 10018908     libucrt:lcidtoname_downlevel.obj
 0002:00004914       ??_C@_1M@COAJPDHI@?$AAc?$AAs?$AA?9?$AAc?$AAz?$AA?$AA@ 10018914     libucrt:lcidtoname_downlevel.obj
 0002:00004920       ??_C@_1M@DHBHFONH@?$AAc?$AAy?$AA?9?$AAg?$AAb?$AA?$AA@ 10018920     libucrt:lcidtoname_downlevel.obj
 0002:0000492c       ??_C@_1M@IMGKELGA@?$AAd?$AAa?$AA?9?$AAd?$AAk?$AA?$AA@ 1001892c     libucrt:lcidtoname_downlevel.obj
 0002:00004938       ??_C@_1M@NNDGDNGA@?$AAd?$AAe?$AA?9?$AAa?$AAt?$AA?$AA@ 10018938     libucrt:lcidtoname_downlevel.obj
 0002:00004944       ??_C@_1M@IKDBHEEM@?$AAd?$AAe?$AA?9?$AAc?$AAh?$AA?$AA@ 10018944     libucrt:lcidtoname_downlevel.obj
 0002:00004950       ??_C@_1M@GFFOJMCJ@?$AAd?$AAe?$AA?9?$AAd?$AAe?$AA?$AA@ 10018950     libucrt:lcidtoname_downlevel.obj
 0002:0000495c       ??_C@_1M@MDNLKBPM@?$AAd?$AAe?$AA?9?$AAl?$AAi?$AA?$AA@ 1001895c     libucrt:lcidtoname_downlevel.obj
 0002:00004968       ??_C@_1M@NJBEEJNL@?$AAd?$AAe?$AA?9?$AAl?$AAu?$AA?$AA@ 10018968     libucrt:lcidtoname_downlevel.obj
 0002:00004974       ??_C@_1O@GNNELBAP@?$AAd?$AAi?$AAv?$AA?9?$AAm?$AAv?$AA?$AA@ 10018974     libucrt:lcidtoname_downlevel.obj
 0002:00004984       ??_C@_1M@EJLEOGAE@?$AAe?$AAl?$AA?9?$AAg?$AAr?$AA?$AA@ 10018984     libucrt:lcidtoname_downlevel.obj
 0002:00004990       ??_C@_1M@GMPONJN@?$AAe?$AAn?$AA?9?$AAa?$AAu?$AA?$AA@ 10018990     libucrt:lcidtoname_downlevel.obj
 0002:0000499c       ??_C@_1M@NIDIIPGF@?$AAe?$AAn?$AA?9?$AAb?$AAz?$AA?$AA@ 1001899c     libucrt:lcidtoname_downlevel.obj
 0002:000049a8       ??_C@_1M@JEHMIMFO@?$AAe?$AAn?$AA?9?$AAc?$AAa?$AA?$AA@ 100189a8     libucrt:lcidtoname_downlevel.obj
 0002:000049b4       ??_C@_1M@IGMJCDLA@?$AAe?$AAn?$AA?9?$AAc?$AAb?$AA?$AA@ 100189b4     libucrt:lcidtoname_downlevel.obj
 0002:000049c0       ??_C@_1M@BNFIGBKG@?$AAe?$AAn?$AA?9?$AAg?$AAb?$AA?$AA@ 100189c0     libucrt:lcidtoname_downlevel.obj
 0002:000049cc       ??_C@_1M@LKIFDIGP@?$AAe?$AAn?$AA?9?$AAi?$AAe?$AA?$AA@ 100189cc     libucrt:lcidtoname_downlevel.obj
 0002:000049d8       ??_C@_1M@PJKFGCCO@?$AAe?$AAn?$AA?9?$AAj?$AAm?$AA?$AA@ 100189d8     libucrt:lcidtoname_downlevel.obj
 0002:000049e4       ??_C@_1M@KPPKEPBO@?$AAe?$AAn?$AA?9?$AAn?$AAz?$AA?$AA@ 100189e4     libucrt:lcidtoname_downlevel.obj
 0002:000049f0       ??_C@_1M@GMDGLDOB@?$AAe?$AAn?$AA?9?$AAp?$AAh?$AA?$AA@ 100189f0     libucrt:lcidtoname_downlevel.obj
 0002:000049fc       ??_C@_1M@ONGIBJNA@?$AAe?$AAn?$AA?9?$AAt?$AAt?$AA?$AA@ 100189fc     libucrt:lcidtoname_downlevel.obj
 0002:00004a08       ??_C@_1M@LLODPCMM@?$AAe?$AAn?$AA?9?$AAu?$AAs?$AA?$AA@ 10018a08     libucrt:lcidtoname_downlevel.obj
 0002:00004a14       ??_C@_1M@LAKFNPAN@?$AAe?$AAn?$AA?9?$AAz?$AAa?$AA?$AA@ 10018a14     libucrt:lcidtoname_downlevel.obj
 0002:00004a20       ??_C@_1M@MFNHNHEO@?$AAe?$AAn?$AA?9?$AAz?$AAw?$AA?$AA@ 10018a20     libucrt:lcidtoname_downlevel.obj
 0002:00004a2c       ??_C@_1M@EJEINPHM@?$AAe?$AAs?$AA?9?$AAa?$AAr?$AA?$AA@ 10018a2c     libucrt:lcidtoname_downlevel.obj
 0002:00004a38       ??_C@_1M@GNKPCCJA@?$AAe?$AAs?$AA?9?$AAb?$AAo?$AA?$AA@ 10018a38     libucrt:lcidtoname_downlevel.obj
 0002:00004a44       ??_C@_1M@LEEGFONL@?$AAe?$AAs?$AA?9?$AAc?$AAl?$AA?$AA@ 10018a44     libucrt:lcidtoname_downlevel.obj
 0002:00004a50       ??_C@_1M@KGPDPBDF@?$AAe?$AAs?$AA?9?$AAc?$AAo?$AA?$AA@ 10018a50     libucrt:lcidtoname_downlevel.obj
 0002:00004a5c       ??_C@_1M@EIAHOHH@?$AAe?$AAs?$AA?9?$AAc?$AAr?$AA?$AA@ 10018a5c     libucrt:lcidtoname_downlevel.obj
 0002:00004a68       ??_C@_1M@LLPGMBIN@?$AAe?$AAs?$AA?9?$AAd?$AAo?$AA?$AA@ 10018a68     libucrt:lcidtoname_downlevel.obj
 0002:00004a74       ??_C@_1M@DKHMKNJA@?$AAe?$AAs?$AA?9?$AAe?$AAc?$AA?$AA@ 10018a74     libucrt:lcidtoname_downlevel.obj
 0002:00004a80       ??_C@_1M@GKGFPKAP@?$AAe?$AAs?$AA?9?$AAe?$AAs?$AA?$AA@ 10018a80     libucrt:lcidtoname_downlevel.obj
 0002:00004a8c       ??_C@_1M@LKHKGDLN@?$AAe?$AAs?$AA?9?$AAg?$AAt?$AA?$AA@ 10018a8c     libucrt:lcidtoname_downlevel.obj
 0002:00004a98       ??_C@_1M@HEIIGGJD@?$AAe?$AAs?$AA?9?$AAh?$AAn?$AA?$AA@ 10018a98     libucrt:lcidtoname_downlevel.obj
 0002:00004aa4       ??_C@_1M@FBDHPPGD@?$AAe?$AAs?$AA?9?$AAm?$AAx?$AA?$AA@ 10018aa4     libucrt:lcidtoname_downlevel.obj
 0002:00004ab0       ??_C@_1M@DPAGLNDH@?$AAe?$AAs?$AA?9?$AAn?$AAi?$AA?$AA@ 10018ab0     libucrt:lcidtoname_downlevel.obj
 0002:00004abc       ??_C@_1M@MDGOPGDD@?$AAe?$AAs?$AA?9?$AAp?$AAa?$AA?$AA@ 10018abc     libucrt:lcidtoname_downlevel.obj
 0002:00004ac8       ??_C@_1M@EMAMGBGE@?$AAe?$AAs?$AA?9?$AAp?$AAe?$AA?$AA@ 10018ac8     libucrt:lcidtoname_downlevel.obj
 0002:00004ad4       ??_C@_1M@IBMCAOEC@?$AAe?$AAs?$AA?9?$AAp?$AAr?$AA?$AA@ 10018ad4     libucrt:lcidtoname_downlevel.obj
 0002:00004ae0       ??_C@_1M@FGMDIJED@?$AAe?$AAs?$AA?9?$AAp?$AAy?$AA?$AA@ 10018ae0     libucrt:lcidtoname_downlevel.obj
 0002:00004aec       ??_C@_1M@IIDEOLLL@?$AAe?$AAs?$AA?9?$AAs?$AAv?$AA?$AA@ 10018aec     libucrt:lcidtoname_downlevel.obj
 0002:00004af8       ??_C@_1M@GAOBIPA@?$AAe?$AAs?$AA?9?$AAu?$AAy?$AA?$AA@ 10018af8     libucrt:lcidtoname_downlevel.obj
 0002:00004b04       ??_C@_1M@JKFFICHJ@?$AAe?$AAs?$AA?9?$AAv?$AAe?$AA?$AA@ 10018b04     libucrt:lcidtoname_downlevel.obj
 0002:00004b10       ??_C@_1M@PNMLOJDF@?$AAe?$AAt?$AA?9?$AAe?$AAe?$AA?$AA@ 10018b10     libucrt:lcidtoname_downlevel.obj
 0002:00004b1c       ??_C@_1M@GHHLIKEI@?$AAe?$AAu?$AA?9?$AAe?$AAs?$AA?$AA@ 10018b1c     libucrt:lcidtoname_downlevel.obj
 0002:00004b28       ??_C@_1M@PBNONODE@?$AAf?$AAa?$AA?9?$AAi?$AAr?$AA?$AA@ 10018b28     libucrt:lcidtoname_downlevel.obj
 0002:00004b34       ??_C@_1M@JEEHPMIL@?$AAf?$AAi?$AA?9?$AAf?$AAi?$AA?$AA@ 10018b34     libucrt:lcidtoname_downlevel.obj
 0002:00004b40       ??_C@_1M@LMDCNDBA@?$AAf?$AAo?$AA?9?$AAf?$AAo?$AA?$AA@ 10018b40     libucrt:lcidtoname_downlevel.obj
 0002:00004b4c       ??_C@_1M@JKEOHLDK@?$AAf?$AAr?$AA?9?$AAb?$AAe?$AA?$AA@ 10018b4c     libucrt:lcidtoname_downlevel.obj
 0002:00004b58       ??_C@_1M@NOHADPMI@?$AAf?$AAr?$AA?9?$AAc?$AAa?$AA?$AA@ 10018b58     libucrt:lcidtoname_downlevel.obj
 0002:00004b64       ??_C@_1M@KDHIHAEC@?$AAf?$AAr?$AA?9?$AAc?$AAh?$AA?$AA@ 10018b64     libucrt:lcidtoname_downlevel.obj
 0002:00004b70       ??_C@_1M@MMBBFGAK@?$AAf?$AAr?$AA?9?$AAf?$AAr?$AA?$AA@ 10018b70     libucrt:lcidtoname_downlevel.obj
 0002:00004b7c       ??_C@_1M@PAFNENNF@?$AAf?$AAr?$AA?9?$AAl?$AAu?$AA?$AA@ 10018b7c     libucrt:lcidtoname_downlevel.obj
 0002:00004b88       ??_C@_1M@EOHDJGDD@?$AAf?$AAr?$AA?9?$AAm?$AAc?$AA?$AA@ 10018b88     libucrt:lcidtoname_downlevel.obj
 0002:00004b94       ??_C@_1M@FAPLLOPF@?$AAg?$AAl?$AA?9?$AAe?$AAs?$AA?$AA@ 10018b94     libucrt:lcidtoname_downlevel.obj
 0002:00004ba0       ??_C@_1M@FOPBFLOO@?$AAg?$AAu?$AA?9?$AAi?$AAn?$AA?$AA@ 10018ba0     libucrt:lcidtoname_downlevel.obj
 0002:00004bac       ??_C@_1M@KBMCINPM@?$AAh?$AAe?$AA?9?$AAi?$AAl?$AA?$AA@ 10018bac     libucrt:lcidtoname_downlevel.obj
 0002:00004bb8       ??_C@_1M@BBPHKFPJ@?$AAh?$AAi?$AA?9?$AAi?$AAn?$AA?$AA@ 10018bb8     libucrt:lcidtoname_downlevel.obj
 0002:00004bc4       ??_C@_1M@PMBNDPHD@?$AAh?$AAr?$AA?9?$AAb?$AAa?$AA?$AA@ 10018bc4     libucrt:lcidtoname_downlevel.obj
 0002:00004bd0       ??_C@_1M@BPCKOEGE@?$AAh?$AAr?$AA?9?$AAh?$AAr?$AA?$AA@ 10018bd0     libucrt:lcidtoname_downlevel.obj
 0002:00004bdc       ??_C@_1M@GACBMHKE@?$AAh?$AAu?$AA?9?$AAh?$AAu?$AA?$AA@ 10018bdc     libucrt:lcidtoname_downlevel.obj
 0002:00004be8       ??_C@_1M@MILPAJJC@?$AAh?$AAy?$AA?9?$AAa?$AAm?$AA?$AA@ 10018be8     libucrt:lcidtoname_downlevel.obj
 0002:00004bf4       ??_C@_1M@BABBICEC@?$AAi?$AAd?$AA?9?$AAi?$AAd?$AA?$AA@ 10018bf4     libucrt:lcidtoname_downlevel.obj
 0002:00004c00       ??_C@_1M@BIKNHHPF@?$AAi?$AAs?$AA?9?$AAi?$AAs?$AA?$AA@ 10018c00     libucrt:lcidtoname_downlevel.obj
 0002:00004c0c       ??_C@_1M@NMPCJPHE@?$AAi?$AAt?$AA?9?$AAc?$AAh?$AA?$AA@ 10018c0c     libucrt:lcidtoname_downlevel.obj
 0002:00004c18       ??_C@_1M@GHKGFEDF@?$AAi?$AAt?$AA?9?$AAi?$AAt?$AA?$AA@ 10018c18     libucrt:lcidtoname_downlevel.obj
 0002:00004c24       ??_C@_1M@NIEJCJJA@?$AAj?$AAa?$AA?9?$AAj?$AAp?$AA?$AA@ 10018c24     libucrt:lcidtoname_downlevel.obj
 0002:00004c30       ??_C@_1M@JILFNBIM@?$AAk?$AAa?$AA?9?$AAg?$AAe?$AA?$AA@ 10018c30     libucrt:lcidtoname_downlevel.obj
 0002:00004c3c       ??_C@_1M@PACPMGPH@?$AAk?$AAk?$AA?9?$AAk?$AAz?$AA?$AA@ 10018c3c     libucrt:lcidtoname_downlevel.obj
 0002:00004c48       ??_C@_1M@IELFGMHA@?$AAk?$AAn?$AA?9?$AAi?$AAn?$AA?$AA@ 10018c48     libucrt:lcidtoname_downlevel.obj
 0002:00004c54       ??_C@_1O@IBBJHCH@?$AAk?$AAo?$AAk?$AA?9?$AAi?$AAn?$AA?$AA@ 10018c54     libucrt:lcidtoname_downlevel.obj
 0002:00004c64       ??_C@_1M@DMHAEOGC@?$AAk?$AAo?$AA?9?$AAk?$AAr?$AA?$AA@ 10018c64     libucrt:lcidtoname_downlevel.obj
 0002:00004c70       ??_C@_1M@HBAHBIGA@?$AAk?$AAy?$AA?9?$AAk?$AAg?$AA?$AA@ 10018c70     libucrt:lcidtoname_downlevel.obj
 0002:00004c7c       ??_C@_1M@KPMILCJG@?$AAl?$AAt?$AA?9?$AAl?$AAt?$AA?$AA@ 10018c7c     libucrt:lcidtoname_downlevel.obj
 0002:00004c88       ??_C@_1M@BDEKKCA@?$AAl?$AAv?$AA?9?$AAl?$AAv?$AA?$AA@ 10018c88     libucrt:lcidtoname_downlevel.obj
 0002:00004c94       ??_C@_1M@ELCKCCJJ@?$AAm?$AAi?$AA?9?$AAn?$AAz?$AA?$AA@ 10018c94     libucrt:lcidtoname_downlevel.obj
 0002:00004ca0       ??_C@_1M@CBOOLAPA@?$AAm?$AAk?$AA?9?$AAm?$AAk?$AA?$AA@ 10018ca0     libucrt:lcidtoname_downlevel.obj
 0002:00004cac       ??_C@_1M@GPHNBJKN@?$AAm?$AAl?$AA?9?$AAi?$AAn?$AA?$AA@ 10018cac     libucrt:lcidtoname_downlevel.obj
 0002:00004cb8       ??_C@_1M@PABJILIG@?$AAm?$AAn?$AA?9?$AAm?$AAn?$AA?$AA@ 10018cb8     libucrt:lcidtoname_downlevel.obj
 0002:00004cc4       ??_C@_1M@FGBKKIPG@?$AAm?$AAr?$AA?9?$AAi?$AAn?$AA?$AA@ 10018cc4     libucrt:lcidtoname_downlevel.obj
 0002:00004cd0       ??_C@_1M@NDBPDDAL@?$AAm?$AAs?$AA?9?$AAb?$AAn?$AA?$AA@ 10018cd0     libucrt:lcidtoname_downlevel.obj
 0002:00004cdc       ??_C@_1M@OPIHOOPI@?$AAm?$AAs?$AA?9?$AAm?$AAy?$AA?$AA@ 10018cdc     libucrt:lcidtoname_downlevel.obj
 0002:00004ce8       ??_C@_1M@PPDBCNFM@?$AAm?$AAt?$AA?9?$AAm?$AAt?$AA?$AA@ 10018ce8     libucrt:lcidtoname_downlevel.obj
 0002:00004cf4       ??_C@_1M@KDJDKMDD@?$AAn?$AAb?$AA?9?$AAn?$AAo?$AA?$AA@ 10018cf4     libucrt:lcidtoname_downlevel.obj
 0002:00004d00       ??_C@_1M@KFCFLMJP@?$AAn?$AAl?$AA?9?$AAb?$AAe?$AA?$AA@ 10018d00     libucrt:lcidtoname_downlevel.obj
 0002:00004d0c       ??_C@_1M@KPOPDDGO@?$AAn?$AAl?$AA?9?$AAn?$AAl?$AA?$AA@ 10018d0c     libucrt:lcidtoname_downlevel.obj
 0002:00004d18       ??_C@_1M@LJKPEMLN@?$AAn?$AAn?$AA?9?$AAn?$AAo?$AA?$AA@ 10018d18     libucrt:lcidtoname_downlevel.obj
 0002:00004d24       ??_C@_1M@BDGHHBFL@?$AAn?$AAs?$AA?9?$AAz?$AAa?$AA?$AA@ 10018d24     libucrt:lcidtoname_downlevel.obj
 0002:00004d30       ??_C@_1M@IDEHOAP@?$AAp?$AAa?$AA?9?$AAi?$AAn?$AA?$AA@ 10018d30     libucrt:lcidtoname_downlevel.obj
 0002:00004d3c       ??_C@_1M@HDBKGOGH@?$AAp?$AAl?$AA?9?$AAp?$AAl?$AA?$AA@ 10018d3c     libucrt:lcidtoname_downlevel.obj
 0002:00004d48       ??_C@_1M@LJLLCMEH@?$AAp?$AAt?$AA?9?$AAb?$AAr?$AA?$AA@ 10018d48     libucrt:lcidtoname_downlevel.obj
 0002:00004d54       ??_C@_1M@NCMONAAL@?$AAp?$AAt?$AA?9?$AAp?$AAt?$AA?$AA@ 10018d54     libucrt:lcidtoname_downlevel.obj
 0002:00004d60       ??_C@_1O@EAKMAJDN@?$AAq?$AAu?$AAz?$AA?9?$AAb?$AAo?$AA?$AA@ 10018d60     libucrt:lcidtoname_downlevel.obj
 0002:00004d70       ??_C@_1O@BHHPIGDN@?$AAq?$AAu?$AAz?$AA?9?$AAe?$AAc?$AA?$AA@ 10018d70     libucrt:lcidtoname_downlevel.obj
 0002:00004d80       ??_C@_1O@GBAPEKMJ@?$AAq?$AAu?$AAz?$AA?9?$AAp?$AAe?$AA?$AA@ 10018d80     libucrt:lcidtoname_downlevel.obj
 0002:00004d90       ??_C@_1M@CLGLEFBO@?$AAr?$AAo?$AA?9?$AAr?$AAo?$AA?$AA@ 10018d90     libucrt:lcidtoname_downlevel.obj
 0002:00004d9c       ??_C@_1M@CEEDODME@?$AAr?$AAu?$AA?9?$AAr?$AAu?$AA?$AA@ 10018d9c     libucrt:lcidtoname_downlevel.obj
 0002:00004da8       ??_C@_1M@HPKKKMPP@?$AAs?$AAa?$AA?9?$AAi?$AAn?$AA?$AA@ 10018da8     libucrt:lcidtoname_downlevel.obj
 0002:00004db4       ??_C@_1M@BKMAIGOJ@?$AAs?$AAe?$AA?9?$AAf?$AAi?$AA?$AA@ 10018db4     libucrt:lcidtoname_downlevel.obj
 0002:00004dc0       ??_C@_1M@NDPIFLFI@?$AAs?$AAe?$AA?9?$AAn?$AAo?$AA?$AA@ 10018dc0     libucrt:lcidtoname_downlevel.obj
 0002:00004dcc       ??_C@_1M@DANKKHJ@?$AAs?$AAe?$AA?9?$AAs?$AAe?$AA?$AA@ 10018dcc     libucrt:lcidtoname_downlevel.obj
 0002:00004dd8       ??_C@_1M@PNBLONPJ@?$AAs?$AAk?$AA?9?$AAs?$AAk?$AA?$AA@ 10018dd8     libucrt:lcidtoname_downlevel.obj
 0002:00004de4       ??_C@_1M@LFMODOAL@?$AAs?$AAl?$AA?9?$AAs?$AAi?$AA?$AA@ 10018de4     libucrt:lcidtoname_downlevel.obj
 0002:00004df0       ??_C@_1O@DFKOMPG@?$AAs?$AAm?$AAa?$AA?9?$AAn?$AAo?$AA?$AA@ 10018df0     libucrt:lcidtoname_downlevel.obj
 0002:00004e00       ??_C@_1O@NDKPBNNH@?$AAs?$AAm?$AAa?$AA?9?$AAs?$AAe?$AA?$AA@ 10018e00     libucrt:lcidtoname_downlevel.obj
 0002:00004e10       ??_C@_1O@PLLKBHAB@?$AAs?$AAm?$AAj?$AA?9?$AAn?$AAo?$AA?$AA@ 10018e10     libucrt:lcidtoname_downlevel.obj
 0002:00004e20       ??_C@_1O@CLEPOGCA@?$AAs?$AAm?$AAj?$AA?9?$AAs?$AAe?$AA?$AA@ 10018e20     libucrt:lcidtoname_downlevel.obj
 0002:00004e30       ??_C@_1O@DLGJGKMK@?$AAs?$AAm?$AAn?$AA?9?$AAf?$AAi?$AA?$AA@ 10018e30     libucrt:lcidtoname_downlevel.obj
 0002:00004e40       ??_C@_1O@OJDJGAJC@?$AAs?$AAm?$AAs?$AA?9?$AAf?$AAi?$AA?$AA@ 10018e40     libucrt:lcidtoname_downlevel.obj
 0002:00004e50       ??_C@_1M@BOFOGHPB@?$AAs?$AAq?$AA?9?$AAa?$AAl?$AA?$AA@ 10018e50     libucrt:lcidtoname_downlevel.obj
 0002:00004e5c       ??_C@_1BG@LJBBIPGB@?$AAs?$AAr?$AA?9?$AAb?$AAa?$AA?9?$AAc?$AAy?$AAr?$AAl?$AA?$AA@ 10018e5c     libucrt:lcidtoname_downlevel.obj
 0002:00004e74       ??_C@_1BG@JLBENFOE@?$AAs?$AAr?$AA?9?$AAb?$AAa?$AA?9?$AAl?$AAa?$AAt?$AAn?$AA?$AA@ 10018e74     libucrt:lcidtoname_downlevel.obj
 0002:00004e8c       ??_C@_1BG@KODPNHE@?$AAs?$AAr?$AA?9?$AAs?$AAp?$AA?9?$AAc?$AAy?$AAr?$AAl?$AA?$AA@ 10018e8c     libucrt:lcidtoname_downlevel.obj
 0002:00004ea4       ??_C@_1BG@CIOGKHPB@?$AAs?$AAr?$AA?9?$AAs?$AAp?$AA?9?$AAl?$AAa?$AAt?$AAn?$AA?$AA@ 10018ea4     libucrt:lcidtoname_downlevel.obj
 0002:00004ebc       ??_C@_1M@NGFJLMAC@?$AAs?$AAv?$AA?9?$AAf?$AAi?$AA?$AA@ 10018ebc     libucrt:lcidtoname_downlevel.obj
 0002:00004ec8       ??_C@_1M@MPJEJAJC@?$AAs?$AAv?$AA?9?$AAs?$AAe?$AA?$AA@ 10018ec8     libucrt:lcidtoname_downlevel.obj
 0002:00004ed4       ??_C@_1M@MPNDHLFK@?$AAs?$AAw?$AA?9?$AAk?$AAe?$AA?$AA@ 10018ed4     libucrt:lcidtoname_downlevel.obj
 0002:00004ee0       ??_C@_1O@KOHBJJI@?$AAs?$AAy?$AAr?$AA?9?$AAs?$AAy?$AA?$AA@ 10018ee0     libucrt:lcidtoname_downlevel.obj
 0002:00004ef0       ??_C@_1M@LDCEFHA@?$AAt?$AAa?$AA?9?$AAi?$AAn?$AA?$AA@ 10018ef0     libucrt:lcidtoname_downlevel.obj
 0002:00004efc       ??_C@_1M@CNJOFAK@?$AAt?$AAe?$AA?9?$AAi?$AAn?$AA?$AA@ 10018efc     libucrt:lcidtoname_downlevel.obj
 0002:00004f08       ??_C@_1M@GNAECACD@?$AAt?$AAh?$AA?9?$AAt?$AAh?$AA?$AA@ 10018f08     libucrt:lcidtoname_downlevel.obj
 0002:00004f14       ??_C@_1M@CHBIHOJO@?$AAt?$AAn?$AA?9?$AAz?$AAa?$AA?$AA@ 10018f14     libucrt:lcidtoname_downlevel.obj
 0002:00004f20       ??_C@_1M@GCCMIGPJ@?$AAt?$AAr?$AA?9?$AAt?$AAr?$AA?$AA@ 10018f20     libucrt:lcidtoname_downlevel.obj
 0002:00004f2c       ??_C@_1M@CELMCNBK@?$AAt?$AAt?$AA?9?$AAr?$AAu?$AA?$AA@ 10018f2c     libucrt:lcidtoname_downlevel.obj
 0002:00004f38       ??_C@_1M@KLMCELGA@?$AAu?$AAk?$AA?9?$AAu?$AAa?$AA?$AA@ 10018f38     libucrt:lcidtoname_downlevel.obj
 0002:00004f44       ??_C@_1M@EPAJJAJF@?$AAu?$AAr?$AA?9?$AAp?$AAk?$AA?$AA@ 10018f44     libucrt:lcidtoname_downlevel.obj
 0002:00004f50       ??_C@_1BG@GEGPMCDJ@?$AAu?$AAz?$AA?9?$AAu?$AAz?$AA?9?$AAc?$AAy?$AAr?$AAl?$AA?$AA@ 10018f50     libucrt:lcidtoname_downlevel.obj
 0002:00004f68       ??_C@_1BG@EGGKJILM@?$AAu?$AAz?$AA?9?$AAu?$AAz?$AA?9?$AAl?$AAa?$AAt?$AAn?$AA?$AA@ 10018f68     libucrt:lcidtoname_downlevel.obj
 0002:00004f80       ??_C@_1M@GFOCLFF@?$AAv?$AAi?$AA?9?$AAv?$AAn?$AA?$AA@ 10018f80     libucrt:lcidtoname_downlevel.obj
 0002:00004f8c       ??_C@_1M@CPAMEDFI@?$AAx?$AAh?$AA?9?$AAz?$AAa?$AA?$AA@ 10018f8c     libucrt:lcidtoname_downlevel.obj
 0002:00004f98       ??_C@_1O@EBKIFIGN@?$AAz?$AAh?$AA?9?$AAc?$AAh?$AAs?$AA?$AA@ 10018f98     libucrt:lcidtoname_downlevel.obj
 0002:00004fa8       ??_C@_1O@NMHPGANE@?$AAz?$AAh?$AA?9?$AAc?$AAh?$AAt?$AA?$AA@ 10018fa8     libucrt:lcidtoname_downlevel.obj
 0002:00004fb8       ??_C@_1M@LPINJOMC@?$AAz?$AAh?$AA?9?$AAc?$AAn?$AA?$AA@ 10018fb8     libucrt:lcidtoname_downlevel.obj
 0002:00004fc4       ??_C@_1M@OCJEJODD@?$AAz?$AAh?$AA?9?$AAh?$AAk?$AA?$AA@ 10018fc4     libucrt:lcidtoname_downlevel.obj
 0002:00004fd0       ??_C@_1M@DNDLJINH@?$AAz?$AAh?$AA?9?$AAm?$AAo?$AA?$AA@ 10018fd0     libucrt:lcidtoname_downlevel.obj
 0002:00004fdc       ??_C@_1M@MBFDNDND@?$AAz?$AAh?$AA?9?$AAs?$AAg?$AA?$AA@ 10018fdc     libucrt:lcidtoname_downlevel.obj
 0002:00004fe8       ??_C@_1M@IMEPLEPE@?$AAz?$AAh?$AA?9?$AAt?$AAw?$AA?$AA@ 10018fe8     libucrt:lcidtoname_downlevel.obj
 0002:00004ff4       ??_C@_1M@BBGHNHJP@?$AAz?$AAu?$AA?9?$AAz?$AAa?$AA?$AA@ 10018ff4     libucrt:lcidtoname_downlevel.obj
 0002:00005160       __infinity                 10019160     libucrt:87tran.obj
 0002:0000516a       __minfinity                1001916a     libucrt:87tran.obj
 0002:00005174       __logemax                  10019174     libucrt:87tran.obj
 0002:0000519a       __OP_EXPjmptab             1001919a     libucrt:87tran.obj
 0002:000051c0       __indefinite               100191c0     libucrt:87disp.obj
 0002:000051ca       __piby2                    100191ca     libucrt:87disp.obj
 0002:000051d4       __piby4                    100191d4     libucrt:87disp.obj
 0002:00005208       __DEFAULT_CW_in_mem        10019208     libucrt:common.obj
 0002:0000520a       __pi_by_2_to_61            1001920a     libucrt:common.obj
 0002:00005244       ??_C@_03MGHMBJCF@log?$AA@  10019244     libucrt:libm_error.obj
 0002:00005248       ??_C@_05HGHHAHAP@log10?$AA@ 10019248     libucrt:libm_error.obj
 0002:00005250       ??_C@_03KHJOGHMM@exp?$AA@  10019250     libucrt:libm_error.obj
 0002:00005254       ??_C@_03JGHBODFD@pow?$AA@  10019254     libucrt:libm_error.obj
 0002:00005258       ??_C@_04FIHNOPOL@asin?$AA@ 10019258     libucrt:libm_error.obj
 0002:00005260       ??_C@_04PDIFKINK@acos?$AA@ 10019260     libucrt:libm_error.obj
 0002:00005268       ??_C@_04EIAKFFMI@sqrt?$AA@ 10019268     libucrt:libm_error.obj
 0002:00005270       __real@3ff0000000000000    10019270     libucrt:libm_error.obj
 0002:00005290       ___acrt_log10_table_t      10019290     libucrt:log10_tables.obj
 0002:000056a0       ___acrt_log10_table_cb     100196a0     libucrt:log10_tables.obj
 0002:00005ab0       __real@3fe0000000000000    10019ab0     libucrt:powhlp.obj
 0002:00005ab8       ??_C@_04FJHINJAO@tanh?$AA@ 10019ab8     libucrt:fpexcept.obj
 0002:00005ac0       ??_C@_04MLLJIGOK@atan?$AA@ 10019ac0     libucrt:fpexcept.obj
 0002:00005ac8       ??_C@_05KNGEOGJB@atan2?$AA@ 10019ac8     libucrt:fpexcept.obj
 0002:00005ad0       ??_C@_03BLEJJJBH@sin?$AA@  10019ad0     libucrt:fpexcept.obj
 0002:00005ad4       ??_C@_03LALBNOCG@cos?$AA@  10019ad4     libucrt:fpexcept.obj
 0002:00005ad8       ??_C@_03IIINPABG@tan?$AA@  10019ad8     libucrt:fpexcept.obj
 0002:00005adc       ??_C@_04GFPJNGEK@ceil?$AA@ 10019adc     libucrt:fpexcept.obj
 0002:00005ae4       ??_C@_05PBJFFIGL@floor?$AA@ 10019ae4     libucrt:fpexcept.obj
 0002:00005aec       ??_C@_04ODHECPBC@fabs?$AA@ 10019aec     libucrt:fpexcept.obj
 0002:00005af4       ??_C@_04EHEDPDJG@modf?$AA@ 10019af4     libucrt:fpexcept.obj
 0002:00005afc       ??_C@_05CEJMAHNP@ldexp?$AA@ 10019afc     libucrt:fpexcept.obj
 0002:00005b04       ??_C@_05KBKMEMPO@_cabs?$AA@ 10019b04     libucrt:fpexcept.obj
 0002:00005b0c       ??_C@_06MEIMCGCF@_hypot?$AA@ 10019b0c     libucrt:fpexcept.obj
 0002:00005b14       ??_C@_04KEPJIHGP@fmod?$AA@ 10019b14     libucrt:fpexcept.obj
 0002:00005b1c       ??_C@_05GKKHEGJL@frexp?$AA@ 10019b1c     libucrt:fpexcept.obj
 0002:00005b24       ??_C@_03MJLDFKDL@_y0?$AA@  10019b24     libucrt:fpexcept.obj
 0002:00005b28       ??_C@_03NAKIGLHK@_y1?$AA@  10019b28     libucrt:fpexcept.obj
 0002:00005b2c       ??_C@_03ONILCKOB@_yn?$AA@  10019b2c     libucrt:fpexcept.obj
 0002:00005b30       ??_C@_05JGDBENOH@_logb?$AA@ 10019b30     libucrt:fpexcept.obj
 0002:00005b38       ??_C@_0L@KDOEJCKC@_nextafter?$AA@ 10019b38     libucrt:fpexcept.obj
 0002:00005c30       ??_C@_04COOMCNPB@sinh?$AA@ 10019c30     libucrt:fpexcept.obj
 0002:00005c38       ??_C@_04HPJJNFIM@cosh?$AA@ 10019c38     libucrt:fpexcept.obj
 0002:00005c40       __d_inf                    10019c40     libucrt:util.obj
 0002:00005c48       __d_max                    10019c48     libucrt:util.obj
 0002:00005c50       __d_mzero                  10019c50     libucrt:util.obj
 0002:00005c58       ??_C@_1BA@BALFACEM@?$AAC?$AAO?$AAN?$AAO?$AAU?$AAT?$AA$?$AA?$AA@ 10019c58     libucrt:initcon.obj
 0002:00005cc8       __load_config_used         10019cc8     LIBCMT:loadcfg.obj
 0002:00005d70       ___safe_se_handler_table   10019d70     <linker-defined>
 0002:00006054       ___rtc_iaa                 1001a054     LIBCMT:_initsect_.obj
 0002:00006058       ___rtc_izz                 1001a058     LIBCMT:_initsect_.obj
 0002:0000605c       ___rtc_taa                 1001a05c     LIBCMT:_initsect_.obj
 0002:00006060       ___rtc_tzz                 1001a060     LIBCMT:_initsect_.obj
 0002:0000658c       __IMPORT_DESCRIPTOR_VERSION 1001a58c     version:VERSION.dll
 0002:000065a0       __IMPORT_DESCRIPTOR_KERNEL32 1001a5a0     kernel32:KERNEL32.dll
 0002:000065b4       __IMPORT_DESCRIPTOR_USER32 1001a5b4     user32:USER32.dll
 0002:000065c8       __IMPORT_DESCRIPTOR_GDI32  1001a5c8     gdi32:GDI32.dll
 0002:000065dc       __IMPORT_DESCRIPTOR_ADVAPI32 1001a5dc     advapi32:ADVAPI32.dll
 0002:000065f0       __NULL_IMPORT_DESCRIPTOR   1001a5f0     version:VERSION.dll
 0003:00000000       ?gbLinesColorPanel@@3HA    1001b000     ConEmuLn.obj
 0003:00000004       ?gcrLinesColorPanel@@3KA   1001b004     ConEmuLn.obj
 0003:00000008       ?gcrLinesColorEditor@@3KA  1001b008     ConEmuLn.obj
 0003:0000000c       ?gcrLinesColorViewer@@3KA  1001b00c     ConEmuLn.obj
 0003:00000010       ?gcrHilightPlugBack@@3KA   1001b010     ConEmuLn.obj
 0003:00000014       ?Far3Func@@3PAUExportFunc@@A 1001b014     ConEmuLn.obj
 0003:00000038       ?gSettings@@3PAUConEmuLnSettings@@A 1001b038     ConEmuLn.obj
 0003:000000e8       ?guid_ConEmuLn@@3U_GUID@@A 1001b0e8     ConEmuLn2800.obj
 0003:000000f8       ?guid_ConEmuLnCfgDlg@@3U_GUID@@A 1001b0f8     ConEmuLn2800.obj
 0003:00000108       ?guid_ConEmuLnPluginMenu@@3U_GUID@@A 1001b108     ConEmuLn2800.obj
 0003:00000118       ?guid_ConEmuLnPluginConfig@@3U_GUID@@A 1001b118     ConEmuLn2800.obj
 0003:00000128       ___security_cookie         1001b128     LIBCMT:gs_cookie.obj
 0003:0000012c       ___security_cookie_complement 1001b12c     LIBCMT:gs_cookie.obj
 0003:00000130       ___scrt_native_dllmain_reason 1001b130     LIBCMT:utility.obj
 0003:00000140       ___isa_enabled             1001b140     LIBCMT:_cpu_disp_.obj
 0003:00000160       __NLG_Destination          1001b160     libvcruntime:_exsup_.obj
 0003:00000170       ___abort_behavior          1001b170     libucrt:abort.obj
 0003:0000017c       __pwctype                  1001b17c     libucrt:ctype.obj
 0003:00000188       ___acrt_initial_locale_data 1001b188     libucrt:nlsdata.obj
 0003:00000240       ___acrt_initial_locale_pointers 1001b240     libucrt:nlsdata.obj
 0003:00000248       ___acrt_wide_c_locale_string 1001b248     libucrt:nlsdata.obj
 0003:00000250       __iob                      1001b250     libucrt:_file.obj
 0003:000003f0       __mbctype                  1001b3f0     libucrt:mbctype.obj
 0003:000004f8       __mbcasemap                1001b4f8     libucrt:mbctype.obj
 0003:000005f8       ___acrt_initial_multibyte_data 1001b5f8     libucrt:mbctype.obj
 0003:00000818       ___acrt_current_multibyte_data 1001b818     libucrt:mbctype.obj
 0003:0000081c       ___globallocalestatus      1001b81c     libucrt:glstatus.obj
 0003:00000820       ___acrt_lconv_static_decimal 1001b820     libucrt:localeconv.obj
 0003:00000824       ___acrt_lconv_static_W_decimal 1001b824     libucrt:localeconv.obj
 0003:00000828       ___acrt_lconv_c            1001b828     libucrt:localeconv.obj
 0003:00000880       ___dcrt_lowio_console_output_handle 1001b880     libucrt:initcon.obj
 0003:00000890       __fltused                  1001b890     LIBCMT:fltused.obj
 0003:000008a0       ?ghPluginModule@@3PAUHINSTANCE__@@A 1001b8a0     ConEmuLn.obj
 0003:000008a4       ?gFarVersion@@3UFarVersion@@A 1001b8a4     ConEmuLn.obj
 0003:000008b0       ?gbBackgroundEnabled@@3HA  1001b8b0     ConEmuLn.obj
 0003:000008b4       ?gbLinesColorEditor@@3HA   1001b8b4     ConEmuLn.obj
 0003:000008b8       ?gbLinesColorViewer@@3HA   1001b8b8     ConEmuLn.obj
 0003:000008bc       ?giHilightType@@3HA        1001b8bc     ConEmuLn.obj
 0003:000008c0       ?gbHilightPlugins@@3HA     1001b8c0     ConEmuLn.obj
 0003:000008c4       ?gbInStartPlugin@@3_NA     1001b8c4     ConEmuLn.obj
 0003:000008c5       ?gbSetStartupInfoOk@@3_NA  1001b8c5     ConEmuLn.obj
 0003:000008c8       ?gbInfoW_OK@@3HA           1001b8c8     ConEmuLn.obj
 0003:000008d4       ?InfoW1900@@3PAUPluginStartupInfo@@A 1001b8d4     ConEmuLn1900.obj
 0003:000008d8       ?FSFW1900@@3PAUFarStandardFunctions@@A 1001b8d8     ConEmuLn1900.obj
 0003:00000ae0       ?InfoW2800@@3PAUPluginStartupInfo@@A 1001bae0     ConEmuLn2800.obj
 0003:00000ae4       ?FSFW2800@@3PAUFarStandardFunctions@@A 1001bae4     ConEmuLn2800.obj
 0003:00000cf0       ?InfoW995@@3PAUPluginStartupInfo@@A 1001bcf0     ConEmuLn995.obj
 0003:00000cf4       ?FSFW995@@3PAUFarStandardFunctions@@A 1001bcf4     ConEmuLn995.obj
 0003:00000f00       ?InfoA@@3PAUPluginStartupInfo@@A 1001bf00     ConEmuLnA.obj
 0003:00000f04       ?FSFA@@3PAUFarStandardFunctions@@A 1001bf04     ConEmuLnA.obj
 0003:00001010       ?_OptionsStorage@?1??__local_stdio_printf_options@@9@4_KA 1001c010     common-kernel32:MStrSafe.obj
 0003:00001018       ?ghHeap@@3PAXA             1001c018     common-kernel32:Memory.obj
 0003:0000101c       ?g_LastDeletePtr@@3PAXA    1001c01c     common-kernel32:Memory.obj
 0003:00001348       ?__type_info_root_node@@3U__type_info_node@@A 1001c348     LIBCMT:tncleanup.obj
 0003:00001350       ?_OptionsStorage@?1??__local_stdio_scanf_options@@9@4_KA 1001c350     LIBCMT:default_local_stdio_options.obj
 0003:00001374       ___scrt_current_native_startup_state 1001c374     LIBCMT:utility.obj
 0003:00001378       ___scrt_native_startup_lock 1001c378     LIBCMT:utility.obj
 0003:00001380       ___scrt_debugger_hook_flag 1001c380     LIBCMT:utility_desktop.obj
 0003:00001384       ___isa_available           1001c384     LIBCMT:_cpu_disp_.obj
 0003:00001388       ___favor                   1001c388     LIBCMT:_cpu_disp_.obj
 0003:0000138c       ?pArgList@UnDecorator@@0PAVReplicator@@A 1001c38c     libvcruntime:undname.obj
 0003:00001390       ?pZNameList@UnDecorator@@0PAVReplicator@@A 1001c390     libvcruntime:undname.obj
 0003:00001394       ?pTemplateArgList@UnDecorator@@0PAVReplicator@@A 1001c394     libvcruntime:undname.obj
 0003:00001398       ?gName@UnDecorator@@0PBDB  1001c398     libvcruntime:undname.obj
 0003:0000139c       ?name@UnDecorator@@0PBDB   1001c39c     libvcruntime:undname.obj
 0003:000013a0       ?disableFlags@UnDecorator@@0KA 1001c3a0     libvcruntime:undname.obj
 0003:000013a4       ?fExplicitTemplateParams@UnDecorator@@0_NA 1001c3a4     libvcruntime:undname.obj
 0003:000013a5       ?fGetTemplateArgumentList@UnDecorator@@0_NA 1001c3a5     libvcruntime:undname.obj
 0003:000013a8       ?m_pGetParameter@UnDecorator@@0P6APADJ@ZA 1001c3a8     libvcruntime:undname.obj
 0003:000013ac       ?m_CHPENameOffset@UnDecorator@@0KA 1001c3ac     libvcruntime:undname.obj
 0003:000013b0       ?m_recursionLevel@UnDecorator@@0KA 1001c3b0     libvcruntime:undname.obj
 0003:0000142c       ___pPurecall               1001c42c     libvcruntime:purevirt_data.obj
 0003:00001430       ?__WinRTOutOfMemoryExceptionCallback@@3P6GPAXXZA 1001c430     libvcruntime:ehhelpers.obj
 0003:00001548       __environ_table            1001c548     libucrt:environment_initialization.obj
 0003:0000154c       __wenviron_table           1001c54c     libucrt:environment_initialization.obj
 0003:00001550       ___dcrt_initial_wide_environment 1001c550     libucrt:environment_initialization.obj
 0003:00001554       ___dcrt_initial_narrow_environment 1001c554     libucrt:environment_initialization.obj
 0003:00001558       ___acrt_atexit_table       1001c558     libucrt:onexit.obj
 0003:00001564       ___acrt_at_quick_exit_table 1001c564     libucrt:onexit.obj
 0003:00001574       ___acrt_locale_changed_data 1001c574     libucrt:wsetlocale.obj
 0003:00001578       ___acrt_current_locale_data 1001c578     libucrt:nlsdata.obj
 0003:0000157c       __nstream                  1001c57c     libucrt:_file.obj
 0003:00001580       ___piob                    1001c580     libucrt:_file.obj
 0003:00001588       ___acrt_stdout_buffer      1001c588     libucrt:_sftbuf.obj
 0003:0000158c       ___acrt_stderr_buffer      1001c58c     libucrt:_sftbuf.obj
 0003:00001590       ___pioinfo                 1001c590     libucrt:ioinit.obj
 0003:00001790       __nhandle                  1001c790     libucrt:ioinit.obj
 0003:000019ac       ___mblocalename            1001c9ac     libucrt:mbctype.obj
 0003:000019b0       ___mbcodepage              1001c9b0     libucrt:mbctype.obj
 0003:000019b4       ___ismbcodepage            1001c9b4     libucrt:mbctype.obj
 0003:000019b8       ___mbulinfo                1001c9b8     libucrt:mbctype.obj
 0003:000019cc       ___argc                    1001c9cc     libucrt:argv_data.obj
 0003:000019d0       ___argv                    1001c9d0     libucrt:argv_data.obj
 0003:000019d4       ___wargv                   1001c9d4     libucrt:argv_data.obj
 0003:000019d8       __acmdln                   1001c9d8     libucrt:argv_data.obj
 0003:000019dc       __wcmdln                   1001c9dc     libucrt:argv_data.obj
 0003:000019e0       __pgmptr                   1001c9e0     libucrt:argv_data.obj
 0003:000019e4       ___acrt_heap               1001c9e4     libucrt:heap_handle.obj
 0003:00001a00       ___acrt_lconv_static_null  1001ca00     libucrt:localeconv.obj
 0003:00001a04       ___acrt_lconv_static_W_null 1001ca04     libucrt:localeconv.obj
 0003:00001a10       ___fastflag                1001ca10     libucrt:fp_flags.obj
 0003:00001a18       ___scrt_ucrt_dll_is_in_use 1001ca18     <common>
 0003:00001a1c       ___dyn_tls_init_callback   1001ca1c     <common>
 0003:00001a20       __pmatherr                 1001ca20     <common>
 0003:00001a24       ___use_sse2_mathfcns       1001ca24     <common>

 entry point at        0001:00004159

 Static symbols

 0000:fffe0000       .debug$S                   10000000     kernel32:KERNEL32.dll
 0000:fffe0000       .debug$S                   10000000     advapi32:ADVAPI32.dll
 0000:fffe0000       .debug$S                   10000000     kernel32:KERNEL32.dll
 0000:fffe0000       .debug$S                   10000000     kernel32:KERNEL32.dll
 0000:fffe0000       .debug$S                   10000000     kernel32:KERNEL32.dll
 0000:fffe0000       .debug$S                   10000000     kernel32:KERNEL32.dll
 0000:fffe0000       .debug$S                   10000000     kernel32:KERNEL32.dll
 0000:fffe0000       .debug$S                   10000000     advapi32:ADVAPI32.dll
 0000:fffe0000       .debug$S                   10000000     advapi32:ADVAPI32.dll
 0000:fffe0000       .debug$S                   10000000     advapi32:ADVAPI32.dll
 0000:fffe0000       .debug$S                   10000000     advapi32:ADVAPI32.dll
 0000:fffe0000       .debug$S                   10000000     gdi32:GDI32.dll
 0000:fffe0000       .debug$S                   10000000     gdi32:GDI32.dll
 0000:fffe0000       .debug$S                   10000000     gdi32:GDI32.dll
 0000:fffe0000       .debug$S                   10000000     gdi32:GDI32.dll
 0000:fffe0000       .debug$S                   10000000     version:VERSION.dll
 0000:fffe0000       .debug$S                   10000000     version:VERSION.dll
 0000:fffe0000       .debug$S                   10000000     version:VERSION.dll
 0000:fffe0000       .debug$S                   10000000     kernel32:KERNEL32.dll
 0000:fffe0000       .debug$S                   10000000     kernel32:KERNEL32.dll
 0000:fffe0000       .debug$S                   10000000     kernel32:KERNEL32.dll
 0000:fffe0000       .debug$S                   10000000     ConEmuLn.exp
 0000:fffe0000       .debug$S                   10000000     kernel32:KERNEL32.dll
 0000:fffe0000       .debug$S                   10000000     kernel32:KERNEL32.dll
 0000:fffe0000       .debug$S                   10000000     kernel32:KERNEL32.dll
 0000:fffe0000       .debug$S                   10000000     kernel32:KERNEL32.dll
 0000:fffe0000       .debug$S                   10000000     kernel32:KERNEL32.dll
 0000:fffe0000       .debug$S                   10000000     kernel32:KERNEL32.dll
 0000:fffe0000       .debug$S                   10000000     kernel32:KERNEL32.dll
 0000:fffe0000       .debug$S                   10000000     user32:USER32.dll
 0000:fffe0000       .debug$S                   10000000     user32:USER32.dll
 0000:fffe0000       .debug$S                   10000000     user32:USER32.dll
 0000:fffe0000       .debug$S                   10000000     gdi32:GDI32.dll
 0000:fffe0000       .debug$S                   10000000     gdi32:GDI32.dll
 0000:fffe0000       .debug$S                   10000000     kernel32:KERNEL32.dll
 0000:fffe0000       .debug$S                   10000000     kernel32:KERNEL32.dll
 0000:fffe0000       .debug$S                   10000000     kernel32:KERNEL32.dll
 0000:fffe0000       .debug$S                   10000000     kernel32:KERNEL32.dll
 0000:fffe0000       .debug$S                   10000000     kernel32:KERNEL32.dll
 0000:fffe0000       .debug$S                   10000000     kernel32:KERNEL32.dll
 0000:fffe0000       .debug$S                   10000000     kernel32:KERNEL32.dll
 0000:fffe0000       .debug$S                   10000000     kernel32:KERNEL32.dll
 0000:fffe0000       .debug$S                   10000000     kernel32:KERNEL32.dll
 0000:fffe0000       .debug$S                   10000000     kernel32:KERNEL32.dll
 0000:fffe0000       .debug$S                   10000000     kernel32:KERNEL32.dll
 0000:fffe0000       .debug$S                   10000000     kernel32:KERNEL32.dll
 0000:fffe0000       .debug$S                   10000000     kernel32:KERNEL32.dll
 0000:fffe0000       .debug$S                   10000000     kernel32:KERNEL32.dll
 0000:fffe0000       .debug$S                   10000000     kernel32:KERNEL32.dll
 0000:fffe0000       .debug$S                   10000000     kernel32:KERNEL32.dll
 0000:fffe0000       .debug$S                   10000000     kernel32:KERNEL32.dll
 0000:fffe0000       .debug$S                   10000000     kernel32:KERNEL32.dll
 0000:fffe0000       .debug$S                   10000000     kernel32:KERNEL32.dll
 0000:fffe0000       .debug$S                   10000000     kernel32:KERNEL32.dll
 0000:fffe0000       .debug$S                   10000000     kernel32:KERNEL32.dll
 0000:fffe0000       .debug$S                   10000000     kernel32:KERNEL32.dll
 0000:fffe0000       .debug$S                   10000000     kernel32:KERNEL32.dll
 0000:fffe0000       .debug$S                   10000000     kernel32:KERNEL32.dll
 0000:fffe0000       .debug$S                   10000000     kernel32:KERNEL32.dll
 0000:fffe0000       .debug$S                   10000000     kernel32:KERNEL32.dll
 0000:fffe0000       .debug$S                   10000000     kernel32:KERNEL32.dll
 0000:fffe0000       .debug$S                   10000000     kernel32:KERNEL32.dll
 0000:fffe0000       .debug$S                   10000000     kernel32:KERNEL32.dll
 0000:fffe0000       .debug$S                   10000000     kernel32:KERNEL32.dll
 0000:fffe0000       .debug$S                   10000000     kernel32:KERNEL32.dll
 0000:fffe0000       .debug$S                   10000000     kernel32:KERNEL32.dll
 0000:fffe0000       .debug$S                   10000000     kernel32:KERNEL32.dll
 0000:fffe0000       .debug$S                   10000000     kernel32:KERNEL32.dll
 0000:fffe0000       .debug$S                   10000000     kernel32:KERNEL32.dll
 0000:fffe0000       .debug$S                   10000000     kernel32:KERNEL32.dll
 0000:fffe0000       .debug$S                   10000000     kernel32:KERNEL32.dll
 0000:fffe0000       .debug$S                   10000000     kernel32:KERNEL32.dll
 0000:fffe0000       .debug$S                   10000000     kernel32:KERNEL32.dll
 0000:fffe0000       .debug$S                   10000000     kernel32:KERNEL32.dll
 0000:fffe0000       .debug$S                   10000000     kernel32:KERNEL32.dll
 0000:fffe0000       .debug$S                   10000000     kernel32:KERNEL32.dll
 0000:fffe0000       .debug$S                   10000000     kernel32:KERNEL32.dll
 0000:fffe0000       .debug$S                   10000000     kernel32:KERNEL32.dll
 0000:fffe0000       .debug$S                   10000000     kernel32:KERNEL32.dll
 0000:fffe0000       .debug$S                   10000000     kernel32:KERNEL32.dll
 0000:fffe0000       .debug$S                   10000000     kernel32:KERNEL32.dll
 0000:fffe0000       .debug$S                   10000000     kernel32:KERNEL32.dll
 0000:fffe0000       .debug$S                   10000000     kernel32:KERNEL32.dll
 0000:fffe0000       .debug$S                   10000000     kernel32:KERNEL32.dll
 0000:fffe0000       .debug$S                   10000000     kernel32:KERNEL32.dll
 0000:fffe0000       .debug$S                   10000000     kernel32:KERNEL32.dll
 0000:fffe0000       .debug$S                   10000000     kernel32:KERNEL32.dll
 0000:fffe0000       .debug$S                   10000000     kernel32:KERNEL32.dll
 0000:fffe0000       .debug$S                   10000000     kernel32:KERNEL32.dll
 0000:fffe0000       .debug$S                   10000000     kernel32:KERNEL32.dll
 0000:fffe0000       .debug$S                   10000000     kernel32:KERNEL32.dll
 0000:fffe0000       .debug$S                   10000000     kernel32:KERNEL32.dll
 0000:fffe0000       .debug$S                   10000000     kernel32:KERNEL32.dll
 0000:fffe0000       .debug$S                   10000000     kernel32:KERNEL32.dll
 0000:fffe0000       .debug$S                   10000000     kernel32:KERNEL32.dll
 0000:fffe0000       .debug$S                   10000000     kernel32:KERNEL32.dll
 0000:fffe0000       .debug$S                   10000000     kernel32:KERNEL32.dll
 0000:fffe0000       .debug$S                   10000000     kernel32:KERNEL32.dll
 0000:fffe0000       .debug$S                   10000000     kernel32:KERNEL32.dll
 0000:fffe0000       .debug$S                   10000000     kernel32:KERNEL32.dll
 0000:fffe0000       .debug$S                   10000000     kernel32:KERNEL32.dll
 0000:fffe0000       .debug$S                   10000000     kernel32:KERNEL32.dll
 0000:fffe0000       .debug$S                   10000000     kernel32:KERNEL32.dll
 0000:fffe0000       .debug$S                   10000000     kernel32:KERNEL32.dll
 0000:fffe0000       .debug$S                   10000000     kernel32:KERNEL32.dll
 0000:fffe0000       .debug$S                   10000000     kernel32:KERNEL32.dll
 0000:fffe0000       .debug$S                   10000000     kernel32:KERNEL32.dll
 0000:fffe0000       .debug$S                   10000000     kernel32:KERNEL32.dll
 0000:fffe0000       .debug$S                   10000000     kernel32:KERNEL32.dll
 0000:fffe0000       .debug$S                   10000000     kernel32:KERNEL32.dll
 0000:fffe0000       .debug$S                   10000000     kernel32:KERNEL32.dll
 0000:fffe0000       .debug$S                   10000000     kernel32:KERNEL32.dll
 0000:fffe0000       .debug$S                   10000000     kernel32:KERNEL32.dll
 0000:fffe0000       .debug$S                   10000000     kernel32:KERNEL32.dll
 0001:000000da       ?ChangeExports@@YA_NPBUExportFunc@@PAUHINSTANCE__@@@Z 100010da f   ConEmuLn.obj
 0001:0000031e       ?LoadFarVersion@@YA_NAAUFarVersion@@AAY0CAA@_W@Z 1000131e f   ConEmuLn.obj
 0001:000003ae       ?LoadFarVersion@@YA_NPB_WAAUFarVersion@@AAY0CAA@_W@Z 100013ae f   ConEmuLn.obj
 0001:00000432       ?LoadModuleVersion@@YA_NPB_WAAUtagVS_FIXEDFILEINFO@@PA_WI@Z 10001432 f   ConEmuLn.obj
 0001:00000da0       ?StringCopyWorkerW@@YGJPA_WIPAIPB_WI@Z 10001da0 f   ConEmuLn.obj
 0001:00000e05       ?StringLengthWorkerW@@YGJPB_WIPAI@Z 10001e05 f   ConEmuLn.obj
 0001:00000e4c       ?StringValidateDestAndLengthW@@YGJPB_WIPAII@Z 10001e4c f   ConEmuLn.obj
 0001:00000f3a       ?ConfigDlgProc@@YGHPAXHH0@Z 10001f3a f   ConEmuLn1900.obj
 0001:0000105f       ?ConfigureProc@@YAHH@Z     1000205f f   ConEmuLn1900.obj
 0001:00001b12       ?ConfigDlgProc@@YGHPAXHH0@Z 10002b12 f   ConEmuLn2800.obj
 0001:00001c37       ?ConfigureProc@@YAHH@Z     10002c37 f   ConEmuLn2800.obj
 0001:00002767       ?ConfigDlgProc@@YGJPAXHHJ@Z 10003767 f   ConEmuLn995.obj
 0001:0000288c       ?ConfigureProc@@YAHH@Z     1000388c f   ConEmuLn995.obj
 0001:00003195       ?ConfigDlgProc@@YGJPAXHHJ@Z 10004195 f   ConEmuLnA.obj
 0001:000032be       ?ConfigureProc@@YAHH@Z     100042be f   ConEmuLnA.obj
 0001:00003e20       $$000000                   10004e20     LIBCMT:chkstk.obj
 0001:00003e4d       ?dllmain_crt_dispatch@@YGHQAUHINSTANCE__@@KQAX@Z 10004e4d f   LIBCMT:dll_dllmain.obj
 0001:00003ea0       ?dllmain_crt_process_attach@@YAHQAUHINSTANCE__@@QAX@Z 10004ea0 f   LIBCMT:dll_dllmain.obj
 0001:00003f9d       ?dllmain_crt_process_detach@@YAH_N@Z 10004f9d f   LIBCMT:dll_dllmain.obj
 0001:00004023       ?dllmain_dispatch@@YAHQAUHINSTANCE__@@KQAX@Z 10005023 f   LIBCMT:dll_dllmain.obj
 0001:0000429f       ___get_entropy             1000529f f   LIBCMT:gs_support.obj
 0001:00004374       ?find_pe_section@@YAPAU_IMAGE_SECTION_HEADER@@QAEI@Z 10005374 f   LIBCMT:utility.obj
 0001:000047f0       $$000000                   100057f0     LIBCMT:_sehprolg4_.obj
 0001:00004a00       $$000000                   10005a00     libvcruntime:memmove.obj
 0001:00004c64       TrailingUpVec              10005c64     libvcruntime:memmove.obj
 0001:00004d10       TrailingDownVec            10005d10     libvcruntime:memmove.obj
 0001:00004f80       $$000000                   10005f80     libvcruntime:memset.obj
 0001:000050e0       _ValidateLocalCookies      100060e0 f   libvcruntime:_chandler4_.obj
 0001:00005300       $$000000                   10006300     libvcruntime:_exsup4_.obj
 0001:00005390       __unwind_handler4          10006390 f   libvcruntime:_exsup4_.obj
 0001:0000569c       ?try_get_first_available_module@@YAPAUHINSTANCE__@@QBW4module_id@?A0x9a4b7766@@0@Z 1000669c f   libvcruntime:winapi_downlevel.obj
 0001:00005762       ?try_get_function@@YAPAXW4function_id@?A0x9a4b7766@@QBDQBW4module_id@2@2@Z 10006762 f   libvcruntime:winapi_downlevel.obj
 0001:00005970       $$000000                   10006970     libvcruntime:_exsup_.obj
 0001:00005991       __unwind_handler           10006991 f   libvcruntime:_exsup_.obj
 0001:00005ab0       $$000000                   10006ab0     libvcruntime:memcpy.obj
 0001:00005d14       TrailingUpVec              10006d14     libvcruntime:memcpy.obj
 0001:00005dc0       TrailingDownVec            10006dc0     libvcruntime:memcpy.obj
 0001:00006030       $$000000                   10007030     libvcruntime:lowhelpr.obj
 0001:00006c4d       ??$common_vsprintf@Vstandard_base@__crt_stdio_output@@_W@@YAH_KQA_WIQB_WQAU__crt_locale_pointers@@QAD@Z 10007c4d f   libucrt:output.obj
 0001:0000734b       $LN54                      1000834b     libucrt:output.obj
 0001:0000783c       $LN19                      1000883c     libucrt:output.obj
 0001:0000817e       ?atexit_exception_filter@@YAHK@Z 1000917e f   libucrt:exit.obj
 0001:00008191       ?common_exit@@YAXHW4_crt_exit_cleanup_mode@@W4_crt_exit_return_mode@@@Z 10009191 f   libucrt:exit.obj
 0001:000082aa       ?exit_or_terminate_process@@YAXI@Z 100092aa f   libucrt:exit.obj
 0001:000082eb       ?is_managed_app@@YA_NXZ    100092eb f   libucrt:exit.obj
 0001:0000832f       ?try_cor_exit_process@@YAXI@Z 1000932f f   libucrt:exit.obj
 0001:000083d3       ??$common_configure_argv@D@@YAHW4_crt_argv_mode@@@Z 100093d3 f   libucrt:argv_parsing.obj
 0001:000084f7       ??$parse_command_line@D@@YAXPADPAPAD0PAI2@Z 100094f7 f   libucrt:argv_parsing.obj
 0001:000086cc       ??$common_initialize_environment_nolock@D@@YAHXZ 100096cc f   libucrt:environment_initialization.obj
 0001:00008725       ??$create_environment@D@@YAQAPADQAD@Z 10009725 f   libucrt:environment_initialization.obj
 0001:000087f6       ??$free_environment@_W@@YAXQAPA_W@Z 100097f6 f   libucrt:environment_initialization.obj
 0001:000087f6       ??$free_environment@D@@YAXQAPAD@Z 100097f6 f   libucrt:environment_initialization.obj
 0001:00008865       ??$uninitialize_environment_internal@D@@YAXAAPAPAD@Z 10009865 f   libucrt:environment_initialization.obj
 0001:00008880       ??$uninitialize_environment_internal@_W@@YAXAAPAPA_W@Z 10009880 f   libucrt:environment_initialization.obj
 0001:00008981       ??R<lambda_275893d493268fdec8709772e3fcec0e>@@QBEHXZ 10009981 f   libucrt:onexit.obj
 0001:00008afb       _initialize_global_variables 10009afb f   libucrt:initialization.obj
 0001:00008b0d       _initialize_c              10009b0d f   libucrt:initialization.obj
 0001:00008b27       _uninitialize_c            10009b27 f   libucrt:initialization.obj
 0001:00008b27       _initialize_environment    10009b27 f   libucrt:initialization.obj
 0001:00008b27       _uninitialize_global_state_isolation 10009b27 f   libucrt:initialization.obj
 0001:00008b27       _initialize_global_state_isolation 10009b27 f   libucrt:initialization.obj
 0001:00008b27       _report_memory_leaks       10009b27 f   libucrt:initialization.obj
 0001:00008b2a       _uninitialize_environment  10009b2a f   libucrt:initialization.obj
 0001:00008b32       _initialize_pointers       10009b32 f   libucrt:initialization.obj
 0001:00008b6f       _uninitialize_vcruntime    10009b6f f   libucrt:initialization.obj
 0001:00008b78       _uninitialize_allocated_memory 10009b78 f   libucrt:initialization.obj
 0001:00008ce0       $$000000                   10009ce0     libucrt:strncmp.obj
 0001:0000937a       ?construct_ptd@@YAXQAU__acrt_ptd@@QAPAU__crt_locale_data@@@Z 1000a37a f   libucrt:per_thread_data.obj
 0001:000093f3       ?destroy_fls@@YGXPAX@Z     1000a3f3 f   libucrt:per_thread_data.obj
 0001:00009414       ?destroy_ptd@@YAXQAU__acrt_ptd@@@Z 1000a414 f   libucrt:per_thread_data.obj
 0001:000094bd       ?replace_current_thread_locale_nolock@@YAXQAU__acrt_ptd@@QAU__crt_locale_data@@@Z 1000a4bd f   libucrt:per_thread_data.obj
 0001:0000979f       ??$common_tox_l@$1?internal_isupper_l@@YA_NHQAU__crt_locale_pointers@@@Z$1?internal_map_lower@@YAHH0@Z@@YAHHKQAU__crt_locale_pointers@@@Z 1000a79f f   libucrt:tolower_toupper.obj
 0001:000098e9       ?internal_isupper_l@@YA_NHQAU__crt_locale_pointers@@@Z 1000a8e9 f   libucrt:tolower_toupper.obj
 0001:00009d2d       ?fp_format_a@@YAHQBNPADIQADIH_NIQAU__crt_locale_pointers@@@Z 1000ad2d f   libucrt:cvt.obj
 0001:0000a030       ?fp_format_e@@YAHQBNQADI1IH_NIQAU__crt_locale_pointers@@@Z 1000b030 f   libucrt:cvt.obj
 0001:0000a0cb       ?fp_format_e_internal@@YAHQADIH_NIQAU_strflt@@1QAU__crt_locale_pointers@@@Z 1000b0cb f   libucrt:cvt.obj
 0001:0000a216       ?fp_format_f@@YAHQBNQADI1IHQAU__crt_locale_pointers@@@Z 1000b216 f   libucrt:cvt.obj
 0001:0000a2a3       ?fp_format_f_internal@@YAHQADIHQAU_strflt@@_NQAU__crt_locale_pointers@@@Z 1000b2a3 f   libucrt:cvt.obj
 0001:0000a37a       ?fp_format_g@@YAHQBNQADI1IH_NIQAU__crt_locale_pointers@@@Z 1000b37a f   libucrt:cvt.obj
 0001:0000a442       ?fp_format_nan_or_infinity@@YAHW4__acrt_fp_class@@_NPADI1@Z 1000b442 f   libucrt:cvt.obj
 0001:0000a53a       ?shift_bytes@@YAXQADI0H@Z  1000b53a f   libucrt:cvt.obj
 0001:0000a82f       ?initialize_inherited_file_handles_nolock@@YAXXZ 1000b82f f   libucrt:ioinit.obj
 0001:0000a8e5       ?initialize_stdio_handles_nolock@@YAXXZ 1000b8e5 f   libucrt:ioinit.obj
 0001:0000aabd       ?try_get_function@@YAPAXW4function_id@?A0x352e5c4b@@QBDQBW4module_id@2@2@Z 1000babd f   libucrt:winapi_thunks.obj
 0001:0000ab59       ?try_get_module@@YAPAUHINSTANCE__@@W4module_id@?A0x352e5c4b@@@Z 1000bb59 f   libucrt:winapi_thunks.obj
 0001:0000afb5       ?<helper_func_cdecl>@<lambda_62bb7ecb46d0a77b591a051c43eb5ad1>@@CAHPBX0@Z 1000bfb5 f   libucrt:argv_wildcards.obj
 0001:0000afcd       ??$common_expand_argv_wildcards@D@@YAHQAPADQAPAPAD@Z 1000bfcd f   libucrt:argv_wildcards.obj
 0001:0000b15d       ??$copy_and_add_argument_to_buffer@D@@YAHQBD0IAAV?$argument_list@D@?A0xb0e4b824@@@Z 1000c15d f   libucrt:argv_wildcards.obj
 0001:0000b1f3       ??$expand_argument_wildcards@D@@YAHQAD0AAV?$argument_list@D@?A0xb0e4b824@@@Z 1000c1f3 f   libucrt:argv_wildcards.obj
 0001:0000b4ce       ??R<lambda_ad1ced32f4ac17aa236e5ef05d6b3b7c>@@QBEXXZ 1000c4ce f   libucrt:mbctype.obj
 0001:0000b592       ?CPtoLocaleName@@YAPB_WH@Z 1000c592 f   libucrt:mbctype.obj
 0001:0000b5d0       ?getSystemCP@@YAHH@Z       1000c5d0 f   libucrt:mbctype.obj
 0001:0000b643       ?setSBCS@@YAXPAU__crt_multibyte_data@@@Z 1000c643 f   libucrt:mbctype.obj
 0001:0000b6a8       ?setSBUpLow@@YAXPAU__crt_multibyte_data@@@Z 1000c6a8 f   libucrt:mbctype.obj
 0001:0000b83c       ?setmbcp_internal@@YAHH_N@Z 1000c83c f   libucrt:mbctype.obj
 0001:0000bbee       _memcpy_s                  1000cbee f   libucrt:cfout.obj
 0001:0000bbee       _memcpy_s                  1000cbee f   libucrt:mbctype.obj
 0001:0000bc6f       ?x_ismbbtype_l@@YAHPAU__crt_locale_pointers@@IHH@Z 1000cc6f f   libucrt:ismbbyte.obj
 0001:0000bcf9       ?find_end_of_double_null_terminated_sequence@@YAPB_WQB_W@Z 1000ccf9 f   libucrt:get_environment_from_os.obj
 0001:0000c042       ?get_global_action_nolock@@YAPAP6AXH@ZH@Z 1000d042 f   libucrt:signal.obj
 0001:0000c084       ?siglookup@@YAPAU__crt_signal_action_t@@HQAU1@@Z 1000d084 f   libucrt:signal.obj
 0001:0000c9f3       ?free_crt_array_internal@@YAXQAPBXI@Z 1000d9f3 f   libucrt:inittime.obj
 0001:0000cb13       ?__acrt_LCMapStringA_stat@@YAHPAU__crt_locale_pointers@@PB_WKPBDHPADHHH@Z 1000db13 f   libucrt:lcmapstringa.obj
 0001:0000e810       _common_flush_all          1000f810 f   libucrt:fflush.obj
 0001:0000ec04       ?GetTableIndexFromLocaleName@@YAHPB_W@Z 1000fc04 f   libucrt:lcidtoname_downlevel.obj
 0001:0000ecf0       ?shortsort@@YAXPAD0IP6AHPBX1@Z@Z 1000fcf0 f   libucrt:qsort.obj
 0001:0000ed90       ?swap@@YAXPAD0I@Z          1000fd90 f   libucrt:qsort.obj
 0001:0000f16a       ??$common_tcsncpy_s@D@@YAHQADIQBDI@Z 1001016a f   libucrt:strncpy_s.obj
 0001:0000f230       $$000000                   10010230     libucrt:strpbrk.obj
 0001:0000f314       ?initialize_multibyte@@YAHXZ 10010314 f   libucrt:multibyte_initializer.obj
 0001:0000f490       $$000000                   10010490     libucrt:log10.obj
 0001:0000f5e0       $$000000                   100105e0     libucrt:ceil_pentium4.obj
 0001:0000f6fd       ?write_double_translated_ansi_nolock@@YA?AUwrite_result@?A0x47fa6670@@HQBDI@Z 100106fd f   libucrt:write.obj
 0001:0000f8b0       ?write_double_translated_unicode_nolock@@YA?AUwrite_result@?A0x47fa6670@@QBDI@Z 100108b0 f   libucrt:write.obj
 0001:0000f91d       ?write_requires_double_translation_nolock@@YA_NH@Z 1001091d f   libucrt:write.obj
 0001:0000f993       ?write_text_ansi_nolock@@YA?AUwrite_result@?A0x47fa6670@@HQBDI@Z 10010993 f   libucrt:write.obj
 0001:0000fa72       ?write_text_utf16le_nolock@@YA?AUwrite_result@?A0x47fa6670@@HQBDI@Z 10010a72 f   libucrt:write.obj
 0001:0000fb60       ?write_text_utf8_nolock@@YA?AUwrite_result@?A0x47fa6670@@HQBDI@Z 10010b60 f   libucrt:write.obj
 0001:0000ff84       ??$common_lseek_nolock@_J@@YA_JH_JH@Z 10010f84 f   libucrt:lseek.obj
 0001:00010248       ___get_abstract_control_sse2 10011248 f   libucrt:_fenvutils.obj
 0001:000102c5       ___get_abstract_control_x87 100112c5 f   libucrt:_fenvutils.obj
 0001:00010338       ___get_machine_control     10011338 f   libucrt:_fenvutils.obj
 0001:000103a9       ___get_machine_control_sse2 100113a9 f   libucrt:_fenvutils.obj
 0001:00010429       ___get_machine_status_sse2 10011429 f   libucrt:_fenvutils.obj
 0001:0001048a       ___get_machine_status_x87  1001148a f   libucrt:_fenvutils.obj
 0001:000107d0       $$000000                   100117d0     libucrt:log10_pentium4.obj
 0001:00010a60       $$000000                   10011a60     libucrt:87tran.obj
 0001:00010c60       $$000000                   10011c60     libucrt:87disp.obj
 0001:00010e60       $$000000                   10011e60     libucrt:common.obj
 0001:00010ff0       $$000000                   10011ff0     libucrt:genexcep.obj
 0001:00011560       $$000000                   10012560     libucrt:_strnicm.obj
 0001:00012380       $$000000                   10013380     LIBCMT:ulldvrm.obj
 0001:00012420       $$000000                   10013420     LIBCMT:llmul.obj
 0001:00012460       $$000000                   10013460     LIBCMT:_sehprolg4gs_.obj
 0001:000124c0       $$000000                   100134c0     LIBCMT:lldvrm.obj
 0001:000125a0       $$000000                   100135a0     LIBCMT:ullshr.obj
 0001:000125c0       $$000000                   100135c0     LIBCMT:alloca16.obj
 0001:000125f0       $$000000                   100135f0     LIBCMT:llshl.obj
 0001:00012610       $$000000                   10013610     LIBCMT:_ftol2_.obj
 0001:000126d0       $$000000                   100136d0     libvcruntime:strrchr.obj
 0001:00012810       $$000000                   10013810     libvcruntime:strchr.obj
 0002:0000073c       _GS_ExceptionPointers      1001473c     LIBCMT:gs_report.obj
 0002:00000748       ?tokenTable@@3QBQBDB       10014748     libvcruntime:undname.obj
 0002:00000784       ?rttiTable@@3QBQBDB        10014784     libvcruntime:undname.obj
 0002:00000798       ?nameTable@@3QBQBDB        10014798     libvcruntime:undname.obj
 0002:00000ecc       ?module_names@?A0x9a4b7766@@3QBQB_WB 10014ecc     libvcruntime:winapi_downlevel.obj
 0002:00000f84       ?candidate_modules@?1??try_get_FlsAlloc@@YAP6GKP6GXPAX@Z@ZXZ@4QBW4module_id@?A0x9a4b7766@@B 10014f84     libvcruntime:winapi_downlevel.obj
 0002:00000f98       ?candidate_modules@?1??try_get_FlsFree@@YAP6GHK@ZXZ@4QBW4module_id@?A0x9a4b7766@@B 10014f98     libvcruntime:winapi_downlevel.obj
 0002:00000fa8       ?candidate_modules@?1??try_get_FlsGetValue@@YAP6GPAXK@ZXZ@4QBW4module_id@?A0x9a4b7766@@B 10014fa8     libvcruntime:winapi_downlevel.obj
 0002:00000fbc       ?candidate_modules@?1??try_get_FlsSetValue@@YAP6GHKPAX@ZXZ@4QBW4module_id@?A0x9a4b7766@@B 10014fbc     libvcruntime:winapi_downlevel.obj
 0002:00000fd0       ?candidate_modules@?1??try_get_InitializeCriticalSectionEx@@YAP6GHPAU_RTL_CRITICAL_SECTION@@KK@ZXZ@4QBW4module_id@?A0x9a4b7766@@B 10014fd0     libvcruntime:winapi_downlevel.obj
 0002:00001138       ___acrt_initializers       10015138     libucrt:initialization.obj
 0002:000011b0       _errtable                  100151b0     libucrt:errno.obj
 0002:00002030       _module_names              10016030     libucrt:winapi_thunks.obj
 0002:000024e4       ?candidate_modules@?1??try_get_FlsAlloc@@YAP6GKP6GXPAX@Z@ZXZ@4QBW4module_id@?A0x352e5c4b@@B 100164e4     libucrt:winapi_thunks.obj
 0002:000024ec       ?candidate_modules@?1??try_get_FlsFree@@YAP6GHK@ZXZ@4QBW4module_id@?A0x352e5c4b@@B 100164ec     libucrt:winapi_thunks.obj
 0002:000024f4       ?candidate_modules@?1??try_get_FlsGetValue@@YAP6GPAXK@ZXZ@4QBW4module_id@?A0x352e5c4b@@B 100164f4     libucrt:winapi_thunks.obj
 0002:000024fc       ?candidate_modules@?1??try_get_FlsSetValue@@YAP6GHKPAX@ZXZ@4QBW4module_id@?A0x352e5c4b@@B 100164fc     libucrt:winapi_thunks.obj
 0002:00002504       ?candidate_modules@?1??try_get_GetCurrentPackageId@@YAP6GJPAIPAE@ZXZ@4QBW4module_id@?A0x352e5c4b@@B 10016504     libucrt:winapi_thunks.obj
 0002:00002520       ?candidate_modules@?1??try_get_InitializeCriticalSectionEx@@YAP6GHPAU_RTL_CRITICAL_SECTION@@KK@ZXZ@4QBW4module_id@?A0x352e5c4b@@B 10016520     libucrt:winapi_thunks.obj
 0002:00002528       ?candidate_modules@?1??try_get_LCMapStringEx@@YAP6GHPB_WK0HPA_WHPAU_nlsversioninfo@@PAXJ@ZXZ@4QBW4module_id@?A0x352e5c4b@@B 10016528     libucrt:winapi_thunks.obj
 0002:00002540       ?candidate_modules@?1??try_get_LocaleNameToLCID@@YAP6GKPB_WK@ZXZ@4QBW4module_id@?A0x352e5c4b@@B 10016540     libucrt:winapi_thunks.obj
 0002:0000255c       __mb_locale_names          1001655c     libucrt:mbctype.obj
 0002:00002f90       _LcidToLocaleNameTable     10016f90     libucrt:lcidtoname_downlevel.obj
 0002:000040b0       _LocaleNameToIndexTable    100180b0     libucrt:lcidtoname_downlevel.obj
 0002:00005000       LOG_name                   10019000     libucrt:log10.obj
 0002:00005010       _One                       10019010     libucrt:ceil_pentium4.obj
 0002:00005020       _Bns                       10019020     libucrt:ceil_pentium4.obj
 0002:00005030       _Zero                      10019030     libucrt:ceil_pentium4.obj
 0002:00005040       _S                         10019040     libucrt:ceil_pentium4.obj
 0002:00005050       _NegZero                   10019050     libucrt:ceil_pentium4.obj
 0002:00005060       emask                      10019060     libucrt:log10_pentium4.obj
 0002:00005070       CC                         10019070     libucrt:log10_pentium4.obj
 0002:00005080       Magic                      10019080     libucrt:log10_pentium4.obj
 0002:00005090       hi_mask                    10019090     libucrt:log10_pentium4.obj
 0002:000050a0       LOG10_2                    100190a0     libucrt:log10_pentium4.obj
 0002:000050b0       place_L                    100190b0     libucrt:log10_pentium4.obj
 0002:000050d0       One                        100190d0     libucrt:log10_pentium4.obj
 0002:000050e0       Zero                       100190e0     libucrt:log10_pentium4.obj
 0002:000050f0       Two52                      100190f0     libucrt:log10_pentium4.obj
 0002:00005100       Infs                       10019100     libucrt:log10_pentium4.obj
 0002:00005110       NaN                        10019110     libucrt:log10_pentium4.obj
 0002:00005120       coeff                      10019120     libucrt:log10_pentium4.obj
 0002:0000517e       _log2max                   1001917e     libucrt:87tran.obj
 0002:00005188       _smallarg                  10019188     libucrt:87tran.obj
 0002:00005192       _half                      10019192     libucrt:87tran.obj
 0002:000051de       One                        100191de     libucrt:87disp.obj
 0002:000051e6       Three                      100191e6     libucrt:87disp.obj
 0002:000051ee       XAMtoTagTab                100191ee     libucrt:87disp.obj
 0002:00005200       One                        10019200     libucrt:common.obj
 0002:00005214       DblMax                     10019214     libucrt:common.obj
 0002:0000521c       DblMin                     1001921c     libucrt:common.obj
 0002:00005224       IeeeAdjO                   10019224     libucrt:common.obj
 0002:0000522c       IeeeAdjU                   1001922c     libucrt:common.obj
 0002:00005234       _infinity                  10019234     libucrt:common.obj
 0002:0000523c       _zero                      1001923c     libucrt:common.obj
 0002:00005278       _over                      10019278     libucrt:fpctrl.obj
 0002:00005284       _under                     10019284     libucrt:fpctrl.obj
 0002:00005b48       ?_names@?1??_get_fname@@9@9 10019b48     libucrt:fpexcept.obj
 0002:00006068       __sehtable$?dllmain_crt_process_attach@@YAHQAUHINSTANCE__@@QAX@Z 1001a068     LIBCMT:dll_dllmain.obj
 0002:00006088       __sehtable$?dllmain_crt_process_detach@@YAH_N@Z 1001a088     LIBCMT:dll_dllmain.obj
 0002:000060a8       __sehtable$?dllmain_dispatch@@YAHQAUHINSTANCE__@@KQAX@Z 1001a0a8     LIBCMT:dll_dllmain.obj
 0002:000060c8       __sehtable$___scrt_is_nonwritable_in_current_image 1001a0c8     LIBCMT:utility.obj
 0002:000060e8       __sehtable$___DestructExceptionObject 1001a0e8     libvcruntime:ehhelpers.obj
 0002:00006108       __sehtable$?common_exit@@YAXHW4_crt_exit_cleanup_mode@@W4_crt_exit_return_mode@@@Z 1001a108     libucrt:exit.obj
 0002:00006130       __sehtable$??$?RV<lambda_995298e7d72eb4c2aab26c0585b3abe5>@@AAV<lambda_275893d493268fdec8709772e3fcec0e>@@V<lambda_293819299cbf9a7022e18b56a874bb5c>@@@?$__crt_seh_guarded_call@H@@QAEH$$QAV<lambda_995298e7d72eb4c2aab26c0585b3abe5>@@AAV<lambda_275893d493268fdec8709772e3fcec0e>@@$$QAV<lambda_293819299cbf9a7022e18b56a874bb5c>@@@Z 1001a130     libucrt:onexit.obj
 0002:00006150       __sehtable$_terminate      1001a150     libucrt:terminate.obj
 0002:00006170       __sehtable$??$?RV<lambda_9df27f884b057bc3edfc946cb5b7cf47>@@AAV<lambda_e69574bed617af4e071282c136b37893>@@V<lambda_cc0d902bcbbeb830f749456577db4721>@@@?$__crt_seh_guarded_call@X@@QAEX$$QAV<lambda_9df27f884b057bc3edfc946cb5b7cf47>@@AAV<lambda_e69574bed617af4e071282c136b37893>@@$$QAV<lambda_cc0d902bcbbeb830f749456577db4721>@@@Z 1001a170     libucrt:per_thread_data.obj
 0002:00006190       __sehtable$??$?RV<lambda_3518db117f0e7cdb002338c5d3c47b6c>@@AAV<lambda_b2ea41f6bbb362cd97d94c6828d90b61>@@V<lambda_abdedf541bb04549bc734292b4a045d4>@@@?$__crt_seh_guarded_call@X@@QAEX$$QAV<lambda_3518db117f0e7cdb002338c5d3c47b6c>@@AAV<lambda_b2ea41f6bbb362cd97d94c6828d90b61>@@$$QAV<lambda_abdedf541bb04549bc734292b4a045d4>@@@Z 1001a190     libucrt:per_thread_data.obj
 0002:000061b0       __sehtable$??$?RV<lambda_51b6e8b1eb166f2a3faf91f424b38130>@@AAV<lambda_6250bd4b2a391816dd638c3bf72b0bcb>@@V<lambda_0b5a4a3e68152e1d9b943535f5f47bed>@@@?$__crt_seh_guarded_call@X@@QAEX$$QAV<lambda_51b6e8b1eb166f2a3faf91f424b38130>@@AAV<lambda_6250bd4b2a391816dd638c3bf72b0bcb>@@$$QAV<lambda_0b5a4a3e68152e1d9b943535f5f47bed>@@@Z 1001a1b0     libucrt:per_thread_data.obj
 0002:000061d0       __sehtable$??$?RV<lambda_5b71d36f03204c0beab531769a5b5694>@@AAV<lambda_be2b3da3f62db62e9dad5dc70221a656>@@V<lambda_8f9ce462984622f9bf76b59e2aaaf805>@@@?$__crt_seh_guarded_call@X@@QAEX$$QAV<lambda_5b71d36f03204c0beab531769a5b5694>@@AAV<lambda_be2b3da3f62db62e9dad5dc70221a656>@@$$QAV<lambda_8f9ce462984622f9bf76b59e2aaaf805>@@@Z 1001a1d0     libucrt:per_thread_data.obj
 0002:000061f0       __sehtable$___acrt_uninitialize_locale 1001a1f0     libucrt:wsetlocale.obj
 0002:00006210       __sehtable$___acrt_initialize_lowio 1001a210     libucrt:ioinit.obj
 0002:00006230       __sehtable$___acrt_update_thread_multibyte_data 1001a230     libucrt:mbctype.obj
 0002:00006250       __sehtable$??$?RV<lambda_978dc153c237d78434369da87b74ff60>@@AAV<lambda_ad1ced32f4ac17aa236e5ef05d6b3b7c>@@V<lambda_4a8533e2866a575feecb8298ce776b0d>@@@?$__crt_seh_guarded_call@X@@QAEX$$QAV<lambda_978dc153c237d78434369da87b74ff60>@@AAV<lambda_ad1ced32f4ac17aa236e5ef05d6b3b7c>@@$$QAV<lambda_4a8533e2866a575feecb8298ce776b0d>@@@Z 1001a250     libucrt:mbctype.obj
 0002:00006270       __sehtable$__query_new_handler 1001a270     libucrt:new_handler.obj
 0002:00006290       __sehtable$_raise          1001a290     libucrt:signal.obj
 0002:000062b0       __sehtable$??$?RV<lambda_a048d3beccc847880fc8490e18b82769>@@AAV<lambda_ec61778202f4f5fc7e7711acc23c3bca>@@V<lambda_f7496a158712204296dd6628a163878e>@@@?$__crt_seh_guarded_call@P6AXH@Z@@QAEP6AXH@Z$$QAV<lambda_a048d3beccc847880fc8490e18b82769>@@AAV<lambda_ec61778202f4f5fc7e7711acc23c3bca>@@$$QAV<lambda_f7496a158712204296dd6628a163878e>@@@Z 1001a2b0     libucrt:signal.obj
 0002:000062d0       __sehtable$___acrt_update_thread_locale_data 1001a2d0     libucrt:locale_refcounting.obj
 0002:000062f0       __sehtable$__fcloseall     1001a2f0     libucrt:closeall.obj
 0002:00006310       __sehtable$_common_flush_all 1001a310     libucrt:fflush.obj
 0002:00006338       __sehtable$___acrt_lowio_ensure_fh_exists 1001a338     libucrt:osfinfo.obj
 0002:00006358       __sehtable$__write         1001a358     libucrt:write.obj
 0002:00006378       __sehtable$_fclose         1001a378     libucrt:fclose.obj
 0002:00006398       __sehtable$??$?RV<lambda_61cee617f5178ae960314fd4d05640a0>@@AAV<lambda_6978c1fb23f02e42e1d9e99668cc68aa>@@V<lambda_9cd88cf8ad10232537feb2133f08c833>@@@?$__crt_seh_guarded_call@H@@QAEH$$QAV<lambda_61cee617f5178ae960314fd4d05640a0>@@AAV<lambda_6978c1fb23f02e42e1d9e99668cc68aa>@@$$QAV<lambda_9cd88cf8ad10232537feb2133f08c833>@@@Z 1001a398     libucrt:commit.obj
 0002:000063b8       __sehtable$??$?RV<lambda_123407a5e2ac06da108355a851863b7a>@@AAV<lambda_2fe9b910cf3cbf4a0ab98a02ba45b3ec>@@V<lambda_ae55bdf541ad94d75914d381c370e64d>@@@?$__crt_seh_guarded_call@H@@QAEH$$QAV<lambda_123407a5e2ac06da108355a851863b7a>@@AAV<lambda_2fe9b910cf3cbf4a0ab98a02ba45b3ec>@@$$QAV<lambda_ae55bdf541ad94d75914d381c370e64d>@@@Z 1001a3b8     libucrt:close.obj
 0002:000063d8       __sehtable$__IsNonwritableInCurrentImage 1001a3d8     LIBCMT:pesect.obj
 0002:00006400       .edata                     1001a400     ConEmuLn.exp
 0002:00006428       rgpv                       1001a428     ConEmuLn.exp
 0002:00006464       rgszName                   1001a464     ConEmuLn.exp
 0002:000064a0       rgwOrd                     1001a4a0     ConEmuLn.exp
 0002:000064be       szName                     1001a4be     ConEmuLn.exp
 0002:000064cb       $N00001                    1001a4cb     ConEmuLn.exp
 0002:000064da       $N00002                    1001a4da     ConEmuLn.exp
 0002:000064e9       $N00003                    1001a4e9     ConEmuLn.exp
 0002:000064ef       $N00004                    1001a4ef     ConEmuLn.exp
 0002:000064f9       $N00005                    1001a4f9     ConEmuLn.exp
 0002:00006504       $N00006                    1001a504     ConEmuLn.exp
 0002:0000650c       $N00007                    1001a50c     ConEmuLn.exp
 0002:00006515       $N00008                    1001a515     ConEmuLn.exp
 0002:00006524       $N00009                    1001a524     ConEmuLn.exp
 0002:00006535       $N00010                    1001a535     ConEmuLn.exp
 0002:00006547       $N00011                    1001a547     ConEmuLn.exp
 0002:00006555       $N00012                    1001a555     ConEmuLn.exp
 0002:00006560       $N00013                    1001a560     ConEmuLn.exp
 0002:0000656c       $N00014                    1001a56c     ConEmuLn.exp
 0002:0000657b       $N00015                    1001a57b     ConEmuLn.exp
 0002:000067ca       .idata$6                   1001a7ca     version:VERSION.dll
 0002:0000686c       .idata$6                   1001a86c     kernel32:KERNEL32.dll
 0002:0000689e       .idata$6                   1001a89e     user32:USER32.dll
 0002:00006900       .idata$6                   1001a900     gdi32:GDI32.dll
 0002:00006960       .idata$6                   1001a960     advapi32:ADVAPI32.dll
 0003:00000150       ?__vcrt_flsindex@@3KA      1001b150     libvcruntime:per_thread_data.obj
 0003:00000174       _errno_no_memory           1001b174     libucrt:errno.obj
 0003:00000178       _doserrno_no_memory        1001b178     libucrt:errno.obj
 0003:00000180       ___acrt_flsindex           1001b180     libucrt:per_thread_data.obj
 0003:000002f8       ___rgctypeflag             1001b2f8     libucrt:mbctype.obj
 0003:00000300       ___rgcode_page_info        1001b300     libucrt:mbctype.obj
 0003:000008cc       ?gfRegisterBackground@@3P6GHPAURegisterBackgroundArg@@@ZA 1001b8cc     ConEmuLn.obj
 0003:000008d0       ?bWasRegistered@?1??StartPlugin@@YAXH@Z@4_NA 1001b8d0     ConEmuLn.obj
 0003:000008dc       ?szMenu@?1??GetPluginInfoW1900@@YAXPAX@Z@4PAPA_WA 1001b8dc     ConEmuLn1900.obj
 0003:000008e0       ?szMenu1@?1??GetPluginInfoW1900@@YAXPAX@Z@4PA_WA 1001b8e0     ConEmuLn1900.obj
 0003:00000ae8       ?szMenu@?1??GetPluginInfoW2800@@YAXPAX@Z@4PAPA_WA 1001bae8     ConEmuLn2800.obj
 0003:00000af0       ?szMenu1@?1??GetPluginInfoW2800@@YAXPAX@Z@4PA_WA 1001baf0     ConEmuLn2800.obj
 0003:00000cf8       ?gszRootKeyW995@@3PA_WA    1001bcf8     ConEmuLn995.obj
 0003:00000cfc       ?szMenu@?1??GetPluginInfoW995@@YAXPAX@Z@4PAPA_WA 1001bcfc     ConEmuLn995.obj
 0003:00000d00       ?szMenu1@?1??GetPluginInfoW995@@YAXPAX@Z@4PA_WA 1001bd00     ConEmuLn995.obj
 0003:00000f08       ?gszRootKeyA@@3PA_WA       1001bf08     ConEmuLnA.obj
 0003:00000f0c       ?szMenu@?1??GetPluginInfo@@9@4@4PAPADA 1001bf0c     ConEmuLnA.obj
 0003:00000f10       ?szMenu1@?1??GetPluginInfo@@9@4@4PADA 1001bf10     ConEmuLnA.obj
 0003:00001020       ?__proc_attached@@3HA      1001c020     LIBCMT:dll_dllmain.obj
 0003:00001028       _GS_ExceptionRecord        1001c028     LIBCMT:gs_report.obj
 0003:00001078       _GS_ContextRecord          1001c078     LIBCMT:gs_report.obj
 0003:00001358       ?module_local_atexit_table@@3U_onexit_table_t@@A 1001c358     LIBCMT:utility.obj
 0003:00001364       ?module_local_at_quick_exit_table@@3U_onexit_table_t@@A 1001c364     LIBCMT:utility.obj
 0003:00001370       ?module_local_atexit_table_initialized@@3_NA 1001c370     LIBCMT:utility.obj
 0003:0000137c       ?is_initialized_as_dll@@3_NA 1001c37c     LIBCMT:utility.obj
 0003:000013b4       ?heap@@3V_HeapManager@@A   1001c3b4     libvcruntime:undname.obj
 0003:000013c8       ?__vcrt_startup_thread_ptd@@3U__vcrt_ptd@@A 1001c3c8     libvcruntime:per_thread_data.obj
 0003:000013f0       ___vcrt_lock_table         1001c3f0     libvcruntime:locks.obj
 0003:00001408       ___vcrt_locks_initialized  1001c408     libvcruntime:locks.obj
 0003:0000140c       ?module_handles@@3PAPAUHINSTANCE__@@A 1001c40c     libvcruntime:winapi_downlevel.obj
 0003:00001418       ?encoded_function_pointers@@3PAPAXA 1001c418     libvcruntime:winapi_downlevel.obj
 0003:00001434       _c_termination_complete    1001c434     libucrt:exit.obj
 0003:00001438       _thread_local_exit_callback_func 1001c438     libucrt:exit.obj
 0003:0000143c       ?c_exit_complete@?5??common_exit@@YAXHW4_crt_exit_cleanup_mode@@W4_crt_exit_return_mode@@@Z@4_NA 1001c43c     libucrt:exit.obj
 0003:00001440       ?program_name@?5???$common_configure_argv@D@@YAHW4_crt_argv_mode@@@Z@4PADA 1001c440     libucrt:argv_parsing.obj
 0003:00001570       ___acrt_invalid_parameter_handler 1001c570     libucrt:invalid_parameter.obj
 0003:00001584       _enable_percent_n          1001c584     libucrt:printf_count_output.obj
 0003:00001798       ___acrt_lock_table         1001c798     libucrt:locks.obj
 0003:000018d0       ___acrt_locks_initialized  1001c8d0     libucrt:locks.obj
 0003:000018d8       _module_handles            1001c8d8     libucrt:winapi_thunks.obj
 0003:00001928       _encoded_function_pointers 1001c928     libucrt:winapi_thunks.obj
 0003:000019a8       ?state_cache@?1??__acrt_is_packaged_app@@9@4JA 1001c9a8     libucrt:winapi_thunks.obj
 0003:000019c4       _fSystemSet                1001c9c4     libucrt:mbctype.obj
 0003:000019c8       ?initialized@?1??__acrt_initialize_multibyte@@9@4_NA 1001c9c8     libucrt:mbctype.obj
 0003:000019e8       ___acrt_new_handler        1001c9e8     libucrt:new_handler.obj
 0003:000019ec       _ctrlc_action              1001c9ec     libucrt:signal.obj
 0003:000019f0       _ctrlbreak_action          1001c9f0     libucrt:signal.obj
 0003:000019f4       _abort_action              1001c9f4     libucrt:signal.obj
 0003:000019f8       _term_action               1001c9f8     libucrt:signal.obj
 0003:000019fc       _user_matherr              1001c9fc     libucrt:matherr.obj
 0003:00001a08       ___acrt_global_new_mode    1001ca08     libucrt:new_mode.obj
 0003:00001a0c       ___acrt_app_type           1001ca0c     libucrt:report_runtime_error.obj
 0003:00001a14       __pmatherr_set             1001ca14     libucrt:libm_error.obj
 0004:000000a0       $R000000                   1001d0a0     ConEmuLn.res
 0004:000003b8       $R000318                   1001d3b8     ConEmuLn.res
